:100000000C94A50C0C94E79A0C94BC9A0C94919ABD
:100010000C94669A0C943B9A0C94109A0C94E59963
:100020000C94BA990C94D60C0C94D60C0C94D60C57
:100030000C94D60C0C94D60C0C94D60C0C945577CE
:100040000C94D60C0C94D60C0C94D60C0C94D60CA8
:100050000C94D60C0C94D60C0C94D60C0C941E99C3
:100060000C94D60C0C942A9D0C94009D0C94D60CE8
:100070000C94D60C0C94D60C0C94D60C0C94D60C78
:100080000C94D60C0C94D60C0C94D60C0C94D60C68
:100090000C9417950C9487940C94CE940C94DC6675
:1000A0000C94D60C0C94D60C0C94D60C0C94D60C48
:1000B0000C94D60C0C94D60C0C94D60C0C94D60C38
:1000C0000C94D60C0C94D60C0C94D60C0C94D69C98
:1000D0000C94AC9C0C94D60C0C94829C0C94589C64
:1000E0000C94D60CF510BF11D8120E130E13EF128C
:1000F000B5110E130E130E13BF11BF11BF117A11DC
:1001000011111E117A117A119C11AC111E119C1142
:100110007A11381222122212381238124512501255
:10012000191238123812A71DC41DF41DFC1DFF1D25
:10013000F41DD31DF41D091E0C1EE31D171E1A1EEF
:10014000A8238323C323C323C323C323C323C323DA
:10015000C323C323C3230920DC220123EB22FA2279
:10016000C323C323C323C323C323C323C32397238B
:100170009F29932993299F299F297A2987298729AC
:100180009F299F293D2C9C2D6C2C8A2C9C2DA72CC3
:100190009C2DD62CF42C112D442D722D072E1E2EA5
:1001A0000B2E0B2E1E2E0F2E1E2E132E132E132E45
:1001B000132E132E0B2E443B9B3A163A383A9B3A99
:1001C0009B3A383A163A9B3A9B3A9B3A713A663ACE
:1001D0005C3A873A7C3A8243714374437C437C4364
:1001E000744371437C437C437C437143714371434B
:1001F0002D482A482A482D482D482F482F48E247A5
:100200002D482D482D532D532D532D532A532A530A
:1002100031533153315331533153315331533153BE
:100220002A532A53315331533153315331532F53BE
:100230002D53D761DA61C961CD61D3611162DE618D
:10024000E261E861EC61F061F661FA61FE61116200
:10025000046208620C62A662AB62B062BA62C462F7
:100260003D63CE62D662DE62E862F262FC620B63DC
:1002700015633D631F6329633363DC96DF96F7964E
:100280000E97569769978997BCAA99AAA0AAA7AA78
:10029000AEAAC3AACAAA07634236B79BD8A71A391F
:1002A000685618AEBAAB558C1D3CB7CC5763BD6DC4
:1002B000EDFD753EF6177231BF000000803F08006B
:1002C0000000BE922449123EABAAAA2ABECDCCCCD5
:1002D0004C3E00000080BEABAAAAAA3E000000006F
:1002E000BF000000803F0000000000084178D3BB41
:1002F0004387D1133D190E3CC3BD4282AD2B3E68EE
:10030000EC8276BED98FE1A93E4C80EFFFBE01C4DE
:10031000FF7F3F00000000000C941D170C94DC963A
:100320000C94EC610C947C980C94DE620C94776DC8
:100330000C9424860C9408620C94CD610C94E247D2
:100340000C9469970C94D62C0C94F0610C947E98C4
:100350000C94C6750C94AB170C9463800C947E6659
:100360000C944D9E0C9433630C94C9610C947143AE
:100370000C94CB980C94BCAA0C94DA660C94549D03
:100380000C94CC9D0C94BA620C9415630C94171EBB
:100390000C942A530C94FA220C943C9E0C943982AF
:1003A0000C947C480C94F6970C9422120C94ED3229
:1003B0000C94939D0C94D31D0C94072E0C947948A7
:1003C0000C94E8610C947C3A0C941A1E0C94204B0B
:1003D0000C9491760C9406760C94D7610C946580FD
:1003E0000C94E2610C94B14E0C94F41D0C9476665E
:1003F0000C9411620C94069E0C94D6620C940F2EF1
:100400000C940C330C945C3A0C942A480C94CE62F5
:100410000C943C920C94FA610C9456970C94EF3225
:100420000C9474480C94112D0C945A480C94A618F2
:100430000C94A72C0C94AB620C94A6620C949C11A7
:100440000C94DE9D0C94E4750C94FD380C94442DB2
:100450000C949B3A0C9401880C947A7E0C946B75E6
:100460000C94AEAA0C94D3610C9421980C94EF12C6
:100470000C9406400C94663A0C944B920C942963AD
:100480000C94F7960C941C7F0C946C2C0C94092003
:100490000C941E110C947A110C94C03E0C94383AB2
:1004A0000C941E7D0C946E920C9462660C94AD7F3D
:1004B0000C9444980C9438120C941B4E0C942F48B6
:1004C0000C94D8120C941A1C0C940C620C94717B32
:1004D0000C945B7E0C9402390C9407400C94C79EDC
:1004E0000C94A8230C94C37D0C94EE150C949723C4
:1004F0000C94DF800C9419120C94687B0C94E01718
:100500000C9401230C94EA150C944C870C94F42C55
:100510000C9445120C943D630C9452980C94497FB2
:100520000C9473A70C940B630C942C7C0C94309853
:100530000C9487290C941B1C0C9452660C94257BFC
:100540000C9474800C942D480C942F530C942E868C
:100550000C941C800C94CA750C940F390C94478130
:100560000C9455750C943C180C94B24E0C94267B4C
:100570000C940E970C94CA800C9450120C94163A5A
:100580000C9481480C943C7B0C9474390C94FF1DA2
:100590000C94CC4A0C94132E0C9411110C940E1341
:1005A0000C94CAAA0C9483230C94A0AA0C94F63839
:1005B0000C94F2620C9451660C94DA610C947148BC
:1005C0000C94CA4A0C94714E0C940A400C947A9E76
:1005D0000C94BF110C94A37E0C94C41D0C94B77B97
:1005E0000C94A71D0C94AC110C94DF960C94407BDA
:1005F0000C9499AA0C94107D0C94FB810C94BA7AFB
:100600000C9482430C94F6610C9493290C94B511CC
:100610000C941E2E0C94713A0C94F6150C94AB6647
:100620000C942D530C9470800C94447B0C949D4836
:100630000C9466A60C9446A00C94D80C0C94F797D6
:100640000C9431530C94C3230C94091E0C94B59B49
:100650000C94707B0C9453660C94FA150C94E8621D
:100660000C94F8320C94FF4A0C940D9E0C94DE61AD
:100670000C946A9E0C94A4480C947A290C94777577
:100680000C94873A0C94FC620C947C430C94F21505
:100690000C9463160C94C4620C94D4150C94A7AA01
:1006A0000C9402400C94FE610C945D7B0C9474439A
:1006B0000C94FC1D0C9461160C94EB220C94443B9E
:1006C0000C94314C0C94A3750C945D3B0C94547BAE
:1006D0000C940C1E0C94719D0C949C2D0C94FE1586
:1006E0000C94AD800C943D2C0C9404620C94DC2290
:1006F0000C94C3AA0C94E31D0C94B0620C948A2C45
:100700000C949F290C9489970C941F630C94A19DC1
:100710000C9475750C94CE4A0C940B2E0C94722D7F
:100720000C94F5106364696E6F70737578585B0094
:100730004452590046414E5F4F4E4C5900584F4E5F
:100740000048414C54003D0050696E3A003D005055
:10075000696E3A002048616C7465640A003D00527D
:100760006573746F7265643A20003A204E6F20738F
:10077000746F7265642076616C756573202D2064DA
:10078000656661756C740A00416C726561647920FC
:100790004163746976650A005475726E696E6720EC
:1007A000584F4E0A00416C72656164792048616C53
:1007B0007465640A00416C726561647920496E61F8
:1007C00063746976650A00416C72656164792041E1
:1007D00063746976650A005475726E696E67205895
:1007E0004F4E0A00584F464620736B69707065641F
:1007F0002E205072657620636D643A005475726ED7
:100800006564206F66662066726F6D3A005265738C
:10081000746F7265642066726F6D3A00536B697015
:10082000204772700049676E6F7265642C206368A0
:10083000616E6E656C20636D643D0029003E003C76
:1008400000205061723D280020436D643D0020531C
:100850007566663D00205375623D00204974656DE4
:100860003D0052414D3D002F00496E3A20002D3E83
:10087000002000230050656E646564207374617409
:1008800065207265747269657665643A003D004C56
:10089000454741435920494E3A00736174006875D9
:1008A000650066616E006D6F646500536574436D2D
:1008B000643A00536574466C61673A00436C724653
:1008C0006C61673A002056616C3D002053746F7272
:1008D000652000737566666978436F64653A0052F7
:1008E000474200485356004C4F57004D4544495528
:1008F0004D0048494748004445435245415345004F
:10090000494E4352454153450044495341424C45A9
:100910004400454E41424C45440046414C5345003D
:100920005452554500584F464600544F47474C4592
:1009300000524553540054787432436D643A004772
:100940006F7420495020616464726573733A0027A4
:100950006970205B69705B2C646E735B2C67775BDE
:100960002C7375626E65745D5D5D5D27202D20734F
:100970006574207374617469632049500A0046618C
:10098000696C656420746F20636F6E666967757249
:10099000652045746865726E6574207573696E674D
:1009A00020444843502E20596F752063616E207398
:1009B0006574206970206D616E75616C6C792100C1
:1009C0005374617274696E67206C616E00246E6F7F
:1009D0006465730024666F726D61740024646174D1
:1009E000617479706500302D31303000696E746546
:1009F0006765720068737600636F6C6F72004F4EAC
:100A00002C4F46462C48414C542C524553542C589C
:100A10004F4E2C584F46462C544F47474C45006587
:100A20006E756D00666C6F617400322E312E300071
:100A300024686F6D696500757074696D652C6672E8
:100A400065656865617000396431356637615F32AC
:100A50003032302D30352D3037004C69676874489E
:100A600075622000246E616D6500726561647900B5
:100A70002074727920616761696E20696E2035206B
:100A80007365636F6E6473006661696C65642C20C6
:100A900072633D004177616974696E6720666F72A9
:100AA0002072657461696E656420746F7069637328
:100AB00000636F6E6E65637465642061732000204F
:100AC0002E2E2E0020757365723A003A000A41748A
:100AD00074656D7074696E67204D51545420636F56
:100AE0006E6E656374696F6E20746F20002473747A
:100AF00061746500646973636F6E6E6563746564C9
:100B0000005573696E67204D5154542070617373A2
:100B1000776F72642066726F6D20636F6E666967AF
:100B200000446576696365204E616D653A005265E3
:100B300062696E6420737563636573732E20495018
:100B400020616464726573733A004572726F723A21
:100B500020726562696E64206661696C0052656E20
:100B60006577656420737563636573732E204950E0
:100B700020616464726573733A004572726F723AF1
:100B80002072656E65776564206661696C004E6FE2
:100B9000206C696E6B00416363657074696E6720D9
:100BA000636F6D6D616E64732E2E2E0A003D0049D9
:100BB0004E3A00204E6F20656D6974206461746147
:100BC000210020436F756E74657220747970652EF4
:100BD0002076616C3D00494E3A0020436F756E747B
:100BE000657220747970652E20494E434F525245EC
:100BF000435420496E74657272757074206E756D01
:100C0000626572212121004952513A002500C2B08B
:100C10004320483D002044485432322074797065A6
:100C20002E20543D00494E3A0043757272656E7431
:100C3000204C414E20636F6E6669672869702C6492
:100C40006E732C67772C7375626E6574293A000A8F
:100C500055736520746865736520636F6D6D616E93
:100C600064733A202768656C7027202D20746869AA
:100C70007320746578740A276D61632064653A6136
:100C8000643A62653A65663A66653A3030272073A1
:100C9000657420616E642073746F7265204D4143EA
:100CA0002D6164647265737320696E2045455052EE
:100CB0004F4D0A276970205B69705B2C646E735B13
:100CC0002C67775B2C7375626E65745D5D5D5D2767
:100CD000202D2073657420737461746963204950FA
:100CE0000A277361766527202D207361766520635E
:100CF0006F6E66696720696E204E5652414D0A2715
:100D000067657427205B636F6E6669672061646442
:100D1000725D27202D2067657420636F6E6669679A
:100D20002066726F6D207072652D636F6E666967E5
:100D3000757265642055524C20616E642073746F27
:100D4000726520616464720A276C6F616427202DCC
:100D5000206C6F616420636F6E6669672066726FD6
:100D60006D204E5652414D0A2770776427202D2062
:100D7000646566696E65204D5154542070617373CB
:100D8000776F72640A276B696C6C27202D2074655D
:100D90007374207761746368646F670A27636C6596
:100DA000617227202D20636C656172204545505289
:100DB0004F4D0A277265626F6F7427202D20726570
:100DC000626F6F7420636F6E74726F6C6C6572000B
:100DD000536F6674207265626F6F74696E672E2E32
:100DE0002E00444D58696E2042756666657220611A
:100DF0006C6C6F632065727200496E697420696E55
:100E00002063683A000944533234383220657272E4
:100E10006F7200312D776972652073686F72746527
:100E2000642E0009526573657420646F6E65000955
:100E3000436865636B696E6720666F7220312D575A
:100E400069726520646576696365732E2E2E004491
:100E500053323438322D3130302070726573656E04
:100E600074004453323438325F3130305F4932439A
:100E70005F544F5F31575F42524944474520696E86
:100E800069740020416464723A00646576230052FC
:100E9000414D3D000A312D7769726520000A6D7160
:100EA000747420000A6D6F6462757320000A696EA5
:100EB0007075747320000A6974656D7320000A43AD
:100EC0006F6E666967757265643A002C003D00506C
:100ED000696E3A002C003D4C4F5700546865726DA6
:100EE0006F3A004F6E6520776972652052656164C4
:100EF000790A00444D58206F7574207374617274C0
:100F000065642E204368616E6E656C733A20004400
:100F10004D5820696E20737461727465642E20438D
:100F200068616E6E656C733A006363733831313A91
:100F30002064617461206E6F7420617661696C61F8
:100F4000626C6500636373383131206E6F742069A1
:100F50006E697469616C697A6564004C4F57004D25
:100F6000454449554D00484947480046414E5F4F6A
:100F70004E4C5900445259004845415400434F4F8C
:100F80004C004155544F007261770071756569746A
:100F9000007377696E67006C6F636B002076616C1D
:100FA0007565206973200020756E6B6E6F776E0A11
:100FB0000020696E6163746976650A00206163745C
:100FC0006976650A00204772703A0020696E616395
:100FD000746976650A00206163746976650A002089
:100FE000696E76616C6964004D6F64627573206F21
:100FF00070206661696C65640A003D0056432300F9
:1010000020636D643D003D0056435F686561742355
:10101000002D3E005075623A2000636D6400434F1E
:101020004F4C0048454154004155544F002D3E005F
:101030005075623A2000736574002D3E0050756251
:101040003A20002D3E005075623A2000556E6B6EBE
:101050006F776E20636D64200A004F4646004F4E46
:1010600000537461747573206465666665726564A7
:101070000A004E6F7420737570706F72746564200F
:1010800072656720747970650A00293A0028543A1D
:10109000003D3E00206973200044656C6574696EF4
:1010A0006720636F6E662E2052414D207761733A40
:1010B00000556E6C6F636B696E6720636F6E666957
:1010C00067202E2E2E00536B697070696E672E2E6E
:1010D000004F4F4D21005D20000A5B003A004D415A
:1010E000433A004D6F746F722074696D656F75744B
:1010F00000556E6B6E6F776E20636D64003A204E04
:101100006F2073746F7265642076616C75657320EF
:101110002D2064656661756C740A00526573746F86
:101120007265643A2000466F726365642065786575
:10113000637574696F6E002076616C3A00556E6B52
:101140006E6F776E20636D64003A204E6F2073746B
:101150006F7265642076616C756573202D206465FF
:101160006661756C740A002C002C00526573746FF4
:101170007265643A200020636D643D002D00537455
:101180006F726564204558543A00202D3E2000209F
:101190002D3E2000203A2000494E3A002C20002EFF
:1011A0000000002200250028002B002E0031003412
:1011B0000002010000050108010B0100000A0B02FA
:1011C000090C0D0E080703040100000000000000D8
:1011D000000000000000000000000000000000000F
:1011E00000000000000000121110000000000000CC
:1011F00000000000000000000000000000000000EF
:101200000053686F77002C002C006873763A20003A
:10121000312D7769726520636F756E743A200020F6
:10122000416464723A00646576230020616C6976DB
:101230006500204E6F64653A0053656172636869AA
:101240006E6700312D776972652064697361626C25
:101250006564202873686F727465642900696E0084
:10126000735F6F7574006D79686F6D6500000021A4
:1012700000240027002A002D003000330001010067
:1012800000040107010A01010210202008081020B3
:101290004010204080020102010804020101020402
:1012A00008102040808040201008040201800402C1
:1012B0000180402010080402010804020101020418
:1012C0000810204080010204081020408005050518
:1012D00005070508080808020202020A0A080804AD
:1012E00004040401010101010101010303030303DB
:1012F000030303040707070C0C0C0C0C0C0C0C026A
:1013000002020206060606060606060B0B0B0B0B70
:101310000B0B0B005EBCE2613FDD83C29C7E20A311
:10132000FD1F419DC3217FFCA2401E5F01E3BD3E26
:101330006082DC237D9FC1421CFEA0E1BF5D038073
:10134000DE3C62BEE0025CDF81633D7C22C09E1D0C
:1013500043A1FF4618FAA427799BC584DA3866E5CD
:10136000BB5907DB856739BAE406581947A5FB78EE
:1013700026C49A653BD987045AB8E6A7F91B45C627
:10138000987A24F8A6441A99C7257B3A6486D85BD4
:1013900005E7B98CD2306EEDB3510F4E10F2AC2F81
:1013A0007193CD114FADF3702ECC92D38D6F31B2BE
:1013B000EC0E50AFF1134DCE90722C6D33D18F0CDB
:1013C00052B0EE326C8ED0530DEFB1F0AE4C1291A4
:1013D000CF2D73CA947628ABF517490856B4EA693D
:1013E00037D58B5709EBB536688AD495CB2977F476
:1013F000AA4816E9B7550B88D6346A2B7597C94A9F
:1014000014F6A8742AC896154BA9F7B6E80A54D75B
:10141000896B35436F6E6E65637465642E00436F30
:101420006E6E2E2061626F72746564004C6F616431
:101430006564006C6F6164206661696C6564004E70
:101440006F2073746F72656420636F6E66696700E6
:101450004C6F6164696E6720436F6E6669672066D2
:10146000726F6D20454550524F4D000A726571757F
:10147000657374204D51545420436F6E6669670044
:10148000536176656420746F20454550524F4D007E
:10149000536176696E6720636F6E66696720746F4B
:1014A00020454550524F4D2E2E0053617665640AFB
:1014B000005365742064796E616D69632049500A38
:1014C00000454550524F4D20636C65617265640A5A
:1014D0000050617373776F72642075706461746516
:1014E000640A00636F756C64206E6F7420706172A3
:1014F00073653A2000557064617465640A002B00BE
:101500002D00485454502F312E3120256900204899
:101510005454502F312E310D0A486F73743A2025E0
:10152000730D0A4163636570743A202A2F2A0D0AED
:10153000436F6E6E656374696F6E3A20636C6F7390
:10154000650D0A0025730020000D0A004745540070
:101550006661696C656420746F20636F6E6E65638D
:10156000740A004552524F523A20536572766572A2
:101570002072657475726E65642000446F6E652E0E
:101580000A004170706C79696E672E0A00436F6EB5
:101590006669672070617273696E67206661696C45
:1015A00065640A00676F7420436F6E6669670A009E
:1015B000436F6E666967205552493A2068747470AB
:1015C0003A2F2F002044656661756C7420636F6E3E
:1015D0006669672073657276657220757365643A13
:1015E00020006C617A79686F6D652E7275002053EA
:1015F00061766564000A282B29464153544C4544C2
:10160000000A282B29535049204C4544000A282B16
:10161000294D4F544F5220435452000A282B294140
:1016200043204841494552000A282B294343533857
:10163000313120262048444331303830000A282DEB
:1016400029524553544152545F4C414E5F4F4E5FB7
:101650004D5154545F4552524F5253000A282D2980
:101660004841524452455345542C207573696E6766
:1016700020736F6674000A282B29434F554E54453A
:1016800052000A282B29444854000A282B294F5776
:10169000495245000A282B294D4F44425553000A10
:1016A000282B29444D58000A282B2944533234381A
:1016B000322D313030000A282B294672656552617F
:1016C0006D207072696E74696E6700435553544F94
:1016D0004D5F4649524D574152455F4D4143000AC7
:1016E0004669726D77617265204D414320416464A3
:1016F0007265737320006C617A79686F6D652E7204
:1017000075000A436F6E666967207365727665724D
:101710003A000A282B295741544348444F47003286
:1017200030313130334C0020432B2B2076657273DF
:10173000696F6E3A00396431356637615F32303235
:10174000302D30352D3037000A4C617A79686F6D55
:10175000652E7275204C6967687448756220636FE6
:101760006E74726F6C6C65722000757074696D6553
:1017700000667265656865617000247374617473D6
:1017800000200020000A52414D3D00202D7461725E
:10179000676574207A6F6E652D00204F46460020E5
:1017A0004F4E00204F46460020636D643A002043B0
:1017B00075723A00205365743A002045787069725A
:1017C00065640A0063637338313120697320616C8A
:1017D000726561647920696E697469616C697A65A2
:1017E00064006864633130383020697320616C7242
:1017F0006561647920696E697469616C697A656490
:101800000048444331303830206E6F7420696E696F
:101810007469616C697A6564005265747279696E85
:10182000672056432074656D7020434D440A004D77
:101830006F6462757320706F6C6C696E672065727F
:10184000726F723D002D002050492056616C203A85
:10185000004D6F6462757320706F6C6C696E6720E9
:101860006572726F723D002D0020464D2056616CEE
:10187000203A005265747279696E6720564320439E
:101880004D440A005265747279696E672064696D0F
:101890006D657220434D440A004D6F64627573207C
:1018A000706F6C6C696E67206572726F723D00209C
:1018B00056616C3A20004D423A20004E6F742073FE
:1018C0007570706F727465642072656720747970CA
:1018D000650A00496C6C6567616C20617267756DA3
:1018E000656E74730A003E3E2000496E76616C6935
:1018F0006420636F6D6D616E64003E3E3E004E6F0E
:10190000204D414320636F6E666967757265643A66
:1019100020736574206669726D7761726527732024
:101920004D41430A00000020002300260029002C1E
:10193000002F003200000100000301060109013EF2
:10194000003E003C00543A0073A711241FBECFEFA5
:10195000D1E2DEBFCDBF00E00CBF19E0A0E0B2E0F5
:10196000E6ECF5E701E00BBF02C007900D92AC3644
:10197000B107D9F721E1ACE6B9E001C01D92A73368
:10198000B207E1F71CE0C5EADCE000E006C0219701
:101990000109802FFE010E94D8B5C43AD10780E02A
:1019A0000807A9F70E9418A90C94E1BA0C9400004A
:1019B0002F923F924F925F926F927F928F929F925F
:1019C000AF92BF92CF92DF92EF92FF920F931F934D
:1019D000CF93DF93CDB7DEB7AC970FB6F894DEBFE9
:1019E0000FBECDBF5C012B015BA34AA33DA32CA37B
:1019F000102F1701D9A2C8A2EC2DFD2D309719F098
:101A00008081811114C0D5011D968C91882321F00D
:101A1000C5010D9699A388A321143104A1F4E8A16E
:101A2000F9A1309731F4F5012788308C0CC0EF28EC
:101A300051F480818823B9F3CE0180960E947018FA
:101A40001C01892B81F3C8A0D9A0D5011296ED9174
:101A5000FC911397E080F1800E944C6A3B014C019D
:101A600062E678E085E89CE00E94199B2AE030E07D
:101A7000B401A30185E89CE00E949B9B6BE578E0A4
:101A800085E89CE00E94199BB70185E89CE00E94D4
:101A90004A9C65E578E085E89CE00E94199BB601C8
:101AA00085E89CE00E944A9C6EE478E085E89CE032
:101AB0000E94199B4AE050E0B10185E89CE00E9439
:101AC0003F9C68E478E085E89CE00E94199B4AE02E
:101AD00050E0B20185E89CE00E943F9C61E478E020
:101AE00085E89CE00E94199BF50182819381892BF6
:101AF00009F4A5C01B8E1A8E1D8E1C8E1F8E1E8E85
:101B00002CA13DA12115310579F179014E013AE170
:101B1000830E911CC12CD12C8AA19BA1C816D90679
:101B20001CF593E0C916D104F9F0D7016D907D90B2
:101B30007D01F401619271924F016FE378E085E8D5
:101B40009CE00E94199B4AE050E0B30185E89CE0CC
:101B50000E943F9C6DE378E085E89CE00E94199B21
:101B6000FFEFCF1ADF0AD8CF6BE378E085E89CE07F
:101B70000E94199B85E89CE00E94469CD5011A961C
:101B80008C91873009F44FC0E8A0F9A0E114F1046A
:101B900009F458C06EE570E1C7010E94BBAC892B07
:101BA00009F486C76AE570E1C7010E94BBAC892BC6
:101BB00009F482C761E477E0C7010E94BBAC892BBE
:101BC00009F47EC76DE377E0C7010E94BBAC892BA7
:101BD00009F47AC763E270E1C7010E94BBAC892BAC
:101BE00009F476C76EE170E1C7010E94BBAC892B96
:101BF00009F472C768E270E1C7010E94BBAC892B8F
:101C000009F46EC764E377E0C7010E94BBAC892B7F
:101C100009F46AC760E377E0C7010E94BBAC892B77
:101C200009F466C70FC011110DC06CE178E085E8BA
:101C30009CE00E94199B85E89CE00E94469C8FEFE7
:101C40009FEF99C760E070E0C5010E941F1B3C0137
:101C5000C5010E9472477C01B4E04B165104B1F0FB
:101C60004CF44114510409F4C6C1F3E04F16510479
:101C700091F024C227E042165104A9F10CF41EC2CF
:101C80008AE0481651040CF462C018C218161906EE
:101C90000CF447C010C2D5011A968C91873009F414
:101CA0000DC2C5010E94FD1BC82ED12C853009F044
:101CB00044C76DE078E085E89CE00E94199B4AE00B
:101CC00050E0B60185E89CE00E943F9C85E89CE0DE
:101CD0000E94469CF5018285853009F0ECC17CE0CC
:101CE000472E512CEBC1D5011A968C91873009F4FF
:101CF000E5C1C5010E94FD1BC82ED12C8630A9F478
:101D00006CEF77E085E89CE00E94199B4AE050E088
:101D1000B60185E89CE00E943F9C85E89CE00E941B
:101D2000469C62E0462E512CC9C164EE77E085E8FE
:101D30009CE00E94199B4AE050E0B60185E89CE0D7
:101D40000E943F9C85E89CE00E94469CF6C6F501F7
:101D50000285073009F4B2C12AA13BA1232B21F04F
:101D60008A8D9B8D892B21F485E090E09B8F8A8F53
:101D700039E04316510439F48A8D9B8D91958195F4
:101D800091099B8F8A8FC5010E94051B68A77AA7BE
:101D90008BA79CA7D5011B968D919C911C970097B2
:101DA00049F0DC01ED91FC91028CF38DE02D199549
:101DB0004C0102C0802E912C08A5BAA5BCA3CBA4CF
:101DC000ECA5EF77DE2E6AEB74E085E89CE00E94DC
:101DD0004A9C4AE050E0B60185E89CE00E94A89B3E
:101DE00063EC74E085E89CE00E944A9C4AE050E085
:101DF0006AA585E89CE00E94AE9B6AEC74E085E8E9
:101E00009CE00E944A9C4AE050E068A585E89CE07E
:101E10000E94AE9B85E89CE00E94469C9401215064
:101E2000310939A728A732E02316310451F024F4F0
:101E30002114310431F039C0C1010797029760F1D4
:101E400034C08A8D9B8D800F911D8536910514F0CD
:101E500084E690E09B8F8A8F8A8D9B8D97FF02C0CE
:101E60001B8E1A8E8A8C9B8C67EC74E085E89CE054
:101E70000E944A9C4AE050E0B40185E89CE00E9440
:101E80003F9C85E89CE00E94469CA1E0B0E0BBA39B
:101E9000AAA3412C512C09C0E8A5F9A5329728F036
:101EA000F7E08F16910409F0FEC528A539A5223068
:101EB000310508F003C137E023163104D9F088E07A
:101EC0002816310419F193E02916310409F0F6C0FF
:101ED0008A8D9B8DC80ED91EDB8ECA8E8C8D9D8DF2
:101EE000ACA18A0F911D9D8F8C8F8E8D9F8D800F41
:101EF000911D17C08A8D9B8DC80ED91EDB8ECA8E90
:101F0000BCA18B2F90E09D8F8C8F09C08A8D9B8DFB
:101F1000ECA18E0F911D9D8F8C8FDB8ECA8E802F32
:101F200090E09F8F8E8F8A8D9B8D8E36914014F01E
:101F30001B8E1A8E8A8D9B8D97FF04C08DE691E0D3
:101F40009B8F8A8F8C8D9D8D8536910524F084E63C
:101F500090E09D8F8C8F8C8D9D8D97FF02C01D8E84
:101F60001C8E8E8D9F8D8536910524F084E690E041
:101F70009F8F8E8F8E8D9F8D97FF02C01F8E1E8E1E
:101F80004E8C5F8C8C8C9D8CCA8CDB8C6EEC74E0E0
:101F900085E89CE00E944A9C4AE050E0B60185E852
:101FA0009CE00E943F9C63EC74E085E89CE00E940A
:101FB0004A9C4AE050E0B40185E89CE00E943F9CC6
:101FC0006AEC74E085E89CE00E944A9C4AE050E09C
:101FD000B20185E89CE00E943F9C85E89CE00E945D
:101FE000469C52E0252E312C23E030E03BA32AA36F
:101FF000412C512C63C0D5011A969C911A979730A9
:1020000009F45CC0EAA1FBA1319709F057C01B9607
:102010000D90BC91A02D109749F0ED91FC91119776
:10202000028CF38DE02DCD01199502C0892F90E02F
:1020300001970297D8F5C5010E94051BAB01F7E097
:102040002F163104E1F028E022163104B9F52A8D6B
:102050003B8D592F5F778A8F5B8FB90177277D8FF3
:102060006C8F642F70E07F8F6E8F522FBC01C50183
:102070000E94CD1A83E090E09BA38AA31FC09A8C94
:102080008B8D8F779078792F782B852F90E09D8F8F
:102090008C8F842F90E09F8F8E8F692DC5010E94B9
:1020A000CD1AA3E0B0E0BBA3AAA308C0C101079763
:1020B000029720F442C544244394512CF5018384B3
:1020C00094848114910409F484C0F5E04F165104FE
:1020D00069F126E04216510431F032E04316510412
:1020E00009F05EC03FC0EF2809F021C567ED77E039
:1020F00085E89CE00E94199BD5011B968D919C91CF
:102100001C97C8A0D9A0DC01ED91FC910488F58949
:10211000E02D7101012F9E01265E3F4F4AA15BA178
:1021200061E070E019958C0166E0FCC41E141F0488
:10213000B4F4C8A0D9A0D401ED91FC910488F5892C
:10214000E02D7101012F9E01265E3F4F4AA15BA148
:1021500062E070E0C40119958C0165E0E3C465EBB1
:1021600077E0E7C4C5010E94FD1B8530B1F0C8A02F
:10217000D9A0D401ED91FC910488F589E02D71017D
:10218000012F9E01265E3F4F4AA15BA162E070E0F5
:10219000C40119958C0162E0C5C465EA77E0C9C441
:1021A000C8A0D9A0D401ED91FC910488F589E02D57
:1021B0007101012F9E01265E3F4F4AA15BA1B20132
:1021C000C40119958C014114510409F4AEC4642D65
:1021D000A9C4BDE04B16510408F020C2F2018827C3
:1021E000EE58FF4F8F4F0C94D8B588248394211458
:1021F000310421F01E141F040CF0812CC10107973B
:10220000029708F40BC2F501828590E08A309105AF
:1022100008F0A2C0FC018827E158FF4F8F4F0C94B3
:10222000D8B58C8D9D8D892B49F42AA13BA12330F3
:10223000310521F48FE7D5011A968C93C5010E94D0
:10224000051BD62EC72E982E092FEAA1FBA1E2303E
:10225000F105C9F0E330F10529F1319759F52A8DDF
:102260003B8DD22E97FF26C09F778A8F9B8F872F1B
:1022700090E09D8F8C8F33273F8F2E8F23E030E0AF
:102280003BA32AA317C09A8C0B8D0F779078092B4C
:10229000CC8C70E07F8F6E8F006883E090E09BA312
:1022A0008AA308C09A8C0B8D0F779078092BCC8C61
:1022B000DE8C00684D2D5C2D692D702FC5010E94AC
:1022C000CD1A2114310409F042C01E141F0424F455
:1022D000D1103DC062E005C0EF28C9F5DD20B9F19D
:1022E00061E0C5010E94D21B60E07BE0C5010E9455
:1022F000AF422DC04A8D5B8D052E000C660B770B0F
:10230000C5010E94CD1A2114310409F51E141F04C1
:1023100034F48A8D9B8D892B61F462E007C0EF282D
:1023200041F48A8D9B8D892B21F061E0C5010E94CB
:10233000D21B60E07BE00DC04A8D5B8D052E000C4A
:10234000660B770BC5010E94CD1A112329F060E0BE
:102350007AE0C5010E94AF42811060C1D5011A9692
:102360008C91873009F0A1C359C1E114F10409F03F
:10237000E6C368E977E085E89CE00E94199B642D3C
:10238000C5010E94D21B1E141F0444F4112331F016
:1023900060E071E0C5010E94AF4287C3C5010E94A1
:1023A000051BDC01CB01D82EC92E9A2E0B2FF5016F
:1023B0002285233018F4213018F012C0243009F59A
:1023C0004997A105B1053CF4112329F038E2D32E39
:1023D000C12C912C00E04D2D5C2D692D702F0EC06D
:1023E0000097A105B10539F0F8E1F81720F01123A5
:1023F00011F028E2D22E4D2D592FBD01C5010E94AA
:10240000CD1A4D2D5C2D692D702F4115510561059B
:10241000710509F449C0D5011A968C9190E08A3073
:102420009105F0F5FC018827E757FF4F8F4F0C947B
:10243000D8B5112309F4F2C0C5010E947247892B57
:1024400049F189C30F779A8E0B8F8C2D90E09D8F69
:102450008C8F8D2D90E09F8F8E8F112329F060E05F
:1024600073E0C5010E94AF4293E0892E912C6EC0AB
:102470005B8F4A8F112329F060E073E0C5010E9451
:10248000AF4288248394912C61C05B8F4A8F1123C3
:1024900009F4C4C060E071E0C5010E94AF425BC3B3
:1024A000112309F458C3F6CF2AE030E040E050E0B1
:1024B000BA0185E89CE00E94F79B6AE677E085E830
:1024C0009CE00E94199BF50182858530C9F0A0F43B
:1024D0008150823078F584E690E09B8F8A8F1D8E44
:1024E0001C8E9F8F8E8F007844E650E064E6702F3C
:1024F000C5010E94CD1AB1CF863059F08830D1F491
:1025000084E190E09B8F8A8F44E150E060E070E0CE
:1025100019C084E690E09B8F8A8F44E650E060E02B
:1025200070E0C5010E94CD1A112309F4AACF60E022
:1025300071E0A4CF84E690E09B8F8A8F44E650E060
:1025400060E070E0C5010E94CD1A94CF6E01FAE1FF
:10255000CF0ED11CE12CF12CD601ED91FD916D0136
:10256000FDA3ECA36FE577E085E89CE00E94199B52
:102570004AE050E0B70185E89CE00E943F9C6DE591
:1025800077E085E89CE00E94199B4AE050E06CA14E
:102590007DA185E89CE00E943F9C85E89CE00E942C
:1025A000469CFFEFEF1AFF0A8E149F04A9F6D3C2D0
:1025B000C5010E94FD1B853089F11B8E1A8E1D8E70
:1025C0001C8E1F8E1E8E62E0C5010E94D21B11233D
:1025D00029F160E071E0C5010E94AF421FC01E14E6
:1025E0001F04E4F41B8E1A8E1D8E1C8E1F8E1E8EF1
:1025F000C5010E94FD1B863011F462E001C065E058
:10260000C5010E94D21B60E071E0C5010E94AF428B
:1026100064E577E085E89CE00E94199BCC8CDD8C1A
:10262000C6010D2C000CAA0BBB0B8CA39DA3AEA363
:10263000BFA38E8C9F8C282D30E0AFEFB0E00E94BE
:10264000B5B524E630E040E050E00E9483B5790162
:102650002F3F310521F01CF0EE24EA94F12CD50136
:102660001A968C91843009F41FC150F4813099F18D
:10267000C8F0823009F4B4C0833009F49CC115C29B
:10268000883009F40AC238F4863009F44EC1873024
:1026900009F410C10AC2893009F4F9C18F3709F46D
:1026A000ECC003C2161417040CF0FFC12A8D30E0F1
:1026B000AFEFB0E00E94B5B524E630E040E050E076
:1026C0000E9483B5B9012F3F310519F014F06FEF67
:1026D00070E0C301E6C0B2E3CB16D1040CF062C0D7
:1026E000161417040CF0E0C082E390E08C199D09E9
:1026F000889DD001899DB00D989DB00D11242FEFBC
:1027000030E00E94EFB528E833E140E050E00E945D
:1027100083B5622FC30103960E9441780C8D1D8DF5
:102720002EEF31E0D8010E94EFB522E330E040E027
:1027300050E00E9483B569017A012E8D30E0AFEF41
:10274000B0E00E94B5B524E630E040E050E00E94E1
:1027500083B5D9012F3F310519F014F0AFEFB0E088
:1027600096010E94E7B52FEF30E040E050E00E9474
:1027700083B569017A019801A5E6BFEF0E94E7B52C
:1027800022E330E040E050E00E9483B51FEF120FDB
:102790007601EFEFCE16D10499F194F1EE24EA948C
:1027A000F12C2EC0161417040CF07EC02CA13DA1F4
:1027B0004EA15FA12253310941095109ABE9B0E0B3
:1027C0000E94A2B522E330E040E050E00E9483B5D1
:1027D00014E6120F60E0C30103960E94417810C016
:1027E000161417040CF060C02FEF30E0D6010E94E1
:1027F000EFB524E630E040E050E00E9483B5122FB0
:1028000020E030E040E050E060E070E0CE01019672
:102810000E940994AA8DBB8D2FEF3FEF0E94EFB568
:102820002DE631E040E050E00E9483B5DA01C901B5
:102830004E2D612F0E94FA926B017C01BC0188270A
:102840009927C3010E94417899278F2D7E2D6D2DE8
:10285000C30101960E9441786C2DC30102960E942B
:1028600041788A859B850E9469AB8F81988597FD09
:102870001CC160E00E94416218C116141704A4F440
:1028800060E0C3010E94417860E0C30101960E94AC
:10289000417860E0C30102960E9441786E2DC30129
:1028A00003960E94417801C16A8D7B8DC5010E940B
:1028B000B246FBC0D5011496ED91FC911597808529
:1028C000853009F0F2C0A680B78080914D0A8F5FF5
:1028D00080934D0AA114B10411F1F5018085843073
:1028E000C1F461857285CE0101960E946D4FC8A02A
:1028F000D9A07101012F9E01265E3F4F4AA15BA125
:10290000B201CE0101960E94D80CCE0101960E9420
:10291000FD4FD5011296AD90BC901397DBCF8091FF
:102920004D0A815080934D0AC0C06114710409F4AE
:10293000BCC077FE06C071946194710801E010E09C
:1029400002C000E010E0F62C61E0862D0E9441629A
:10295000012B69F0B1E04B16510429F061E0E6E08B
:102960004E16510409F460E0062F10E011C0F1E0AA
:102970004F16510451F091E080E026E042165104D8
:1029800009F090E0092F182F02C001E010E0602F3D
:102990008F2D0E9412626FE477E085E89CE00E9430
:1029A000199B4AE050E0B30185E89CE00E943F9CFF
:1029B0006DE477E05CC06114710409F468C077FECF
:1029C00006C071946194710801E010E002C000E05B
:1029D00010E0F62C61E0862D0E9441628091A100FA
:1029E000887F8093A10080919100887F80939100DF
:1029F0008091A10082608093A1008091910082600B
:102A000080939100AA8DBB8D012B99F0CD01BB0F56
:102A1000AA0BBB0B9C01AD01245631094109510998
:102A2000AFEFB0E00E94A2B52CE93FEF4FEF5FEFB0
:102A300008C02FEF30E00E94EFB524E630E040E020
:102A400050E00E9483B58901B9018F2D0E947D62FB
:102A500068E477E085E89CE00E94199B4AE050E03A
:102A6000B30185E89CE00E943F9C66E477E085E83E
:102A70009CE00E94199B4AE050E0B80185E89CE088
:102A80000E943F9C85E89CE00E94469C0EC0442D1D
:102A90006A8DC5010E94004608C0442D6A8DC5019B
:102AA0000E94EF4402C080E001C081E090E063C07A
:102AB000EE24E394F12C1FC072E0E72EF12C1BC032
:102AC00065E0E62EF12C17C056E0E52EF12C13C080
:102AD0004AE0E42EF12C0FC03BE0E32EF12C0BC0BA
:102AE0002CE0E22EF12C07C09DE0E92EF12C03C072
:102AF0008EE0E82EF12CC5010E94FD1B082F90E00E
:102B00008E159F0509F49EC865E278E085E89CE093
:102B10000E94199B4AE050E0602F85E89CE00E94EB
:102B2000AE9B89C8C5010E94D21BC80124C067ECB6
:102B300077E085E89CE00E94199B8DEF81C868E8EA
:102B400077E085E89CE00E94199BF501828587303B
:102B500009F415CCF2CFD5011A968C91813009F089
:102B60005DCD8C8D9D8D892B09F058CD8FE7D501DA
:102B70001A968C9353CDAC960FB6F894DEBF0FBE69
:102B8000CDBFDF91CF911F910F91FF90EF90DF901C
:102B9000CF90BF90AF909F908F907F906F905F90FD
:102BA0004F903F902F90089584E690E00895880F0D
:102BB000991F880F991FFC01E752F64F8081918180
:102BC000A281B3810196A11DB11D80839183A2834F
:102BD000B383089585E090E00C94D71584E090E0ED
:102BE0000C94D71583E090E00C94D71582E090E028
:102BF0000C94D71581E090E00C94D71580E090E01C
:102C00000C94D715CF93DF93009709F455C0FC01BE
:102C10002081222309F450C0EC0166E370E10E9498
:102C2000BBAC892BA1F16AE170E1CE010E94BBAC83
:102C3000892B81F166EA78E0CE010E94BBAC892B3A
:102C400061F163EE78E0CE010E94BBAC892B41F1CB
:102C50006FED78E0CE010E94BBAC892B21F162EAD6
:102C600078E0CE010E94BBAC892B01F16EE978E0DF
:102C7000CE010E94BBAC892BE1F06AE978E0CE017D
:102C80000E94BBAC892BC1F488E090E017C082E0C1
:102C900090E014C081E090E011C086E090E00EC0AA
:102CA00083E090E00BC084E090E008C085E090E015
:102CB00005C087E090E002C080E090E0DF91CF9116
:102CC00008950C9469AB0C9469AB8F929F92AF926C
:102CD000BF92CF92DF92EF92FF920F931F93CF9309
:102CE000DF93E0914E0AF0914F0A309709F465C0E6
:102CF000812EF02E932EC22EA52ED42EB72EE62E88
:102D0000BC01CF010E944BA2EC01892B09F458C0F1
:102D10008885853009F054C060E0CE010E948AA207
:102D20008C0161E0CE010E948AA2FC01C185D2859E
:102D3000D80119962D913C911A972130310569F0EF
:102D40002CF4232BE9F56F2DCE0118C0223031056C
:102D500049F027303105A9F033C06F2DCE0103961D
:102D60000E9441786E2DCE010E9441786D2DCE01DA
:102D700001960E9441786C2DCE0102960E94417806
:102D80001FC0892BE9F080858530D1F4C681D781B9
:102D90002097B1F08885843061F40F2D182D2C2DEB
:102DA000392D4D2D5A2D6E2D7B2D89859A850E94AA
:102DB00065160A80DB81C02DEBCF80E090E002C079
:102DC00081E090E0DF91CF911F910F91FF90EF9004
:102DD000DF90CF90BF90AF909F908F900895CF924B
:102DE000DF92EF92FF920F931F93CF93DF93E091C7
:102DF000030AF091040A3097B9F090859530A1F458
:102E000069017A01EB01682FCF010E948AA2FC01BF
:102E10002085243049F481859285009729F0960118
:102E2000A701BE010E946516DF91CF911F910F91FE
:102E3000FF90EF90DF90CF900895AF92BF92CF9226
:102E4000DF92EF92FF920F931F93CF93DF938091C6
:102E5000FC099091FD09892B09F472C0E1E0F0E0D2
:102E6000C0E0D0E0CC24C394D12CB6010C2E02C01B
:102E7000660F771F0A94E2F740917009509171092B
:102E80007F0184E0E80EF11CCF01B12C9C01A091E0
:102E90002E02B0912F02A817B90720F420912E021C
:102EA00030912F02A091B00FB091B10FA20FB31FBC
:102EB000AC90A091FC09B091FD099C012150310911
:102EC000A20FB31F0A2D10E02C9130E00217130758
:102ED00029F0462B572BAC92BB24B3940196E816ED
:102EE000F906A1F65093710940937009BB2011F1C6
:102EF0008091FC099091FD09E80FF91F028110E013
:102F0000218130E0408150E03197608170E0CE0156
:102F10000E94EF160E941299DC01CB01845D9E4F46
:102F2000AF4FBF4F80936C0990936D09A0936E09CA
:102F3000B0936F092196F701C430D10509F095CF00
:102F4000DF91CF911F910F91FF90EF90DF90CF9085
:102F5000BF90AF900895CF92DF92EF92FF920F93C0
:102F60001F93CF93DF93CDB7DEB760970FB6F8947A
:102F7000DEBF0FBECDBF7C016B01CA01B901AE013E
:102F80004F5F5F4F0E94F569D701ED91FC91028878
:102F9000F389E02D9801AE014F5F5F4FB601C70185
:102FA000199560960FB6F894DEBF0FBECDBFDF91C6
:102FB000CF911F910F91FF90EF90DF90CF900895E8
:102FC000CF92DF92EF92FF920F931F93CF93DF93F5
:102FD000CDB7DEB7C054D1090FB6F894DEBF0FBE2F
:102FE000CDBF6115710519F480E090E035C069012D
:102FF0007A018B0140E450E0CE0101960E9439BA7B
:103000006FE270E0CE0101960E9400BA892B41F474
:10301000980143E050E060E4CE0101960E945E69B1
:1030200040E450E0B601CE0101960E941BBA0E9416
:10303000D4918823C9F280914A0A90914B0A04974F
:1030400099F680914C0A8111CFCFB701CE0101963C
:103050000E943AA281E090E0C05CDF4F0FB6F89486
:10306000DEBF0FBECDBFDF91CF911F910F91FF90BB
:10307000EF90DF90CF900895CF92DF92EF92FF9282
:103080000F931F93CF93DF93CDB7DEB760970FB643
:10309000F894DEBF0FBECDBF7C016B01BA01A90160
:1030A000CE0101960E940369D701ED91FC9102883F
:1030B000F389E02D9801AE014F5F5F4FB601C70164
:1030C000199560960FB6F894DEBF0FBECDBFDF91A5
:1030D000CF911F910F91FF90EF90DF90CF900895C7
:1030E0000F931F93CF93DF938C01FC01C081D1819B
:1030F0006FE270E0CE010E9448BA0097C1F0FC0177
:103100001192CF010E940216EC0163ED78E085E890
:103110009CE00E94199B4AE050E0BE0185E89CE0DB
:103120000E943F9C85E89CE00E94469C09C0CE011D
:103130000E940216EC01892B19F0F801118210820D
:10314000CE01DF91CF911F910F9108952F923F9261
:103150004F925F926F927F928F929F92AF92BF92A7
:10316000CF92DF92EF92FF920F931F93CF93DF9353
:10317000CDB7DEB72B970FB6F894DEBF0FBECDBF2D
:103180004C016B01042F38872F83672B09F4DDC1B5
:10319000F901309719F08081811109C0D4011D9681
:1031A0008C91882321F0C4010D9698878F83EF813D
:1031B000F885309721F4F401E788F08C0AC080810B
:1031C0008823C9F3CE0107960E9470187C01892BD1
:1031D00091F35601D5018C91882349F0082E000CFB
:1031E000990B0E9498B9F50181935F01F3CFD60145
:1031F0001C911D3209F4CBC080ED810F8A3008F498
:10320000C6C0153209F4F6C06EE570E1C6010E9431
:10321000BBAC892B09F4E6C06AE570E1C6010E94E7
:10322000BBAC892B09F4E2C061E379E0C6010E94DE
:10323000BBAC892B09F4AEC06AE279E0C6010E94FA
:10324000BBAC892B09F4AAC061E477E0C6010E94F7
:10325000BBAC892B09F4A6C06DE377E0C6010E94E0
:10326000BBAC892B09F4A2C065E279E0C6010E94DB
:10327000BBAC892B09F49EC063E270E1C6010E94D9
:10328000BBAC892B09F49AC06EE170E1C6010E94C3
:10329000BBAC892B09F496C068E270E1C6010E94BC
:1032A000BBAC892B09F492C064E377E0C6010E94AD
:1032B000BBAC892B09F48EC060E377E0C6010E94A5
:1032C000BBAC892B09F48AC060E279E0C6010E9498
:1032D000BBAC892B09F486C06AE179E0C6010E9483
:1032E000BBAC892B09F482C062E179E0C6010E947F
:1032F000BBAC892B09F476C069E079E0C6010E9475
:10330000BBAC892B09F472C060E079E0C6010E9471
:10331000BBAC892B09F46EC067EF78E0C6010E9450
:10332000BBAC892B09F46AC062EF78E0C6010E9449
:10333000BBAC892B09F466C06BEE78E0C6010E9435
:10334000BBAC892B09F462C067EE78E0C6010E942D
:10335000BBAC892B09F45EC01B3709F45FC0133284
:1033600009F461C043E050E063EE78E0C6010E94DA
:10337000DBAC892B09F45CC043E050E06FED78E0F2
:10338000C6010E94DBAC892B09F057C04CC0A12CB0
:10339000B12C56C0E3E0AE2EB12C52C074E0A72E83
:1033A000B12C4EC065E0A62EB12C4AC056E0A52E29
:1033B000B12C46C047E0A42EB12C42C03AE0A32E67
:1033C000B12C3EC02BE0A22EB12C3AC09CE0A92E1D
:1033D000B12C36C08DE0A82EB12C32C01EE0A12E3B
:1033E000B12C2EC0AA24A394B12C2AC0A2E0AA2EEC
:1033F000B12C26C0F8E0AF2EB12C22C0E9E0AE2EF1
:10340000B12C1EC070E1A72EB12C1AC061E1A62E0E
:10341000B12C16C052E1A52EB12C12C04EEFA42E35
:10342000BB24BA940DC03DEFA32EBB24BA9408C0B0
:103430002CEFA22EBB24BA9403C0AA24AA94BA2CBF
:1034400066E379E085E89CE00E94199B4AE050E041
:10345000B50185E89CE00E943F9C85E89CE00E94C5
:10346000469CBFEFAB16BB0609F064F4EEEFAE1658
:10347000EFEFBE060CF069C0FCEFAF16FFEFBF0622
:1034800049F053C0A114B10429F0C501089702976F
:1034900018F04BC0A12CB12CCE0101961C01612C5F
:1034A000712C8A873B862301AFEF4A1A5A0A3201F0
:1034B000F60180818823D1F06F018191882329F062
:1034C0008D3219F080538A30B8F7C6010E9494AC4F
:1034D000182F99876CE270E0C6010E9400BA6C0157
:1034E000892B39F0FFEFCF1ADF0A03C080E090E0AC
:1034F00002C0812F9985D1018D939D931D01C11427
:10350000D10439F093E04916510469F683E0682E3E
:10351000712CCF80D884D401ED91FC910190F08181
:10352000E02D2A853B85A3010CC0CF80D884D4012F
:10353000ED91FC910190F081E02D20E030E040E041
:1035400050E0B501C401199502C080E090E02B96CF
:103550000FB6F894DEBF0FBECDBFDF91CF911F91A4
:103560000F91FF90EF90DF90CF90BF90AF909F9022
:103570008F907F906F905F904F903F902F90089525
:10358000DC011296ED91FC911397309721F081E0C8
:103590009085953009F080E00895CF92DF92EF9208
:1035A000FF92CF93DF93DC011696ED91FC91179774
:1035B000309721F12085223009F56A017B01EC0169
:1035C0006BEC78E085E89CE00E94199B65EC78E064
:1035D00085E89CE00E94199B2AE030E0B701A60133
:1035E00085E89CE00E94F79B85E89CE00E94469C51
:1035F000EE81FF81C186D286E386F486DF91CF918A
:10360000FF90EF90DF90CF900895FC018681978125
:10361000009789F0FC012085223041F0253059F4D3
:1036200060E00E948AA2009731F0FC0161857285FA
:1036300083859485089560E070E0CB0108950F9331
:103640001F93CF93DF93FC01C481D581209791F024
:103650008885823029F4672B69F489859A8514C09E
:10366000853041F48B01CE010E9469A590E00817D6
:1036700019071CF080E090E007C0602FCE010E9487
:103680008AA2FC0181859285DF91CF911F910F91D4
:1036900008950F931F93CF93DF93EB0163E0FC0139
:1036A000828193810E948AA2009741F1AE014095E8
:1036B00050954F6F60E070E0FC0101851285238515
:1036C00034854023512362237323418752876387C4
:1036D00074876CEB78E085E89CE00E94199B4AE0D7
:1036E00050E0BE0185E89CE00E943F9C85E89CE09C
:1036F000DF91CF911F910F910C94469CDF91CF9158
:103700001F910F9108950F931F93CF93DF93EB01B8
:1037100063E0FC01828193810E948AA2009731F1CB
:10372000AE01442760E070E0FC010185128523852D
:103730003485402B512B622B732B41875287638733
:10374000748763EB78E085E89CE00E94199B4AE06F
:1037500050E0BE0185E89CE00E943F9C85E89CE02B
:10376000DF91CF911F910F910C94469CDF91CF91E7
:103770001F910F910895CF93DF93EB0163E0FC015C
:10378000828193810E948AA2009739F0FC01818591
:10379000928588278C239D2302C080E090E0DF91F2
:1037A000CF910895CF93C62F63E0FC01828193816E
:1037B0000E948AA20097F9F0FC0141855285638539
:1037C00074854427662777274C2B41875287638768
:1037D00074876BEA78E085E89CE00E94199B4AE0D8
:1037E00050E06C2F85E89CE00E94AE9B85E89CE051
:1037F000CF910C94469CCF91089563E0FC018281A7
:1038000093810E948AA2009719F0FC018185089596
:103810008FEF0895CF93DF93EC01FB012481358175
:1038200040815181628173810E94F79BCE01DF91BB
:10383000CF910895089508956F927F928F929F92ED
:10384000AF92BF92CF92DF92EF92FF920F931F93AE
:10385000CF93DF93CDB7DEB7C054D1090FB6F8943C
:10386000DEBF0FBECDBF3C014B01FC01E080F1800B
:1038700065ED74E0C7010E944BA25C016AED74E043
:10388000C7010E944BA26C01A114B10419F4892B49
:1038900009F4D3C06FED74E0C7010E944BA28C0104
:1038A00064EE74E0C7010E944BA27C01F3017380B7
:1038B0006FE878E085E89CE00E94199B4AE050E0C0
:1038C000672D85E89CE00E94AE9B6DE878E085E876
:1038D0009CE00E94199B4AE050E0B40185E89CE01E
:1038E0000E943F9C85E89CE00E94469CC114D10444
:1038F000D1F1F60180858430B1F56185728540E4AF
:1039000050E0CE0101960E9439BA0E94D4918823DA
:1039100051F180914C0A811126C06FE270E0CE0116
:1039200001960E9400BA892B51F4F6012185328557
:1039300043E050E060E4CE0101960E945E6981148C
:10394000910409F469C00115110509F462C0F80178
:103950008085843009F05DC0F80161857285FB01C6
:103960008081811165C0A114B10409F466C0F5011C
:103970008085843009F061C061857285CE01019631
:103980000E946D4FCE0101960E94C01A8823E1F17A
:103990008928A9F00115110521F0F80180858430EE
:1039A00061F0C12CD12CE12CF12C01E020E030E0C1
:1039B00040E050E061E070E014C0F80118C0E1148C
:1039C000F10421F0F7018085843081F0C12CD12CE5
:1039D000E12CF12C01E020E030E040E050E062E03A
:1039E00070E0CE0101960E94D80C0EC0F7016185EF
:1039F0007285FB018081882339F020E030E041E0CE
:103A0000CE0101960E94A618CE0101960E94FD4F9C
:103A100014C069EE74E00CC0E114F10421F0F70168
:103A20008085843019F46CEE74E002C0F70195CF04
:103A3000CE0101960E943AA296CFC05CDF4F0FB62E
:103A4000F894DEBF0FBECDBFDF91CF911F910F91D4
:103A5000FF90EF90DF90CF90BF90AF909F908F90AE
:103A60007F906F900895CF92DF92FF920F931F93F4
:103A7000CF93DF93EC01F62E8A0188819981892BFF
:103A800009F412C1EC81FD81309709F40DC18081E8
:103A90009FEF691318C084FF05C14330510509F435
:103AA00001C1F180F2948FE0F82265E778E085E8C3
:103AB0009CE00E94199B4AE050E06F2D85E89CE055
:103AC0000E94AE9B02C084FDEFC0EC81FD8181812C
:103AD0008F70D82EF81661F1CB8063E778E085E827
:103AE0009CE00E94199B4AE050E06C2D85E89CE028
:103AF0000E94AE9B61E778E085E89CE00E94199BFC
:103B00004AE050E06D2D85E89CE00E94AE9B6EE699
:103B100078E085E89CE00E94199B4AE050E06F2D18
:103B200085E89CE00E94AE9B85E89CE00E94469C54
:103B30008F2D90E08D30910508F089C0FC01CC807C
:103B4000DD808827ED56FF4F8F4F0C94D8B5F601D6
:103B50009181292F2F70253009F479C088819981AE
:103B6000263028F4223069F461EF74E04CC027302D
:103B700029F02A3031F467EF74E060C060EF74E040
:103B80004FC064EE74E034C06FED74E088819981B9
:103B90000E944BA2F6012081422F4170322F3095B6
:103BA00030FB20F91FC06EEF74E0888199810E947C
:103BB0004BA2F601208121FB442740F931E0342754
:103BC00030FB21F90FC064E075E0888199810E9483
:103BD0004BA2F601208122FB442740F931E0342733
:103BE00030FB22F9208331C064EE74E08881998132
:103BF0000E944BA240E029C06AE075E002C06FE07D
:103C000075E0888199810E944BA2F6014081417044
:103C10001CC065E175E002C06BE175E088819981A7
:103C20000E944BA2F6014081469541700EC062E2AF
:103C300075E002C068E275E0888199810E944BA21C
:103C4000F601408142FB442740F9009751F4EC8192
:103C5000FD818F2D8F709181907FF92EF82AF1824E
:103C600021C0EC81FD810330110581F02F2D2F70D3
:103C70003181307FF32EF22AF182BC01CE010E9405
:103C80001150EC81FD8180818F7E0BC081818F700E
:103C9000982F9295907F892B8183EC81FD81808183
:103CA0008061808381E001C080E0DF91CF911F912E
:103CB0000F91FF90DF90CF900895FC01238130E0B9
:103CC00080E090E0FC01EE0FFF1FEB5EFE4EA08156
:103CD000B181A217B30731F0A081B181AB2B71F490
:103CE00020813181880F991F880F991FFC01EF5F98
:103CF000FE4E40835183628373830895019685301D
:103D0000910501F70895FF920F931F93CF93DF93CF
:103D1000EC011D821C821A821B8208811981011507
:103D2000110509F456C0F8018085863009F051C0AC
:103D300080913C0B90913D0B892B09F44AC069E1BD
:103D400078E0C8010E944BA2009719F0FC01818520
:103D50008A83F801808191810E9494ACF82E8B8334
:103D60006AE179E0C8010E944BA2009779F51A81B7
:103D700069E678E085E89CE00E94199B4AE050E003
:103D80006F2D85E89CE00E94AE9B67E678E085E8B1
:103D90009CE00E94199B4AE050E0612F85E89CE07E
:103DA0000E94AE9B85E89CE00E94469C40E050E06B
:103DB0006AE179E0888199810E94F5A36AE179E05E
:103DC000888199810E944BA2009719F009969D83E2
:103DD0008C83DF91CF911F910F91FF900895EF9207
:103DE000FF920F931F93CF93DF938091700990916F
:103DF0007109C4E0D0E021E030E0AC01422353235C
:103E0000452B29F0A9014095509584239523220F35
:103E1000331F219791F790937109809370090E9445
:103E2000129900916C0910916D0920916E093091E1
:103E30006F09601771078207930708F459C0012BB7
:103E4000022B032B09F454C010926C0910926D09D7
:103E500010926E0910926F09E12CF12CE091FC098F
:103E6000F091FD09EC0FFD1F038110E0228130E08D
:103E7000418150E0608170E0C7010E94EF168FEF32
:103E8000E81AF80A249684E0E816F10439F7C1E04C
:103E9000D0E080912E0290912F028C179D0728F47C
:103EA00080912E0290912F0201C0CE012091B00F7F
:103EB0003091B10FF901E80FF91F4AE050E060813D
:103EC00085E89CE00E94AE9B6FE275E085E89CE08F
:103ED0000E944A9C2196C131D105D9F685E89CE023
:103EE000DF91CF911F910F91FF90EF900C94469C22
:103EF000DF91CF911F910F91FF90EF900895EF9276
:103F0000FF920F931F93CF93DF93DC011296ED91F5
:103F1000FC911397309701F18A017B01EC016AED66
:103F200074E0808191810E944BA20097A9F0FC016E
:103F30002085243089F461857285E881F9810288C1
:103F4000F389E02D9801A701CE01DF91CF911F9158
:103F50000F91FF90EF90199480E090E0DF91CF9166
:103F60001F910F91FF90EF900895EF92FF920F93A2
:103F70001F93CF93DF93CDB7DEB760970FB6F8945A
:103F8000DEBF0FBECDBF8C01CB01BA017901AE01FE
:103F90004F5F5F4F0E94F569A701BE016F5F7F4FC2
:103FA000C8010E947F1F60960FB6F894DEBF0FBE57
:103FB000CDBFDF91CF911F910F91FF90EF900895AA
:103FC0004F925F926F927F928F929F92AF92BF9229
:103FD000CF92DF92EF92FF920F931F93CF93DF93D5
:103FE000CDB7DEB7C25AD1400FB6F894DEBF0FBED0
:103FF000CDBF20914A0A30914B0AF9013B96E83136
:10400000F10508F0C0C38827E056FF4F8F4F0C948E
:10401000D8B50E9412990091380B1091390B20915C
:104020003A0B30913B0B061717072807390708F0A2
:10403000AAC30CE814E0CE56DE4F19830883C25998
:10404000D140CC56DE4F188219821A821B82C45985
:10405000D140CE57DE4F19830883C258D140CC5788
:10406000DE4F188219821A821B82C458D140CE5961
:10407000DE4F19830883C256D140CC59DE4F1882D7
:1040800019821A821B82C456D140CE5BDE4F19833F
:104090000883C254D140CC5BDE4F188219821A8249
:1040A0001B82C454D14060EC79E085E89CE00E941A
:1040B000199B85E89CE00E94469CBE016E567E4F8F
:1040C00086E090E00E940671892B09F467C161E3E4
:1040D00075E085E89CE00E944A9C1A830983CC56CF
:1040E000DE4F88819981AA81BB81C459D1408B83DD
:1040F0009C83AD83BE83CE0101960E94A05DBE016C
:104100006E577E4F8AE090E00E940671892B09F479
:104110002EC167E475E085E89CE00E944A9C1A8302
:104120000983CC57DE4F88819981AA81BB81C4580D
:10413000D1408B839C83AD83BE83CE0101960E94C8
:10414000A05DBE016E597E4F8EE090E00E94067128
:10415000892B09F4DFC06DE475E085E89CE00E94DE
:104160004A9C1A830983CC59DE4F88819981AA81A0
:10417000BB81C456D1408B839C83AD83BE83CE016B
:1041800001960E94A05DBE016E5B7E4F82E190E0D1
:104190000E940671892B09F477C062E575E085E815
:1041A0009CE00E944A9C1A830983CC5BDE4F888185
:1041B0009981AA81BB81C454D1408B839C83AD83F8
:1041C000BE83CE0101960E94A05D1A830983CC5B59
:1041D000DE4F88819981AA81BB81C454D1408B83F1
:1041E0009C83AD83BE83CF57DF4F19830883C158AB
:1041F000D040CC59DE4F88819981AA81BB81C456B9
:10420000D140CD57DF4F88839983AA83BB83C3589E
:10421000D040CE53DF4F19830883C25CD040CC57C7
:10422000DE4F88819981AA81BB81C458D140CC538B
:10423000DF4F88839983AA83BB83C45CD040CE5F61
:10424000DE4F19830883C250D140CC56DE4F88819F
:104250009981AA81BB81C459D140CC5FDE4F88834C
:104260009983AA83BB83C450D1409E012F5F3F4FE7
:10427000AE014F575F4FBE016E537F4FCE018E5F31
:104280009E4F0E94E66F85C01A830983CC59DE4F8A
:1042900088819981AA81BB81C456D1408B839C833C
:1042A000AD83BE83CF57DF4F19830883C158D040F9
:1042B000CC57DE4F88819981AA81BB81C458D140F7
:1042C000CD57DF4F88839983AA83BB83C358D040DF
:1042D000CE53DF4F19830883C25CD040CC56DE4FEB
:1042E00088819981AA81BB81C459D140CC53DF4FC9
:1042F00088839983AA83BB83C45CD040AE014F5F9F
:104300005F4FBE016F577F4FCE018E539F4F0E946C
:1043100032703FC01A830983CC57DE4F8881998160
:10432000AA81BB81C458D1408B839C83AD83BE835B
:10433000CF57DF4F19830883C158D040CC56DE4F8A
:1043400088819981AA81BB81C459D140CD57DF4F63
:1043500088839983AA83BB83C358D040BE016F5F13
:104360007F4FCE018F579F4F0E94847012C01A83D7
:104370000983CC56DE4F88819981AA81BB81C459BB
:10438000D1408B839C83AD83BE83CE0101960E9476
:10439000CF7085E89CE00E94469C0BC169E575E002
:1043A00085E89CE00E944A9C0FB6F894A8958091FD
:1043B0006000886180936000109260000FBE809161
:1043C000D009811107C085EB99E00E94127C81E041
:1043D0008093D00982E799E090932F0D80932E0D62
:1043E0000E94566FCE0101960E94185B89819A81C6
:1043F0000E94037646E050E06FE17BE089E090E0C8
:104400000E9433A18CE894E09A8389831B821C82EA
:104410001D821E82CE0103960E94ED750E940276D7
:1044200080912E0D90912F0DDC0192961D921D9280
:104430001D921C929597FC0116A217A210A611A618
:104440009A961D921D921D921C929D9740EE5EE2DF
:1044500060E070E046AB57AB60AF71AF40EA5FE041
:1044600060E070E0DA964D935D936D937C93DD97F9
:104470003E9624E1DF011D922A95E9F726E0EFE15F
:10448000FBE0DC01189601900D922A95E1F7FC0102
:10449000EE5BFF4F10820E94C8738C01019709F0F8
:1044A0004AC0CE0101960E94185B89819A810E94C0
:1044B000037660912E0D70912F0D625F7F4FCE01BC
:1044C00001960E944C9CCE0103960E94ED7560916E
:1044D0002E0D70912F0D6A5E7F4FCE0101960E94C6
:1044E0004C9CCE0103960E94FB7560912E0D70913D
:1044F0002F0D6E5E7F4FCE0101960E944C9CCE0127
:1045000003960E94F4750E94027660912E0D7091C0
:104510002F0D625E7F4FCE0101960E944C9C8B81D5
:104520009C81AD81BE8180932A0D90932B0DA09329
:104530002C0DB0932D0D99E288E10FB6F894A89553
:10454000809360000FBE90936000A895012B19F531
:104550006EE779E085E89CE00E94199B6FE479E0C2
:1045600085E89CE00E94199B86EF9FEF90934B0A91
:1045700080934A0A0E941299DC01CB01805A95412E
:10458000AF4FBF4F8093380B9093390BA0933A0BEA
:10459000B0933B0BF8C06FE379E085E89CE00E94A4
:1045A000199BCE0101960E94F65DCE0101960E94F4
:1045B000A05D81E090E0E3C080914D0A8111D0C6FA
:1045C0008091D80981111AC060E070E080E090E02D
:1045D0000E94D283D4C00E9412990091380B10918E
:1045E000390B20913A0B30913B0B06171707280720
:1045F0003907D0F10E94D4918111C5C082E090E0CA
:10460000BEC0A895CE55DE4F1882C25AD140FE01D9
:10461000EE56FE4F119211928EE0DF011D928A95A7
:10462000E9F70091FF091091000A0115110529F021
:10463000C8010E9469A5811121C20E94D4918111F3
:10464000A2C00091FF091091000A0115110509F49B
:104650009AC0C8010E9469A5E82EF12CB2E0EB16C1
:10466000F1040CF025C28FC020E030E043E050E0C0
:1046700061E48E010F5F1F4FC8010E945E6965E70C
:1046800075E0C8010E94F5B9F80101900020E9F732
:10469000CF01801B910B08968138910538F50E9457
:1046A000D491882319F18091DA0D9091DB0D019658
:1046B00011F481E090E09093DB0D8093DA0D80910E
:1046C000DA0D9091DB0D90935F0D8093600D47E0C4
:1046D00050E06AE57DE0C8010E944B91AC01455075
:1046E00051096AE57DE082EA0E946B9184E090E0E6
:1046F00090934B0A80934A0A66E97BE085E89CE048
:104700000E94199B40C00E9412990091380B109191
:10471000390B20913A0B30913B0B061717072807EE
:10472000390788F510924B0A10924A0A2CC00E9451
:1047300012990091380B1091390B20913A0B30915E
:104740003B0B061717072807390708F457CF1BC07C
:104750000E946F83892B09F051CF0E941299DC01CE
:10476000CB0188579C4EAF4FBF4F8093380B90932F
:10477000390BA0933A0BB0933B0B86EF9FEF9093CE
:104780004B0A80934A0A0FB6F894A895809160006E
:10479000886180936000109260000FBE80914A0A89
:1047A00090914B0A181619060CF059C100912E0D64
:1047B00010912F0D0115110509F451C10E94129994
:1047C0004B015C017801FEE3EF0EF11CF7018081E3
:1047D0009181A281B381A5019401281B390B4A0B59
:1047E0005B0BCA01B901683E33E07307810591058F
:1047F00008F446C028EE33E040E050E00E9461B586
:10480000861A970AA80AB90AD7018D929D92AD928D
:10481000BC921397F80186A597A5A0A9B1A9690133
:104820007A01CC0CDD1CEE1CFF1C8C159D05AE0521
:10483000BF0528F416A617A610AA11AA09C0821B44
:10484000930BA40BB50BF80186A797A7A0ABB1AB50
:10485000F80182A993A9A4A9B5A98C159D05AE0557
:10486000BF0528F412AA13AA14AA15AA09C0821B0C
:10487000930BA40BB50BF80182AB93ABA4ABB5AB18
:10488000F80186A597A5A0A9B1A9892B8A2B8B2B06
:1048900069F4EE5BFF4F8081833041F484E08083D4
:1048A000C8010E94C87301967C0102C0E12CF12C62
:1048B000F80182A993A9A4A9B5A9892B8A2B8B2BCE
:1048C000A1F4EE5BFF4F8081833011F081110DC0A8
:1048D0001082F8013E9684E1DF011D928A95E9F786
:1048E000C8010E94C87303967C01B2E0EB16F10484
:1048F00029F0E4E0EE16F10409F04AC0CE01019679
:104900000E94185B89819A810E94037660912E0D26
:1049100070912F0D625F7F4FCE0101960E944C9CDB
:10492000CE0103960E94ED7560912E0D70912F0DB2
:104930006A5E7F4FCE0101960E944C9CCE01039689
:104940000E94FB7560912E0D70912F0D6E5E7F4F52
:10495000CE0101960E944C9CCE0103960E94F475F4
:104960000E94027660912E0D70912F0D625E7F4F36
:10497000CE0101960E944C9C8B819C81AD81BE81B1
:1049800080932A0D90932B0DA0932C0DB0932D0D99
:10499000F3E0EF16F10409F451C064F431E0E316DA
:1049A000F10451F142E0E416F10409F058C06DE55C
:1049B0007BE049C054E0E516F10409F442C085E00B
:1049C000E816F10409F04BC06EE87BE085E89CE056
:1049D0000E94199B85E89CE00E94469C0E94D4910D
:1049E00081110E94235E0E941299DC01CB01805D3F
:1049F0009A48AF4FBF4F13C06AE77BE085E89CE061
:104A00000E94199B0E94D49181110E94235E0E94F2
:104A10001299DC01CB0188519C4FAF4FBF4F80935F
:104A2000380B9093390BA0933A0BB0933B0B86EF66
:104A30009FEF90934B0A80934A0A11C06AE47BE08F
:104A4000DDCF6EE27BE085E89CE00E94199BCE0101
:104A500001960E94F65DCE0101960E94A05D99E24A
:104A600088E10FB6F894A895809360000FBE9093EC
:104A7000600020914A0A30914B0A72C460E070E0F5
:104A8000C8010E945FA78C0190936D0A80936C0A05
:104A900061E27BE085E89CE00E94199BB80185E813
:104AA0009CE00E944A9C85E89CE00E94469CC5CD03
:104AB00061E070E0C8010E945FA73C0192E0E91646
:104AC000F10491F062E0C8010E948AA2FC01818495
:104AD0009284F3E0EF16F10459F063E070E0C8014E
:104AE0000E945FA78C0107C08BE5882E87E0982E77
:104AF0008E010E551E4F40E150E0BE016E567E4FB6
:104B000086E390E00E942B83892B51F425E0E21686
:104B1000F1040CF038C3AE014E565E4F7A0104C06A
:104B2000CE018E569E4F7C017092EE0D6092ED0D7F
:104B30009092F00D8092EF0D8AE090E49093E60D54
:104B40008093E50D5E019EE7A91A9EEFB90A40E148
:104B500050E064EF7AE0C5010E94E9AC6E01AEE975
:104B6000CA1AAEEFDA0A20E030E041E050E060E23D
:104B7000C6010E945E6940E250E06DEE7AE0C60137
:104B80000E94CBAC6DEC7AE085E89CE00E94199B1A
:104B9000B30185E89CE00E944A9C6BEC7AE085E8D2
:104BA0009CE00E94199B4AE050E0B40185E89CE03B
:104BB0000E943F9C64EC7AE085E89CE00E94199B8F
:104BC000B80185E89CE00E944A9C6FEB7AE085E89A
:104BD0009CE00E94199BF8018081811104C0E12CA6
:104BE000F12C00E010E080906C0A90906D0A0E9419
:104BF000D49181114DC18091580D9091590DDC01D6
:104C0000ED91FC910688F789E02D19958823B1F084
:104C100081E090E09093DB0D8093DA0D87E0EAE489
:104C2000F2E0DE01119601900D928A95E1F7FE0106
:104C30003196AFE5BDE0CE01089637C06091ED0D2D
:104C40007091EE0D8091580D9091590D4091EF0D9E
:104C50005091F00DDC01ED91FC916115710521F091
:104C60000088F189E02D16C00684F785E02D2CE838
:104C700034E03A8329834090E90D5090EA0D60902A
:104C8000EB0D7090EC0D4B825C826D827E82BE01DA
:104C90006F5F7F4F1995019709F4BACF8EEF9FEFA1
:104CA0009093F40D8093F30D7EC221912D938E1776
:104CB0009F07D9F70115110529F0E114F10421F03E
:104CC00086EF03C086E301C086EB8093660D1092E9
:104CD000670D8FE08093680DF40101900020E9F7E3
:104CE000CF018819990940968138910508F0C4C010
:104CF0004FE050E06AE57DE0C4010E944B91F6016F
:104D000001900020E9F73197EC19FD09E80FF91F30
:104D10003296E138F10508F0AFC0AC016AE57DE0FC
:104D2000C6010E944B91F50101900020E9F73197EF
:104D3000EA19FB09E80FF91F3296E138F10508F08E
:104D40009BC0AC016AE57DE0C5010E944B91011555
:104D5000110579F1F80101900020E9F73197E01B86
:104D6000F10B9C012E5F3F4FE20FF31FE138F1057D
:104D700008F082C0AC016AE57DE0C8010E944B9159
:104D8000E114F104B1F0F70101900020E9F7319747
:104D9000EE19FF099C012E5F3F4FE20FF31FE13830
:104DA000F10508F069C0AC016AE57DE0C7010E9429
:104DB0004B91AC01455051096AE57DE080E10E94CC
:104DC0006B910E9412996093DC0D7093DD0D8093BE
:104DD000DE0D9093DF0D6093E00D7093E10D8093F5
:104DE000E20D9093E30D8091580D9091590DDC01E7
:104DF000ED91FC910084F185E02D1995892BC1F48A
:104E00000E9412990091E00D1091E10D2091E20DA8
:104E10003091E30DDC01CB01801B910BA20BB30B96
:104E200088399A43A105B105F0F28CEF9FEF20C0BD
:104E3000CE018F579F4F0E94255B6430710581051D
:104E40009105D1F480915D0D811111C00E941299DC
:104E50006093E00D7093E10D8093E20D9093E30D6C
:104E60001092E40D1092F40D1092F30D11C090E029
:104E70009093F40D8093F30D8091580D9091590DFE
:104E8000DC01ED91FC910488F589E02D19958BC129
:104E900000916C0A10916D0A61EB7AE085E89CE064
:104EA0000E94199BB80185E89CE00E944A9C85E815
:104EB0009CE00E94469C81E08093D80920E030E08D
:104EC00043E050E061E4CE018F579F4F0E945E693E
:104ED00065E775E0CE018F579F4F0E94F5B9CE016F
:104EE0008F579F4F0E94166F20E030E042E050E065
:104EF00061E4CE018F579F4F0E945E6969E775E0BC
:104F0000CE018F579F4F0E94F5B9BE016F577F4F5B
:104F100085E89CE00E947EA3CE018F579F4F0E94A0
:104F2000166F20E030E041E050E061E4CE018F57A1
:104F30009F4F0E945E6969E775E0CE018F579F4FD2
:104F40000E94F5B9BE016F577F4F85E89CE00E9433
:104F50007EA3CE018F579F4F0E94166FFE01EE5F1A
:104F6000FE4F119211921EE3DF01212F1D922A950F
:104F7000E9F71A821982FE0133968EE7DF011D924E
:104F80008A95E9F720E030E041E050E060E4CE01AE
:104F90008E5F9E4F0E945E6940E450E06DEE7AE0C5
:104FA000CE018E5F9E4F0E94CBAC40E850E06AE697
:104FB0007AE0CE0101960E94E9ACBE016F5F7F4F9F
:104FC000CE018E5F9E4F0E943AA220E030E041E089
:104FD00050E060E4CE018E5F9E4F0E945E6940E427
:104FE00050E064E67AE0CE018E5F9E4F0E94CBAC2B
:104FF00040E850E06AE57AE0CE0101960E94E9AC13
:1050000040E850E067E47AE0CE0101960E94CBAC24
:10501000BE016F5F7F4FCE018E5F9E4F0E943AA20E
:1050200020E030E041E050E060E4CE018E5F9E4F32
:105030000E945E6940E450E06AE777E1CE018E5F4E
:105040009E4F0E94CBAC40E850E067E37AE0CE018F
:1050500001960E94E9ACBE016F5F7F4FCE018E5F6B
:105060009E4F0E943AA220E030E041E050E060E430
:10507000CE018E5F9E4F0E945E6940E450E060E387
:105080007AE0CE018E5F9E4F0E94CBAC40E850E0AC
:105090006AE27AE0CE0101960E94E9ACBE016F5F40
:1050A0007F4FCE018E5F9E4F0E943AA280914D0AA3
:1050B0008F5F80934D0AA0914E0AB0914F0A1097CE
:1050C00009F443C08091510290915202AE014E5BAF
:1050D0005E4FFA01819391932EE111922A95E9F79F
:1050E0009E012E533F4FF9018193919311921A958E
:1050F000E9F716960D911C911797E0904E0AF090E3
:105100004F0AE114F10471F00115110559F0D801AD
:1051100018968C918530A9F7C8010E9469A588234B
:1051200081F36FC020E030E041E050E060E4CE0168
:105130008E5F9E4F0E945E6940E450E06DEC79E026
:10514000CE018E5F9E4F0E94CBAC80914D0A815064
:1051500080934D0A83E090E090934B0A80934A0A33
:105160000E941299DC01CB0188579C4EAF4FBF4F74
:105170008093380B9093390BA0933A0BB0933B0B71
:1051800064E97AE0BBCA64E070E08091FF09909125
:10519000000A0E945FA77C0161E07BE085E89CE05B
:1051A0000E94199BC1CC0091F30D1091F40D68E899
:1051B0007AE085E89CE00E94199B4AE050E0B80143
:1051C00085E89CE00E943F9C60E77AE085E89CE0EF
:1051D0000E94199B85E89CE00E94469C0E941299BF
:1051E000DC01CB0188579C4EAF4FBF4F8093380BEB
:1051F0009093390BA0933A0BB0933B0B8CE090E06B
:10520000BECA60E0C8010E948AA2FC018185928525
:10521000A385B4858A30910508F463C020E030E0AE
:1052200041E050E060E4CE018E5F9E4F0E945E69D7
:10523000F8016081718140E450E0CE018E5F9E4FA5
:105240000E941BBA6BE775E0CE018E5F9E4F0E94F5
:10525000F5B940E450E06CED79E0CE018E5F9E4FF1
:105260000E94CBACBE016E5B7E4FCE018E5F9E4F27
:105270000E943AA2CE53DF4F8881C25CD04088237F
:1052800061F120E030E041E050E060E4CE018E5F6B
:105290009E4F0E945E69D8016D917C9140E450E080
:1052A000CE018E5F9E4F0E941BBA6BE775E0CE0168
:1052B0008E5F9E4F0E94F5B940E450E064ED79E0C6
:1052C000CE018E5F9E4F0E94CBACBE016E537F4FCE
:1052D000CE018E5F9E4F0E943AA2F8010281138197
:1052E0000CCFFC0140E250E08827E854FF4F8F4F7D
:1052F0000C94D8B564E27AE0CE018E5B9E4F0E949A
:10530000E9ACCE53DF4F1882C25CD04087CF6FE14B
:105310007AE0CE018E5B9E4F0E94E9AC40E450E003
:105320006EEF79E017C068EF79E0CE018E5B9E4F9B
:105330000E94E9AC40E450E064EF79E00BC06CEE11
:1053400079E0CE018E5B9E4F0E94E9AC40E450E0D4
:1053500066EE79E0CE018E539F4F0E94E9AC5ECF9E
:10536000C901CE55DE4F0FB6F894DEBF0FBECDBFDC
:10537000DF91CF911F910F91FF90EF90DF90CF9031
:10538000BF90AF909F908F907F906F905F904F9065
:1053900008952F923F924F925F926F927F928F92D9
:1053A0009F92AF92BF92CF92DF92EF92FF920F93B4
:1053B0001F93CF93DF93CDB7DEB7C257D1090FB696
:1053C000F894DEBF0FBECDBF0091F1091091F20934
:1053D0000115110511F40C94D33280914D0A8F5FA1
:1053E00080934D0A0E941299C090F709D090F80955
:1053F000E090F909F090FA09C616D706E806F90612
:1054000008F052C0D80116962D903C9017972114A1
:105410003104D9F1F1018085863089F566963FAE79
:105420002EAE6697CE018C5A9F4F0E94831E6896BF
:10543000FFAC6897FF2019F16A968EAD9FAD6A9711
:10544000892B09F0ADC01BC00E941299F80173832B
:10545000628367968FAD679780FFA5C3AC14BD04C8
:1054600071F46A96EEADFFAD6A9760816860608303
:10547000617070E0CE018C5A9F4F0E941C1CD101BC
:1054800012962D903C901397C2CF0E941299DC0186
:10549000CB010F96A11DB11D8093F7099093F809D8
:1054A000A093F909B093FA090E9412990091F309A7
:1054B0001091F4092091F5093091F60906171707A4
:1054C0002807390708F065C0E091F109F091F20969
:1054D00026813781E0963FAF2EAFE097AE014F5F58
:1054E0005F4F7A018E010F5B1F4FBE016D5F7F4FD3
:1054F000AE967FAF6EAFAE97E0968EAD9FADE09764
:105500000097B9F1DC0118968C911897863029F52F
:10551000A096BFAFAEAFA097CE01825A9F4F0E9418
:10552000831EA2968FADA2978823B9F0A4968EAD64
:105530009FADA497892B09F0DAC40FC0873008F01B
:10554000E5C6843009F4F9C4853039F461E070E0CF
:10555000CE0188599F4F0E94C03EE096EEADFFAD50
:10556000E0970280F381E02DE096FFAFEEAFE09789
:10557000C3CF0E941299DC01CB0188579C4EAF4FDC
:10558000BF4F8093F3099093F409A093F509B0936A
:10559000F60980914D0A815080934D0A0C94D332C4
:1055A00067968FAD6797803409F00FC16DE775E09E
:1055B00066968EAD9FAD66970E944BA28C018F2D93
:1055C0000E9446635C010115110509F4E9C0F80168
:1055D0008085853009F0E4C0C8010E9469A5E19684
:1055E0008FAFE197843008F46DC063E0C8010E947A
:1055F0008AA2DC0119968D919C911A97FAE0CF2E20
:10560000C89EF001C99EF00D1124E096FFAFEEAFE9
:10561000E09762E0C8010E948AA2DC0119968D9190
:105620009C911A97C89E4001C99E900C1124240198
:10563000092C000C6608770861E0C8010E948AA264
:10564000E3969FAF8EAFE39760E0C8010E948AA205
:10565000FC01C184D284E384F484C5010B2C000CCA
:10566000AA0BBB0B9C01AD012C193D094E095F092A
:10567000E0966EAD7FADE097CB01770FAA0BBB0B29
:10568000BC01CD0164197509860997090E9451B5BD
:10569000E396AEADBFADE39719962D913D914D9137
:1056A0005C911C972C193D094E095F090E9483B536
:1056B000420E531E641E751EE196BFADE197B530D4
:1056C00099F415C08AE08A9D20018B9D500C11240D
:1056D000052C000C66087708812C912CE0E0F8E29C
:1056E000E096FFAFEEAFE09781E090E009C064E0A4
:1056F000C8010E948AA2DC0119968D919C911A978B
:10570000E096EEADFFADE097AF01FF0F660B770BB4
:1057100044155505660577051CF0B301A20104C0C8
:10572000AA24AA94E3E0BE2E2401092C000C6608EA
:10573000770844155505660577051CF02A013B01DD
:1057400002C0A12CB12CE196FFADE197F23009F037
:10575000BFC26501BB0CEE08FF0860E0C8010E94F3
:105760008AA2FC0181859285A385B485C816D906D5
:10577000EA06FB060CF48CC261E0C8010E948AA212
:10578000FC0181859285A385B4858C159D05AE05A8
:10579000BF050CF074CEC12CD12C7601C3947BC212
:1057A0008AE08A9D20018B9D500C1124052C000C51
:1057B00066087708812C912C20E038E2E0963FAF14
:1057C0002EAFE09781E090E083C2813408F044C2BC
:1057D000843008F054CE42E050E06FEFCE018C5A96
:1057E0009F4F0E94331D67961FAD679716951170E6
:1057F00068962FAD689730E0F901E554FE4E84912C
:10580000F901E957FD4E0491F901E353FD4EF4907F
:10581000FF20A1F081110E94BC61EF2DF0E0EE0F9E
:10582000FF1FEB5DF64EA591B491EC910E2391E034
:1058300080E009F490E0C92ED82E02C0C12CD12CF2
:10584000A12EB12C99249394AC14BD0409F0912C91
:105850006A96EEADFFAD6A978181E82FEF708E2FCB
:1058600090E0FC013197EC30F10508F086C1882703
:10587000EE53FF4F8F4F0C94D8B50E9412999B01A5
:10588000AC01442755276A96EEADFFAD6A97828139
:105890009381BC0180E090E018EEE12E13E0F12E40
:1058A00000E010E00E948054882309F466C16696E7
:1058B0000EAD1FAD66976AE075E0C8010E944BA26D
:1058C000892B09F0CDC16FE075E0C8010E944BA2A1
:1058D000892B09F0C5C1D4C00E9412999B01AC016B
:1058E000442755276A96EEADFFAD6A978281938172
:1058F000BC0180E090E01CE2E12EFF24F39400E084
:1059000010E00E948054882309F437C142E050E03F
:1059100064E0D7C00E9412999B01AC01442755272F
:105920006A96EEADFFAD6A9782819381BC0180E0FB
:1059300090E016E9E12EF12C00E010E00E94805486
:10594000882309F41AC142E050E064E0E6C00E94F6
:1059500012999B01AC01442755276A96EEADFFAD25
:105960006A9782819381BC0180E090E018EEE12E7D
:1059700013E0F12E00E010E00E948054882309F427
:10598000FCC066960EAD1FAD669765E175E0C80177
:105990000E944BA2892B09F067C16BE175E0C80139
:1059A0000E944BA2892B09F05FC16AC00E94129924
:1059B0009B01AC01442755276A96EEADFFAD6A976F
:1059C00082819381BC0180E090E01CE2E12EFF2403
:1059D000F39400E010E00E948054882309F4CDC0C5
:1059E00042E050E069E06DC00E9412999B01AC0159
:1059F000442755276A96EEADFFAD6A978281938161
:105A0000BC0180E090E016E9E12EF12C00E010E00E
:105A10000E948054882309F4B0C042E050E069E05D
:105A20007CC00E9412999B01AC01442755276A96BD
:105A3000EEADFFAD6A9782819381BC0180E090E07A
:105A400018EEE12E13E0F12E00E010E00E948054E9
:105A5000882309F492C066960EAD1FAD669762E288
:105A600075E0C8010E944BA2892B09F001C168E2D0
:105A700075E0C8010E944BA2892B09F0F9C0FCC057
:105A800042E050E06DE074C00E9412999B01AC01AD
:105A9000442755276A96EEADFFAD6A9782819381C0
:105AA000BC0180E090E01CE2E12EFF24F39400E0D2
:105AB00010E00E948054882309F45FC042E050E067
:105AC0006CE0CE018C5A9F4F0E94331D6A960EAD3A
:105AD0001FAD6A970E941299D80113967C936E931A
:105AE00012974BC00E9412999B01AC014427552785
:105AF0006A96EEADFFAD6A9782819381BC0180E02A
:105B000090E016E9E12EF12C00E010E00E948054B4
:105B1000882399F142E050E06CE0CE018C5A9F4F0F
:105B20000E94331D6A960EAD1FAD6A970E941299AE
:105B3000F8017383628321C00E9412999B01AC011A
:105B4000442755276A96EEADFFAD6A97828193810F
:105B5000BC0180E090E018E5E12E12E0F12E00E0BB
:105B600010E00E948054882341F042E050E060E061
:105B7000CE018C5A9F4F0E94331D6A960EAD1FAD09
:105B80006A97D8018C9183FB992790F9991609F4AB
:105B90005EC0982F907E09F457CC982F907E90523B
:105BA0008F71892B57C0692D70E0CE018C5A9F4FA1
:105BB0000E941C1C6A96EEADFFAD6A978181AC1401
:105BC000BD04B1F48F70823079F030F4811136C0A9
:105BD00042E050E061E02AC0853031F0873071F555
:105BE00042E050E06AE022C042E050E066E01EC0C1
:105BF000E82FEF708E2F90E0FC013197ED30F1052A
:105C0000E8F48827E253FF4F8F4F0C94D8B542E059
:105C100050E062E00BC042E050E065E007C042E0C7
:105C200050E067E003C042E050E060E0CE018C5AF3
:105C30009F4F0E94331D882309F421CC6A96EEAD54
:105C4000FFAD6A97808190FA83F9808318CC8F71B9
:105C50008066D8018C9313CC823409F4A7CC0FCC86
:105C600042E050E063E084CF42E050E068E080CF63
:105C700042E050E06BE07CCF64E075E0C8010E9438
:105C80004BA2892B09F0FCCE42E050E066E070CFD9
:105C9000C12CD12C76016A96EEADFFAD6A97828158
:105CA0009381092E000CAA0BBB0B8C159D05AE052C
:105CB000BF0509F4E4CBB601CE018C5A9F4F0E9478
:105CC0001C1C6A96EEADFFAD6A97D382C282D7CB19
:105CD0006A96EEADFFAD6A97428153819501241B10
:105CE000350B37FF03C03195219531098217930792
:105CF00024F480818F71808312C03081232F2295FC
:105D000026952770822F90E006974CF42F5F822F04
:105D10008295880F807E232F2F71282B20838081EE
:105D200082958695877090E00597BCF0C401990C28
:105D3000AA0BBB0B84159505A605B70571F0E09677
:105D40006EAD7FADE097CB01770FAA0BBB0B84152F
:105D50009505A605B70509F092CB4A155B0509F430
:105D60008ECBC301B2010E941EB420E030E040E2BD
:105D700051E40E9477B62B013C0168961FAD6897ED
:105D80006FEA7BE085E89CE00E94199B4AE050E0C6
:105D9000612F85E89CE00E94AE9B6DEA7BE085E880
:105DA0009CE00E94199B22E0B301A20185E89CE0DF
:105DB0000E9477A585E89CE00E94469C6696EEAC22
:105DC000FFAC669765ED74E0C7010E944BA28C01A1
:105DD0006AED74E0C7010E944BA27C01009791F12B
:105DE000DC0118968C911897843061F519966D91A5
:105DF0007C911A9740E450E0CE0101960E9439BA96
:105E00006FE270E0CE0101960E9400BA892B51F436
:105E1000F7012185328543E050E060E4CE01019630
:105E20000E945E69AE014F5B5F4FC301B2010E94E9
:105E3000F5690E94D491882329F080914C0A882327
:105E400009F44DC00115110509F442C0D801189696
:105E50008C918430E9F520E030E0A901C301B20162
:105E60000E941FB720E030E040E05FE387FD05C0FF
:105E7000C301B2010E940BB604C0C301B2010E946B
:105E80000AB60E94E9B623967FAF6EAF2397F8015A
:105E900061857285CE0101960E946D4FCE010196FB
:105EA0000E94C01A882381F0C12CD12CE12CF12C46
:105EB00001E09E012F5B3F4F41E050E060E070E069
:105EC000CE0101960E94D80CCE0101960E94FD4F92
:105ED0006A96EEADFFAD6A97B382A282D0CABE01C8
:105EE0006F5B7F4FCE0101960E943AA2ABCF2EE5A9
:105EF00030E02C0F3D1FAC963FAF2EAFAC9749E979
:105F000052E0AA965FAF4EAFAA97A8963FAF2EAFCA
:105F1000A89761E872E0A6967FAF6EAFA697A196AC
:105F20008FADA197863009F009CB61E070E0CE011A
:105F30008C599F4F0E942E8610CBCE01825A9F4FC4
:105F40000E941FA44B015C010E94129968157905FB
:105F50008A059B0508F401CBA2968FADA297F801A4
:105F6000858396E19683282F30E0F901E957FD4EAD
:105F7000E491D8011796EC931797F901E353FD4E7E
:105F8000E4911896EC93189720E83EE340E050E047
:105F90001D962D933D934D935C93509762E00E9424
:105FA00041620E941299DC01CB01805D9740A109FA
:105FB000B109F80181879287A387B48787E3828B31
:105FC000C8010E9465A4882309F477C0D8011696F9
:105FD0008C918C3009F44BC018F48B30E1F06DC01B
:105FE0008551823008F069C0D8011296DC90129772
:105FF0006D2D6F7770E0762F662713968C91682B46
:1060000080E090E00E941CB42DEC3CEC4CEC5DE395
:106010000E947DB449C0F801628170E080E090E0A8
:106020000E941CB44B015C01D8011396DC90D7FE92
:106030000AC09B01AC0160E070E080E89FEB0E9429
:106040000AB64B015C016D2D6F7070E080E090E04E
:106050000E941EB42DEC3CEC4CEC5DE30E947DB440
:10606000A50194010E940BB64B015C012CC0F80104
:10607000D28063816F7070E080E090E00E941EB477
:106080002DEC3CEC4CEC5DE30E947DB44B015C01DB
:106090006D2D70E080E090E00E941CB49B01AC018B
:1060A000C501B4010E940BB64B015C01D7FE0BC0C9
:1060B000B7FAB094B7F8B09406C0812C912C20ECBC
:1060C000A22E2FE7B22EC8010E9465A48823B9F141
:1060D000F80186818B3098F18D3098F085518230AF
:1060E00070F56081718176276727762780E090E0E0
:1060F0000E941CB42DEC3CEC4CEC5DE30E947DB4A2
:106100001BC0618170E080E090E00E941EB42DEC25
:106110003CEC4CEC5DE30E947DB42B013C01F801AA
:10612000608170E080E090E00E941EB49B01AC01B1
:10613000C301B2010E940BB61B012C0106C0212C29
:10614000312C90EC492E9FE7592EA0966EAC7FAC77
:10615000A0976AED74E0C3010E944BA26C0165ED4B
:1061600074E0C3010E944BA2009781F0FC012085DE
:10617000243061F481859285009741F0DC012C91F7
:10618000222321F0B501A4010E94F588A2967FACDC
:10619000A29765E27CE085E89CE00E94199B4AE0BA
:1061A00050E0672D85E89CE00E94AE9B65E17CE0B5
:1061B00085E89CE00E94199B22E0B501A40185E8D6
:1061C0009CE00E9477A56EE07CE085E89CE00E9460
:1061D000199B22E0B201A10185E89CE00E9477A50D
:1061E0006CE07CE085E89CE00E94199B85E89CE0DF
:1061F0000E94469CC114D10409F47FC0F601808539
:10620000843009F07AC020E030E0A901C501B40172
:106210000E9417B4882309F470C020E030E0A9017F
:10622000C201B1010E9417B4882309F466C0A50118
:106230009401C501B4010E9417B481115EC0A2018E
:106240009101C201B1010E9417B4811156C01A8296
:1062500019828EE3AE96AEADBFADAE971D928A9514
:10626000E9F7F6016185728540E450E0C7010E94BC
:1062700039BA6FE270E0C7010E9400BA892B59F465
:10628000D60119962D913C911A9743E050E060E4B5
:10629000C7010E945E6969E178E0C7010E94F5B913
:1062A000AE014C5A5F4FC501B4010E94F5690E94CE
:1062B000D491882329F080914C0A882309F45CC189
:1062C000F70101900020E9F73197EE19FF09EC0F73
:1062D000FD1F88E48083AE014C5A5F4FC201B101BB
:1062E0000E94F5690E94D491882309F492C080919C
:1062F0004C0A882309F447C18CC00E941299AB0153
:10630000BC0148575C4E6F4F7F4FB2C0883009F0D8
:1063100089C0CE01825A9F4F0E941FA44B015C018D
:106320000E941299681579058A059B0508F415C91C
:10633000A496EEADFFADA4978181A296DFACA297A3
:10634000882309F49BC064E0D69EF0011124E75233
:10635000F64F80809180A280B38066ED7BE085E877
:106360009CE00E94199B4AE050E06D2D85E89CE07E
:106370000E94AE9B62EC7BE085E89CE00E94199B4A
:106380002AE030E0B501A40185E89CE00E94F79B7B
:106390006AED74E0A0968EAD9FADA0970E944BA2CF
:1063A0006C01009709F4C9C0DC0118968C9118970C
:1063B000843009F0C2C019966D917C911A9740E41F
:1063C00050E0C7010E9439BA6FE270E0C7010E9435
:1063D00000BA892B49F4F6012185328543E050E06B
:1063E00060E4C7010E945E69BF92AF929F928F9254
:1063F00021E835E03F932F931F930F930E9490BAAB
:106400000E94D4910FB6F894DEBF0FBECDBF8111AC
:106410008EC00E941299AB01BC014856554C6F4F7B
:106420007F4F26C0803109F098C8CE01825A9F4F15
:106430000E941FA44B015C010E9412996815790506
:106440008A059B0508F489C86AED74E0A0968EADB4
:106450009FADA0970E944BA26C01009709F075C0F8
:106460000E941299AB01BC01405D5A486F4F7F4FAB
:10647000CE01825A9F4F0E945D1E6FC8B5E0BD15C8
:1064800008F443C08CE0E1E7F2E0D70101900D92FF
:106490008A95E1F7F701ED0DF11DED0DF11D60E0BD
:1064A00080810E944162E3E0DE16D9F0ED1538F0FC
:1064B000F1E0DF1671F022E0D21679F006C034E088
:1064C000D31699F045E0D416A1F06EEF75E180E0A7
:1064D00013C06AEF75E181E00FC066EF75E182E0FD
:1064E0000BC062EF75E183E007C06EEE75E184E0FA
:1064F00003C06AEE75E185E00E9481AAA496EEAD24
:10650000FFADA49751E0518328C867E07CE085E89F
:106510009CE00E94199B4AE050E0A2966FADA297C2
:1065200085E89CE00E94AE9B6AED7BE008C080910C
:106530004C0A81116ECFB80129C063EB7BE085E87E
:106540009CE00E94199B0C94AD2ADC0118968C915A
:10655000843009F085CF0E941299AB01BC01C701BC
:106560000E9403690E94D491882309F479CF809115
:106570004C0A882379F074CFBE016C5A7F4FC70153
:106580000E9454A49DCEBE016C5A7F4FC7010E9449
:1065900054A43FCFB701D60119968D919C911A97BB
:1065A0000E9454A45DCFCE58DF4F0FB6F894DEBFE3
:1065B0000FBECDBFDF91CF911F910F91FF90EF9054
:1065C000DF90CF90BF90AF909F908F907F906F9013
:1065D0005F904F903F902F9008950C946F8360EDE3
:1065E0007DE085E89CE00E94199BE0E0F0E01994D2
:1065F000CF93C1E068EE73E080E090E00E946563B5
:106600004AE050E06C2F85E89CE00E94AE9BCF5F93
:10661000C43181F7CF9108950F931F93CF93DF93E8
:10662000CDB7DEB728970FB6F894DEBF0FBECDBF4B
:106630000E94998269E27CE085E89CE00E94199BB7
:10664000CE0101960E94F65DCE0101960E94A05DEA
:106650000CE814E01A8309831B821C821D821E82AF
:10666000CE0107960E94185B8F8198850E94037661
:1066700044E050E0BE016D5F7F4F81E090E00E94FA
:1066800003A10E940276CE0101960E94A05D1A83AA
:1066900009831B821C821D821E82CE0107960E94E6
:1066A000185B8F8198850E94037644E050E0BE011C
:1066B0006D5F7F4F85E090E00E9403A10E9402760B
:1066C000CE0101960E94A05D6FE47CE085E89CE02D
:1066D0000E94199B28960FB6F894DEBF0FBECDBF5F
:1066E000DF91CF911F910F9108955F926F927F92EA
:1066F0008F929F92AF92BF92CF92DF92EF92FF92D2
:106700000F931F93CF93DF93CDB7DEB7A1970FB64B
:10671000F894DEBF0FBECDBF20913C0B30913D0BF6
:106720002115310509F44CC590914D0A9F5F909356
:106730004D0A65E875E0C9010E944BA29093040AD6
:106740008093030A009709F4A3C00E9469A5082F4B
:1067500010E00115110509F49BC0000F111F000F77
:10676000111F8091FC099091FD09892B09F07FC0D0
:10677000C8010E94D1AA9093FD098093FC09109250
:10678000AD0F1092AC0F1092060A1092050A1092EB
:10679000AB0F1092AF0F1092AE0F7801013022E0D4
:1067A00012071CF0E12CA2E0FA2EC70101960E940C
:1067B000D1AA9093B10F8093B00F9093AA0F8093BA
:1067C000A90F8E0D9F1D9093A40F8093A30F0E947D
:1067D00012996093A50F7093A60F8093A70F9093C3
:1067E000A80F80E090E0E091B00FF091B10FE80FBA
:1067F000F91F10820196E816F906ACF782E090E0E6
:106800009093AD0F8093AC0F80E98093C9001092F4
:10681000C8001092CD0083E08093CC008EE080937E
:10682000CA00F0922F02E0922E022091B00F309118
:10683000B10F80912E0290912F02820F931F90939F
:10684000A40F8093A30F232B09F423C369EF7DE0EA
:1068500085E89CE00E94199B6AE070E0C8010E94F4
:1068600066A28DE197E19093A20F8093A10F6FE054
:106870007FE085E89CE00E94199B4AE050E0B80167
:1068800085E89CE00E943F9C85E89CE00E94469C35
:106890006BE875E080913C0B90913D0B0E944BA200
:1068A0008C010097B1F00E9469A58111F9C211C055
:1068B00063EF7EE085E89CE00E94199B4AE050E08F
:1068C000B60185E89CE00E943F9C85E89CE00E9420
:1068D000469C00913C0B10913D0B6FE875E0C801A0
:1068E0000E944BA29093020A8093010A6BE176E02A
:1068F000C8010E944BA29093F60F8093F50F00976A
:1069000009F4ADC12091F70F2111A9C1DC01169640
:10691000ED90FC9017978091F30F9091F40F892BD5
:1069200009F0DAC062E67EE085E89CE00E94199BEF
:1069300085E89CE00E94469C81E190E00E94D1AAFB
:106940008C0188E1F801818312821082108A1786F7
:106950000E944CA31093F40F0093F30F83E190E097
:106960000E94D1AAFC0185E29BE7928B818B168362
:1069700005831482108289E0818311E012831383DE
:10698000F0936B0AE0936A0A80EA90E00E94D1AA31
:106990009093670A8093660A88E290E00E94D1AAE9
:1069A0009093630A8093620A0E944CA38091F30F34
:1069B0009091F40F0E947A6880E39DE00E946968DC
:1069C000811181C06FE47EE085E89CE00E9478A29E
:1069D000C090F30FD090F40FC6010E947A6840E097
:1069E00060EFC6010E94BE78C6010E946C68E0910B
:1069F000F30FF091F40F10836FE27EE085E89CE0E6
:106A00000E9478A28091F30F9091F40F0E942A794E
:106A1000882331F063E27EE085E89CE00E9478A262
:106A2000E091F30FF091F40F8281823059F463E129
:106A30007EE085E89CE00E94199B85E89CE00E942E
:106A4000469C47C000916A0A10916B0A0E941299F5
:106A50004B015C01F0E18F0EF7E29F1EA11CB11CFF
:106A6000D8011596ED91FC9116978FEF83871486C8
:106A7000DF0113963B961D92EA17FB07E1F7F80139
:106A8000148277247394BE01665E7F4FD8011596F9
:106A90008D919C9116970E94FA79181644F40E94E1
:106AA0001299681579058A059B0508F42BC286E6BC
:106AB00096EA9093650A8093640AE0916A0AF091DD
:106AC0006B0A128209C065E07EE085E89CE00E94C6
:106AD00078A280E090E002C081E090E0282F217051
:106AE0002093F70F892B31F063EE7EE085E89CE080
:106AF0000E94199B1092690A1092680A01E010E046
:106B0000E114F10409F4ABC08091F70F882309F474
:106B1000A6C0F7018085863009F09BC0C080D18077
:106B2000CE0101965C01460190E1890E911C350170
:106B3000D6018C910E94686A582EF60181810E94CC
:106B4000686A5294F0EF5F228529D5018D935D012B
:106B5000B2E0CB0ED11C8C149D0451F78091680AD1
:106B60009091690A843191050CF073C0880F991FC8
:106B7000E091620AF091630AE80FF91F1183008324
:106B8000A091680AB091690A53E0AA0FBB1F5A95F9
:106B9000E1F78091660A9091670AA80FB91F88E013
:106BA000F30101900D928A95E1F7C090680AD090A8
:106BB000690A6AE87EE085E89CE00E94199B4AE049
:106BC00050E0B60185E89CE00E943F9C63E87EE0CF
:106BD00085E89CE00E94199B8091680A9091690A5F
:106BE00063E0880F991F6A95E1F72091660A30915A
:106BF000670A820F931F0E94BB5A85E89CE00E949F
:106C0000469C6091680A7091690AE3E0660F771FFD
:106C1000EA95E1F78091660A9091670A680F791FFB
:106C2000FB018081883261F480916A0A90916B0A3D
:106C30000E94395A8091F30F9091F40F0E94F768E7
:106C40008091680A9091690A01969093690A8093ED
:106C5000680AD7011296ED90FC90139751CFE090FF
:106C60003C0BF0903D0B6AE975E0C7010E944BA216
:106C70008C0190934F0A80934E0A60EA75E0C70139
:106C80000E944BA290936F0A80936E0A1092460B5B
:106C90001092450B01151105F9F0F801E680F78017
:106CA00000914E0A10914F0A0115110571F0E1147F
:106CB000F10459F0D70118968C918530A9F7C701D6
:106CC0000E9469A5823080F3A2C1F8018681978174
:106CD0009093460B8093450BE0903C0BF0903D0B5E
:106CE00068E875E0C7010E944BA28C019093F209FD
:106CF0008093F10967EA75E0C7010E944BA2909367
:106D0000000A8093FF090115110509F44CC0809118
:106D10004D0A8F5F80934D0AD80116960D911C91F4
:106D20001797FE0131967F0191E8C92E92E0D92E86
:106D300029E9A22E22E0B22E0115110579F1D80120
:106D400018968C91863031F51A830983C7010E9409
:106D5000831E8C818823F1F0ED81FE813097D1F084
:106D600080913C0B90913D0B892BA1F010821182F8
:106D7000128213828B81843008F099C1823008F02E
:106D8000ACC162E08C810E944162ED81FE81818113
:106D9000807F8183F80102811381CECF80914D0ADB
:106DA000815080934D0A6EEB7EE085E89CE00E9466
:106DB000199B66EB7EE085E89CE00E94199B81E0D0
:106DC00020914E0A30914F0A232B09F480E00E9453
:106DD00064836DEA7EE085E89CE00E94199B81E077
:106DE0002091F1093091F209232B09F480E00E94EF
:106DF000648364EA7EE085E89CE00E94199B81E060
:106E00002091010A3091020A232B09F480E00E94AC
:106E100064836DE97EE085E89CE00E94199B81E037
:106E20002091FF093091000A232B09F480E00E9491
:106E3000648364E97EE085E89CE00E94199B81E020
:106E40002091F50F3091F60F232B09F480E00E947A
:106E5000648385E89CE00E94469C0E944C6A6B011A
:106E60007C016FE87EE085E89CE00E94199B2AE0A7
:106E700030E0B701A60185E89CE00E949B9B85E875
:106E80009CE00E94469C80914D0A815080934D0A5F
:106E900097C162EE7DE085E89CE00E9478A2E1CC9B
:106EA0006FEF680FC8010E948AA2DC011996CD908D
:106EB000DD90ED90FC901C979091260B992359F052
:106EC000809170008E7F809370001092260B10923C
:106ED0002A021092290282E18093280291110E94D5
:106EE000E3775601C6010E940B7801E010E0A0167E
:106EF000B1060CF4DDCC60E0C8010E9441780F5F60
:106F00001F4FF5CF67E0CE014A960E946D7899A198
:106F1000891373C066E975E085E89CE00E944A9C8D
:106F2000F8018081811138C0858196810E942A797B
:106F3000BE01665E7F4FD80115968D919C91169784
:106F40000E94E07840E064EBF801858196810E9420
:106F5000BE78D8011596CD90DC901697C6010E9498
:106F60007A78C6010E947A6867E880E39DE00E9413
:106F7000AB6660E880E39DE00E94AB66C6010E94BC
:106F80006C68C6010E947A78D82EF80185819681B6
:106F90000E942A79D5FE38C0AE014F5F5F4FBE0117
:106FA000665E7F4FC8010E946379D8011196DC901C
:106FB0008A8D803109F4A1C0BE01665E7F4FC80191
:106FC0000E94CC798D1518F4F80181810BC08A8D4F
:106FD000803111F48CE006C0BE01665E7F4FC801AF
:106FE0000E94CC79D80111968C93119714968C91AC
:106FF00014978F5F14968C9346CD68E975E085E809
:107000009CE00E944A9C3FCDF8017082C5CFB70139
:10701000CE0101960E94BA55CE0101960E94C01A77
:107020008823D9F18C859D850097E1F0DC01ED91F5
:10703000FC910484F585E02D1995892B49F08C8508
:107040009D85DC01ED91FC910284F385E02D19957D
:107050008C859D85DC01ED91FC910680F781E02D0A
:1070600019951BC060E070E0CE0101960E941F1BC5
:107070008C0197FFA2C0119501951109AA24A39430
:10708000B12CCE0101960E94FD1BC82ED12C8B8500
:107090008530C1F1863009F45AC0D7011296ED90BF
:1070A000FC901397CE0101960E94FD4FF9CD8630DA
:1070B000D9F060F4853009F06DCEFD8EEC8EBB8E7C
:1070C000AA8ECE014A960E94018864CE803439F09F
:1070D000823409F05FCE60E003C060E053CE62E02E
:1070E0008C810E94416256CEFD8EEC8EDB8ECA8E64
:1070F000CE014A960E944C874DCEFCE0FD1508F467
:1071000063CF68CFCD2829F462E0CE0101960E94BA
:10711000D21B61E0802F0E94416260E0802F0E94BC
:1071200012626BED7EE085E89CE00E94199B4AE0CC
:1071300050E0B80185E89CE00E943F9C66ED7EE04F
:1071400085E89CE00E94199B64ED7EE031C0902EA2
:1071500061E0802F0E94416261E0AB2821F0CA9477
:10716000CD2829F403C0CA94CD2809F060E0C62ECA
:10717000D12C892D0E9412626FEC7EE085E89CE0A4
:107180000E94199B4AE050E0B80185E89CE00E940B
:107190003F9C6DEC7EE085E89CE00E94199B4AE0F4
:1071A00050E0B60185E89CE00E943F9C6BEC7EE0DD
:1071B00085E89CE00E94199B70CFA12CB12C61CF77
:1071C000A1960FB6F894DEBF0FBECDBFDF91CF9171
:1071D0001F910F91FF90EF90DF90CF90BF90AF90F5
:1071E0009F908F907F906F905F90089580911D0A7F
:1071F00090911E0A81709927089580910C0A9091B0
:107200000D0A08956CEA75E085E89CE00E947EA373
:1072100010920D0A10920C0A81E090E0089567EB3D
:1072200075E085E89CE00E947EA340E855E260E0BE
:1072300070E08BE49BE00E941D5481E090E090930D
:107240000D0A80930C0A0895EF92FF920F931F93FB
:10725000CF93DF937C018B0101501109A801BC0180
:107260008BE49BE00E94F797F701329660E0CF0134
:107270008E199F098017910718F48191680FF7CF35
:107280008BE49BE00E947E988BE49BE00E94CB986D
:107290006FEB75E085E89CE00E944A9CE701CE0117
:1072A0008E199F0980179107A8F468816A3050F4FD
:1072B00062EC75E085E89CE00E944A9C40E150E069
:1072C000688102C040E150E085E89CE00E94AE9BEE
:1072D0002196E5CF85E89CE0DF91CF911F910F913A
:1072E000FF90EF900C94469C4F925F926F927F922A
:1072F0008F929F92AF92BF92CF92DF92EF92FF92C6
:107300000F931F93CF93DF93CDB7DEB72A970FB6B6
:10731000F894DEBF0FBECDBF4C015B013A012901DD
:1073200067E97FE0C6010E94BBAC892B09F465C107
:1073300061E97FE0C6010E94BBAC892B09F468C1FA
:107340006BE87FE0C6010E94BBAC892B09F477C1D2
:1073500067E87FE0C6010E94BBAC892B09F480C1BD
:1073600085E0E816F10409F4FBC06CF4B1E0EB161B
:10737000F10409F44EC0E2E0EE16F104F9F0EF2852
:1073800009F06EC181C1F1E4EF16F10409F435C1D1
:1073900054F4A6E0EA16F10409F062C1F20180811A
:1073A0008093360A5DC1B2E4EB16F10409F447C1DB
:1073B000E3E4EE16F10409F053C12AC1D2012D9184
:1073C0003C913093450A2093440AC9010A97459796
:1073D00008F046C180EF820F8093420A002309F42F
:1073E0003FC1032E000C440B550BD4011296ED91B6
:1073F000FC9113970280F381E02D60817181ED9102
:10740000FC910684F785E02D04EC15E0C401199584
:1074100027C11982F5013196E031F10508F08BC0E2
:107420008827E552FF4F8F4F0C94D8B580911D0AE5
:10743000816080933C0A6DE070E08AE192E00E94F6
:107440002439002309F41DC1D4011296ED91FC9159
:1074500013970280F381E02D60817181ED91FC91A1
:107460000288F389E02D29EC35E049EE54E021C093
:1074700080911D0A8E7F80933C0A6DE070E08DE064
:1074800092E00E942439002309F4FBC0D401129633
:10749000ED91FC9113970280F381E02D6081718161
:1074A000ED91FC910288F389E02D29EC35E04CEE5A
:1074B00054E0C4011995E5C01092360A80911D0A66
:1074C000816080933C0A62E87FE031C081E0809374
:1074D000360A80911D0A816080933C0A6DE77FE047
:1074E00026C082E08093360A80911D0A81608093D5
:1074F0003C0A68E77FE01BC084E08093360A8091F5
:107500001D0A816080933C0A64E77FE010C083E03D
:107510008093360A6EEC75E085E89CE00E944A9CF8
:1075200080911D0A816080933C0A6BE67FE0CE016A
:1075300001960E94C4AC002309F492C0D4011296B3
:10754000ED91FC9113970280F381E02D60817181B0
:10755000ED91FC910288F389E02D29EC35E047C0DC
:107560001982B0E1AB16B104C9F054F4FCE0AF16D7
:10757000B10419F583E08093380A62E87FE012C015
:1075800081E1A816B10499F0A2E1AA16B104A9F408
:1075900082E08093380A6BE57FE004C01092380ADD
:1075A00066E67FE0CE0101960E94C4AC0CC081E08B
:1075B0008093380A6FE57FE0F5CF672821F0F2016C
:1075C00080818093380A002309F44AC0D4011296BE
:1075D000ED91FC9113970280F381E02D6081718120
:1075E000ED91FC910288F389E02D23ED35E0AE01A9
:1075F0004F5F5F4FC401199533C0F1E0AF16B1047E
:1076000029F082E0A816B10481F02AC080E50AC002
:10761000A1E0AA16B10429F0B2E0AB16B10429F03A
:1076200007C083E080933B0A1BC010923B0A18C03E
:107630006728B1F0F201808180933A0A11C0F1E02D
:10764000AF16B10441F082E0A816B10449F480916C
:107650003C0A877F03C080913C0A886080933C0A83
:107660001092300A81E08093280A8DE48093290AE1
:107670008FE580932A0A65E270E08FE19AE00E942C
:10768000243981E090E002C08FEF9FEF2A960FB679
:10769000F894DEBF0FBECDBFDF91CF911F910F9148
:1076A000FF90EF90DF90CF90BF90AF909F908F9022
:1076B0007F906F905F904F9008954F925F926F927E
:1076C0007F92AF92BF92CF92DF92EF92FF920F9391
:1076D0001F93CF93DF93CDB7DEB7CB55D1090FB64C
:1076E000F894DEBF0FBECDBF6130710509F027C32E
:1076F0007C010E9412990091190A10911A0A209196
:107700001B0A30911C0A5B016C01A01AB10AC20A63
:10771000D30A49E8A41643E1B406C104D104A4F095
:107720006093190A70931A0A80931B0A90931C0A9B
:1077300068ED75E085E89CE00E947EA36DE070E056
:1077400080E092E00E94243964E670E080E090E0FE
:107750000E9465638BE49BE00E94529818161906FC
:107760000CF0EAC28FE1C82E8AE0D82E94E4A92E4C
:107770009AE0B92E86010E9412996093530B709380
:10778000540B8093550B9093560B8BE49BE00E9417
:10779000309897FFD7C20E9412994090530B509097
:1077A000540B6090550B7090560BDC01CB01841983
:1077B0009509A609B70940904F0B5090500B609067
:1077C000510B7090520B84159505A605B705E8F28C
:1077D0008BE49BE00E945298892B59F062E070E0A4
:1077E00080E090E00E9465638BE49BE00E9430980B
:1077F000EFCF8091430A9091180A891709F49CC22F
:107800008093180A8091420A90E040969093450A2E
:107810008093440A80912C0A90E09093170A8093F9
:10782000160A8091360A90E09093150A8093140A04
:107830008091380A90E09093130A8093120A809105
:107840003A0A90E09093110A8093100A80913C0AC2
:1078500090E090931E0A80931D0A80913B0A90E06D
:1078600090930F0A80930E0A80913E0AF701A2813D
:10787000B3812081318112960D90BC91A02D6D9124
:107880007C91D9015296ED91FC91539720EE35E011
:1078900080FF03C049EE54E002C04CEE54E0C70143
:1078A000199580910E0A90910F0A80389105A9F4DC
:1078B000D7011296ED91FC9113970280F381E02D90
:1078C00060817181ED91FC910288F389E02D27EEB2
:1078D00035E049EE54E0C701199580910E0A909168
:1078E0000F0A892BA9F4D7011296ED91FC911397F9
:1078F0000280F381E02D60817181ED91FC9102881D
:10790000F389E02D27EE35E04CEE54E0C7011995E0
:107910006DEE75E085E89CE00E944A9C6AE070E0AC
:1079200080911D0A90911E0A0E9466A280911D0AF4
:10793000F701A281B3812081318112960D90BC9113
:10794000A02D6D917C91D9015296ED91FC915397A8
:1079500024EF35E083FF03C049EE54E002C04CEE53
:1079600054E0C701199580911D0AF701A281B381E6
:107970002081318112960D90BC91A02D6D917C914A
:10798000D9015296ED91FC9153972BEF35E081FF91
:1079900003C049EE54E002C04CEE54E0C701199513
:1079A0002091100A3091110A032E000C440B550B44
:1079B000D7011296ED91FC9113970280F381E02D8F
:1079C00060817181ED91FC910684F785E02D07E0DF
:1079D00016E0C70119958091120A9091130A892B1C
:1079E000A9F4D7011296ED91FC9113970280F381CF
:1079F000E02D60817181ED91FC910288F389E02D89
:107A000023ED35E04EE056E0C70119958091120A4A
:107A10009091130A0197A9F4D7011296ED91FC9168
:107A200013970280F381E02D60817181ED91FC91CB
:107A30000288F389E02D23ED35E043E156E0C701EC
:107A400019958091120A9091130A0297A9F4D7010F
:107A50001296ED91FC9113970280F381E02D6081E5
:107A60007181ED91FC910288F389E02D23ED35E0E1
:107A70004AE156E0C70119958091120A9091130AC4
:107A80000397A9F4D7011296ED91FC911397028008
:107A9000F381E02D60817181ED91FC910288F38981
:107AA000E02D23ED35E04EE156E0C70119958091B8
:107AB000100A9091110AF701A281B38120813181CE
:107AC00012960D90BC91A02D6D917C91D90152968A
:107AD000ED91FC91539727E036E0892B19F44CEE99
:107AE00054E002C049EE54E0C70119952091440AC0
:107AF0003091450A032E000C440B550BD70112960A
:107B0000ED91FC9113970280F381E02D60817181EA
:107B1000ED91FC910684F785E02D04EC15E0C7019A
:107B200019952091160A3091170A032E000C440B68
:107B3000550BD7011296ED91FC9113970280F381BA
:107B4000E02D60817181ED91FC910684F785E02D37
:107B500003E216E0C70119952D961FAE2D9780916F
:107B6000140A9091150A009719F462E87FE016C094
:107B70008130910519F46DE77FE010C082309105E6
:107B800019F468E77FE00AC08330910519F46BE6C9
:107B90007FE004C0049739F464E77FE0CE01845BA2
:107BA0009F4F0E94C4AC2091140A3091150A032EF5
:107BB000000C440B550BD7011296ED91FC911397D5
:107BC0000280F381E02D60817181ED91FC9106844A
:107BD000F785E02D09E216E0C701199580911D0A8D
:107BE000F701A281B3812081318112960D90BC9161
:107BF000A02D6D917C91D9015296ED91FC915397F6
:107C000029EC35E080FF04C0AE01445B5F4F02C049
:107C10004CEE54E0C701199568961FAE1EAE6897EA
:107C20006A961FAE1EAE6A976C961FAE1EAE6C971C
:107C300040E050E06BED78E0CE018A5A9F4F0E9401
:107C40008F99F60160816A3058F441E050E062ECAF
:107C500075E0CE018A5A9F4F0E949C71D6016C91AB
:107C6000CE0101960E94CA714D815E8169817A813F
:107C7000CE018A5A9F4F0E949C7189819A810E94ED
:107C800069ABBFEFCB1ADB0AAC14BD04D1F6689622
:107C90000EAD1FAD68970115110569F0F8018081DF
:107CA000882349F0082E000C990B0E9498B9D8013E
:107CB0008D938D01F3CF6C960EAD1FAD6C970115B2
:107CC000110511F4198215C00A34110510F00AE4E7
:107CD00010E068966EAD7FAD6897A801CE01019661
:107CE0000E9439BAE1E0F0E0EC0FFD1FE00FF11F58
:107CF0001082D7011296ED91FC9113970280F381C7
:107D0000E02D60817181ED91FC910288F389E02D75
:107D10002FE236E0AE014F5F5F4FC7011995BE01FC
:107D20006F5F7F4F85E89CE00E947EA368968EADD2
:107D30009FAD68970E9469AB84E690E00BC080E03D
:107D400090E008C0F80181938F01AE16BF0609F0DC
:107D500012CD3ECDC55ADF4F0FB6F894DEBF0FBE31
:107D6000CDBFDF91CF911F910F91FF90EF90DF90EA
:107D7000CF90BF90AF907F906F905F904F9008959D
:107D80008F929F92AF92BF92CF92DF92EF92FF922B
:107D90000F931F93CF93DF93CDB7DEB760970FB6E6
:107DA000F894DEBF0FBECDBF8C018091070A811110
:107DB00003C064E47FE009C160E083E00E941262D6
:107DC00061E070E080E090E00E946563BE016F5F5B
:107DD0007F4F80E00E94B9A2892B09F0F4C089810D
:107DE00083FFF1C044E0BE016F5F7F4F82E00E94DD
:107DF000C754009791F429813A81322723273227EB
:107E000030934A0D2093490D2B813C813227232743
:107E100032273093480D2093470D0E9497A264E3C8
:107E200076E085E89CE00E944A9C6091490D709143
:107E30004A0D80E090E00E941CB46B017C0122E0BE
:107E4000AB01BC0185E89CE00E9477A56AE376E07F
:107E500085E89CE00E944A9C6091470D7091480D16
:107E600080E090E00E941CB44B015C0122E0AB0179
:107E7000BC0185E89CE00E9477A562E476E085E895
:107E80009CE00E944A9C42E0BE016F5F7F4F81E10F
:107E90000E94C75449815A81892B21F454274527D0
:107EA000542702C040E050E060E070E04093080AD0
:107EB0005093090A60930A0A70930B0A2AE030E093
:107EC00085E89CE00E94F79B20E030E44CE156E41A
:107ED000C701B6010E9417B487FF22C02EE436E026
:107EE000B701A601C8010E94B51F23E536E0B50120
:107EF000A401C8010E94B51F4091080A5091090AC7
:107F000060910A0A70910B0ACE0101960E940369E2
:107F100049E556E0BE016F5F7F4FC8010E947F1F99
:107F20006FE576E085E89CE00E947EA3BE016F5F6E
:107F30007F4F80EE0E94B9A2892B19F419811F3F4F
:107F400039F461E676E085E89CE00E947EA334C0C7
:107F500015FF06C062E876E085E89CE00E944A9C36
:107F600014FF06C066E976E085E89CE00E944A9C22
:107F700013FF06C069EA76E085E89CE00E944A9C0F
:107F800012FF06C06EEB76E085E89CE00E944A9CFA
:107F900011FF06C065ED76E085E89CE00E944A9CF2
:107FA00010FF06C06BEE76E085E89CE00E944A9CDC
:107FB00085E89CE00E94469C61E083E00E9412629A
:107FC00081E090E00CC069E27FE085E89CE00E94DF
:107FD000199B85E89CE00E94469C80E090E06096BA
:107FE0000FB6F894DEBF0FBECDBFDF91CF911F91CA
:107FF0000F91FF90EF90DF90CF90BF90AF909F9048
:108000008F900895FC01848195810895089580E002
:1080100090E00895AF92BF92CF92DF92EF92FF92DD
:108020000F931F93CF93DF93CDB7DEB7C154D10920
:108030000FB6F894DEBF0FBECDBF5C016B018A01A5
:1080400069ED70E185E89CE00E94199BB50185E827
:108050009CE00E944A9C66ED70E185E89CE00E94ED
:10806000199BC114D10409F4A1C00C0D1D1DF80108
:1080700010820E944C6A6A3F71051CF461ED70E148
:108080004DC07601E016F10641F0F70161917F01E4
:1080900085E89CE00E94129BF5CF85E89CE00E9459
:1080A000469C80914A0A90914B0A9E012F5F3F4F58
:1080B000790120E030E0039719F443E050E019C063
:1080C00042E050E061E4C7010E945E69F70101905F
:1080D0000020E9F731978F010E191F09A801B70198
:1080E000C5010E942BBA0097A9F020E030E041E0E2
:1080F00050E061E4C7010E945E69F7010190002031
:10810000E9F731978F010E191F09A801B701C501C1
:108110000E942BBA892B39F066EC70E185E89CE06F
:108120000E94199B43C00A0D1B1D6DEF76E0C8012C
:108130000E940BBA892B69F4F60101900020E9F73F
:108140003197EC19FD09329720F0C6010E94E7959E
:108150002DC06FE270E0C8010E9400BA5C01009778
:1081600041F0FC0110828181843201F1FFEFAF1AEE
:10817000BF0AF80180818432C9F0B801C7010E94AA
:108180006D4FC7010E94C01A882369F041E08091B9
:108190004A0A90914B0A039709F440E09501B60111
:1081A000C7010E94A618C7010E94FD4FCF5BDF4F99
:1081B0000FB6F894DEBF0FBECDBFDF91CF911F91F8
:1081C0000F91FF90EF90DF90CF90BF90AF90089508
:1081D000CF93DF93EC0168EE7FE085E89CE00E949E
:1081E000199B60E074E0CE01DF91CF910C94831B6A
:1081F0006F927F928F929F92AF92BF92CF92DF92B7
:10820000EF92FF920F931F93CF93DF93CDB7DEB71B
:108210002C970FB6F894DEBF0FBECDBF4C01762E63
:10822000672E6A01590181E090E09093440B80939E
:10823000430B40E855E260E070E088EE9BE00E946E
:108240001D547092F70D88EE9BE09093F60D80938D
:10825000F50D1092020F1092040F1092030F0115EA
:10826000110541F00130110539F4FE2CEE24EE2405
:10827000EA9402C0FF24FA94C701A0E0B0E0898329
:108280009A83AB83BC8380E190E09E838D83A601BB
:1082900060E070E04F83588769877A879C878B8777
:1082A0004AE050E0672D762D85E89CE00E943F9CD7
:1082B00061E970E185E89CE00E94199BBE01695F5D
:1082C0007F4F85E89CE00E940A1C8C016DE870E1FC
:1082D0000E94199B4AE050E0B501C8010E943F9CF2
:1082E0006AE870E1C8010E94199BBE016F5F7F4F71
:1082F000C8010E940A1C0E94469CA114B10491F07E
:1083000082E0A816B10409F5D0927D0EC0927C0ED1
:1083100010927F0E10927E0EF092810EE092800EEF
:1083200086E010C0D0927D0EC0927C0EE11003C09A
:1083300080E090E002C080E09FEF90937F0E8093FA
:108340007E0E85E00E94665107C062E770E185E815
:108350009CE00E94199B80E01092440B1092430B0A
:10836000882331F0C4010E94E84080E090E002C020
:1083700081E090E02C960FB6F894DEBF0FBECDBF23
:10838000DF91CF911F910F91FF90EF90DF90CF90F1
:10839000BF90AF909F908F907F906F900895DF92E5
:1083A000EF92FF920F931F93CF93DF9300D000D0F3
:1083B000CDB7DEB76EED70E185E89CE00E94199BB9
:1083C0000FE11BE0D12C80E1E82EF12CF801808137
:1083D000803130F462EC75E085E89CE00E944A9CB4
:1083E000F8018081F5E090E0A0E0B0E089839A8315
:1083F000AB83BC83FE82ED82BE016F5F7F4F85E859
:108400009CE0DF1639F00E940A1C6CED70E10E94BE
:10841000199B04C00E940A1C0E94469CD3940F5FC3
:108420001F4F86E0D812D2CF26960FB6F894DEBF43
:108430000FBECDBFDF91CF911F910F91FF90EF90B5
:10844000DF900895CF92DF92EF92FF9280913C0BE4
:1084500090913D0B892B09F47DC061EB70E185E8BB
:108460009CE00E94199B80914D0A8823E9F00E94AC
:108470005C968091F70F882341F08091F50F9091E1
:10848000F60F892B11F00E94A46A0E94EF1E8091C2
:108490004A0A90914B0A039711F00E94088C0E949F
:1084A00080890E94C929DFCF1092460B1092450B9C
:1084B0000E944C6A6B017C0169E970E185E89CE0EF
:1084C0000E94199B2AE030E0B701A60185E89CE0F4
:1084D0000E949B9B80913C0B90913D0B0E94C45647
:1084E00010923D0B10923C0B1092F2091092F10980
:1084F00010924F0A10924E0A10926F0A10926E0A52
:108500001092000A1092FF091092040A1092030AB6
:108510001092F60F1092F50F1092020A1092010AB3
:108520000E944C6A6B017C0164E970E185E89CE083
:108530000E94199B2AE030E0B701A60185E89CE083
:108540000E949B9B85E89CE0FF90EF90DF90CF908E
:108550000C94469CFF90EF90DF90CF9008958F92FF
:108560009F92BF92CF92DF92EF92FF920F931F9351
:10857000CF93DF93CDB7DEB7C854D1090FB6F894C7
:10858000DEBF0FBECDBF7C018B010E94FD1BB82E4C
:108590004801882428E0922213FD06C080914A0AEF
:1085A00090914B0A039781F4B80166277370C70155
:1085B0000E94831B61E670E185E89CE00E94199BA4
:1085C00088248A94982CF7C160E073E0C7010E9468
:1085D000BB1B082B192B1AAA19AAFE01F3968EE0D1
:1085E000DF011D928A95E9F723961FAE1EAE2397F1
:1085F000709686E0DF011D928A95E9F711FF63C04E
:10860000F70183859485009719F4C284D12C08C0A2
:10861000DC01ED91FC91028CF38DE02D19956C013C
:10862000C7010E94051BB6E0CB16D104B1F19E0133
:108630002F5C3F4FE7E0CE16D10444F4F1E0CF1AAF
:10864000D10842E0C416D10438F029C0A7E0CA1608
:10865000D10429F597FF13C01F926F931F927F9348
:108660009F779F938F9386E097E09F938F931F92BE
:1086700080E18F933F932F930E9453BA1FC01F92A4
:108680006F938CE097E09F938F931F9280E18F937D
:108690003F932F930E9453BA11C01D7F14C09F9324
:1086A0008F937F936F938CE097E09F938F931F92AC
:1086B00080E18F933F932F930E9453BA0FB6F894A3
:1086C000DEBF0FBECDBF10FF1EC08B2D90E08D30E2
:1086D000910590F4FC018827E551FF4F8F4F0C94D2
:1086E000D8B56EE570E102C06AE570E1CE018F5B3E
:1086F0009F4F0E94C4AC07C06CE470E185E89CE029
:108700000E94199B1E7F20E030E043E050E060E3D0
:10871000CE0101960E945E69D7011296ED91FC91FF
:108720001397608171814FE250E0CE0101960E9463
:108730001BBA0E94D491882309F439C180914C0A54
:10874000811135C16801CC24B2E0DB2211FF2DC0BC
:108750008B2D90E08230910541F1059731F1BE01FA
:108760006F5C7F4FCE0101960E943AA266E470E1F1
:1087700085E89CE00E94199BBE016F5F7F4F85E8F2
:108780009CE00E944A9C63E470E185E89CE00E94C2
:10879000199BBE016F5C7F4F85E89CE00E944A9C5C
:1087A00085E89CE00E94469C2AC010FF25C0BE01BF
:1087B0006F5B7F4FCE0101960E943AA26DE370E19C
:1087C00085E89CE00E94199BBE016F5F7F4F85E8A2
:1087D0009CE00E944A9C6AE370E185E89CE00E946C
:1087E000199BBE016F5B7F4F85E89CE00E944A9C0D
:1087F00085E89CE00E94469CCD2809F457C020E003
:1088000030E043E050E060E3CE0101960E945E69F3
:10881000D7011296ED91FC911397608171814FE21F
:1088200050E0CE0101960E941BBA6BE775E0CE01C5
:1088300001960E94F5B940E350E066E370E1CE0195
:1088400001960E94CBAC60E370E185E89CE00E9459
:10885000199BBE016F5F7F4F85E89CE00E944A9C98
:108860006DE270E185E89CE00E94199BBE016F5C9F
:108870007F4F85E89CE00E944A9C85E89CE00E942E
:10888000469C0E94D491882309F491C080914C0A9F
:1088900081118DC0BE016F5C7F4FCE0101960E9499
:1088A0003AA260E072E0C7010E94491B10FF7BC042
:1088B000BAE0BB1681F0BB1538F0E1E0BE1689F0D6
:1088C000F6E0BF1671F019C02BE0B21639F04CE09B
:1088D000B41661F012C063E270E10AC06EE170E1AB
:1088E00007C0D7011A968C91853039F468E270E19F
:1088F000CE018F5B9F4F0E94C4AC20E030E043E08C
:1089000050E060E3CE0101960E945E69D7011296A5
:10891000ED91FC911397608171814FE250E0CE019F
:1089200001960E941BBA6BE775E0CE0101960E948A
:10893000F5B940E350E06AE170E1CE0101960E9492
:10894000CBAC64E170E185E89CE00E94199BBE011C
:108950006F5F7F4F85E89CE00E944A9C61E170E177
:1089600085E89CE00E94199BBE016F5B7F4F85E804
:108970009CE00E944A9C85E89CE00E94469C0E94E4
:10898000D4918823A1F080914C0A811110C0BE01BE
:108990006F5B7F4FCE0101960E943AA260E071E0CA
:1089A000C7010E94491B88248394912C04C0B801FC
:1089B000C7010E94831BC401C85BDF4F0FB6F89448
:1089C000DEBF0FBECDBFDF91CF911F910F91FF9002
:1089D000EF90DF90CF90BF909F908F9008958F92EF
:1089E0009F92AF92BF92EF92FF920F931F93CF93FC
:1089F000DF93CDB7DEB769970FB6F894DEBF0FBE31
:108A0000CDBFDC011496ED91FC91159720852430A3
:108A100009F0D6C0942EA62E7C0161857285CE0108
:108A200001960E946D4FCE0101960E94C01A8823C4
:108A300009F454C08B85893009F050C060E070E0C3
:108A4000CE0101960E941F1BB82E192F68E070E11D
:108A500085E89CE00E94199B4AE050E06B2D712F45
:108A600085E89CE00E943F9C66E070E185E89CE020
:108A70000E94199B4AE050E06A2D0A2C000C770BEB
:108A800085E89CE00E943F9C60E070E185E89CE006
:108A90000E94199B4AE050E0692D092C000C770BCD
:108AA00085E89CE00E943F9C85E89CE00E94469CF3
:108AB0000091430B1091440B0115110591F0692DA4
:108AC000C7010E94D21B4A2DAA0C550B660B770BCF
:108AD000C7010E94CD1AC7010E94E84000E010E0E3
:108AE0006AC081E090E09093440B8093430B40E890
:108AF00055E260E070E088EE9BE00E941D54B09269
:108B0000F70D88EE9BE09093F60D8093F50D109293
:108B1000020F1092040F1092030FB2E09B1609F49B
:108B200057C085E0981609F453C06A2DAA0C770B3C
:108B3000880B990B0E941EB422E538EB42E152E407
:108B40000E940BB620E030E040E251E40E947DB488
:108B50002DEE3EE94CE35EE30E9477B64B015C01EB
:108B600020E030E0A9010E941FB720E030E040E0A3
:108B70005FE387FD28C0C501B4010E940BB60E94C7
:108B8000E9B683ED97E090937D0E80937C0E109272
:108B90007F0E10927E0E7093810E6093800E86E0A1
:108BA0000E9466511092440B1092430B882399F057
:108BB000C7010E94E840CE0101960E94FD4F0EC001
:108BC00000E010E00BC0C501B4010E940AB6D7CF87
:108BD00060E070E0D6CF01E010E0EDCFC80169960B
:108BE0000FB6F894DEBF0FBECDBFDF91CF911F91BE
:108BF0000F91FF90EF90BF90AF909F908F9008954E
:108C0000DF92EF92FF920F931F93CF93DF93EC01CC
:108C1000E62ED42E60E070E00E941F1BF82E192F64
:108C20006CEF7FE085E89CE00E94199B4AE050E0F1
:108C30006F2D712F85E89CE00E943F9C6AEF7FE0DA
:108C400085E89CE00E94199B6E2D0E2C000C770B82
:108C50004AE050E085E89CE00E943F9C85E89CE06B
:108C60000E94469C0091430B1091440B0115110585
:108C700091F06D2DCE010E94D21B4E2DEE0C550BA6
:108C8000660B770BCE010E94CD1ACE010E94E84000
:108C900000E010E05EC081E090E09093440B809390
:108CA000430B40E855E260E070E088EE9BE00E94F4
:108CB0001D54F092F70D88EE9BE09093F60D809393
:108CC000F50D1092020F1092040F1092030F80ED19
:108CD00097E090937D0E80937C0E10927F0E109201
:108CE0007E0EEE2039F085E090E09093810E809327
:108CF000800E04C01092810E1092800E86E00E94B9
:108D0000665162E370E080E090E00E94656382ED6E
:108D100097E090937D0E80937C0E10927F0E1092C0
:108D20007E0E8E2D94E68902A00111245093810EAF
:108D30004093800E86E00E9466511092440B109280
:108D4000430B882321F0CE010E94E84002C001E0DD
:108D500010E0C801DF91CF911F910F91FF90EF902C
:108D6000DF9008952F923F924F925F926F927F9281
:108D70008F929F92AF92BF92CF92DF92EF92FF922B
:108D80000F931F93CF93DF9300D01F92CDB7DEB721
:108D90006C013B010E94FD1B823011F0853011F403
:108DA000612C712CF6010480F581E02DFC83EB83AE
:108DB0008085853009F076C0CF010E9469A5E82E34
:108DC000F12CF2E0EF16F1040CF46CC060E08B8142
:108DD0009C810E948AA2FC014184528461E08B81C3
:108DE0009C810E948AA2FC0181849284A384B48421
:108DF0008091430B9091440B9A83898392E0E9160A
:108E0000F10409F44CC062E08B819C810E948AA22B
:108E1000FC0101851285F3E0EF16F10409F443C06B
:108E200063E08B819C810E948AA2FC0121843284B0
:108E3000F4E0EF16F10449F064E08B819C810E941C
:108E40008AA2FC018185928502C082E090E09C8329
:108E50008B8321143104B1F0E981FA81EF2B31F0D9
:108E6000C6010E94E84080E090E025C09301D10156
:108E70000E94EFB524E630E040E050E00E9483B568
:108E8000790105C089819A81892B51F773012B8162
:108E90003C81A401B201C6010E94F8400CC00FEF52
:108EA0001FEF01C008C08FE3282E312CE2E0F0E074
:108EB000FC83EB83D1CF0F900F900F900F90DF9139
:108EC000CF911F910F91FF90EF90DF90CF90BF90C7
:108ED000AF909F908F907F906F905F904F903F905A
:108EE0002F900895EF92FF920F931F93CF93DF93EC
:108EF000CDB7DEB769970FB6F894DEBF0FBECDBF12
:108F00007C01DC011296ED91FC91139760817181D7
:108F100085E89CE00E944A9CC7010E94C01A81110A
:108F20000DC06FED7FE085E89CE00E94199B85E80D
:108F30009CE00E94469C8FEF9FEFAFC0C7010E944C
:108F4000FD1BF70112851730F1F0853099F028F4F8
:108F5000813049F0823071F016C0863021F0E6EFA2
:108F6000E80FE33080F466ED7FE085E89CE00E9446
:108F7000199B91C06BEC7FE085E89CE00E94199BF7
:108F800080E090E08AC0D7011B968D919C911C9740
:108F9000009741F0DC01ED91FC910688F789E02D06
:108FA00019957BC0C7010E94051B812F90E08A3074
:108FB000910508F054C0FC018827E850FF4F8F4FFF
:108FC0000C94D8B5D7011496ED91FC911597808536
:108FD000853009F047C065EC7FE085E89CE00E94A1
:108FE000199BD7011496ED91FC9115970681178175
:108FF0000115110561F1F8018085843011F5618555
:109000007285CE0101960E946D4FCE0101960E949D
:10901000C01A882391F0CE0101960E94724718165B
:1090200019065CF46CEB7FE085E89CE00E94199BDC
:10903000CE0101960E94FD4F2EC0CE0101960E94E6
:10904000FD4FD80112960D911C911397D1CF61EB72
:109050007FE092CF062F10E007C08B0105C067EAC2
:109060007FE08ACF00E010E06CE97FE085E89CE0DB
:109070000E94199B4AE050E0B80185E89CE00E94FC
:109080003F9C85E89CE00E94469C81E090E0012B9B
:1090900021F480E002C081E074CF69960FB6F894A5
:1090A000DEBF0FBECDBFDF91CF911F910F91FF901B
:1090B000EF900895FC01878190859C0144E03595EF
:1090C00027954A95E1F756E0959587955A95E1F7EA
:1090D0002817390719F081E090E0089582E090E0C8
:1090E000089580E090E008958091480A9091490A9F
:1090F000089583E090E008958091460A9091470A90
:109100000895CF93FC01828193810E94051BC62F95
:1091100067E371E185E89CE00E94199B4AE050E01A
:109120006C2F85E89CE00E94AE9B85E89CE00E9445
:10913000469C8C2F90E0CF910895FC018281938111
:109140000E94051BCB0108952F923F924F925F9290
:109150006F927F928F929F92AF92BF92CF92DF9247
:10916000EF92FF920F931F93CF93DF93CDB7DEB7AC
:109170002D970FB6F894DEBF0FBECDBF5C012B015B
:109180005D874C871901098747013601FC018281FF
:1091900093810E9472479B878A87EE24E394181676
:1091A00019060CF0E12C1414150434F48114910404
:1091B00019F488248394912C1E821D82F5018481E8
:1091C0009581019798878F8361147104D1F0CE0146
:1091D00007969F938F9302979F938F938FE097E0CB
:1091E0009F938F937F926F920E94BFBA0FB6F894AD
:1091F000DEBF0FBECDBF019721F48D819E81988780
:109200008F830F8118856D817E814AE050E085E86B
:109210009CE00E943F9C6CE771E185E89CE00E9425
:10922000199B4AE050E0B80185E89CE00E943F9C11
:1092300066E771E185E89CE00E94199B4AE050E0F6
:10924000B20185E89CE00E943F9C85E89CE00E947A
:10925000469C34E08316910464F482E088169104FD
:1092600044F58114910419F18A94892809F491C074
:109270006CC1E4E08E16910409F067C1F1018081B0
:10928000898382818A8384818B831C820F811885E4
:109290002D813E81CC24C39440E050E0BE016F5F3D
:1092A0007F4FC5010E94AC5E60E07AE046C1EE24CB
:1092B000E394F501828193810E94051B69837A837F
:1092C0008B839C832C853D852230310581F02330B2
:1092D0003105C1F02130310521F5F101808189830B
:1092E0008C8187FD1EC01B821A8280E819C0F101A3
:1092F00080818B838181982F9F778C8180782281D8
:109300002A830CC0F10180818B838181982F9F7704
:109310008C81807822812A8324812983892B80680B
:109320008C830F8118852D813E81C12C40E050E057
:10933000BE016F5F7F4FC5010E94AC5E672809F0D8
:1093400001C149815A816B817C81F50182819381C0
:109350000E94CD1AF501828193818928B9F42A856A
:109360003B85121613062CF4298121110CC062E0F2
:1093700008C0EA85FB85EF2B31F42981222319F0FF
:1093800061E00E94D21B60E07BE0D7C060E07AE041
:10939000D7C0642DF501828193810E94D21BF1E038
:1093A0004F16510431F022E04216510409F4A2C0D4
:1093B000CCC0F50102811381C8010E94051B69839D
:1093C0007A838B839C83672851F00F8118852D81C8
:1093D0003E81C12CEE24E39441E050E096C0672B1F
:1093E000682B692B41F08981893128F4F985FF23A5
:1093F00011F088E2898349815A816B817C81C8019F
:109400000E94CD1A89819A81AB81BC81892B8A2BDC
:109410008B2BE1F12985222339F060E073E0F5011F
:10942000828193810E94AF420981EA809B801C81E6
:109430001F776BE671E185E89CE00E94199B4AE08A
:1094400050E0692D712F85E89CE00E94A89B69E699
:1094500071E185E89CE00E94199B4AE050E06E2D86
:1094600085E89CE00E94AE9B67E671E185E89CE0A0
:109470000E94199B4AE050E0602F85E89CE00E9422
:10948000AE9B85E89CE00E94469C2AC02AE030E022
:1094900040E050E0BA0185E89CE00E94F79B69E457
:1094A00071E185E89CE00E94199B94E69B838C8186
:1094B0001A829983807880688C8349815A816B8174
:1094C0007C81F501828193810E94CD1AF985FF2369
:1094D00039F060E073E0F501828193810E94AF4230
:1094E0000F8118852D813E81C12CEE24E39440E04C
:1094F00050E00BC02D813E810F811885672861F0F7
:10950000C12CEE24E39442E050E0BE016F5F7F4F38
:10951000C5010E94AC5E16C01982C12CEE24E394F2
:1095200040E050E0BE016F5F7F4FC5010E94AC5E1E
:10953000F985FF2339F060E071E0F50182819381C4
:109540000E94AF4281E090E00CC06DE371E185E8DC
:109550009CE00E94199B85E89CE00E94469C80E06C
:1095600090E02D960FB6F894DEBF0FBECDBFDF9111
:10957000CF911F910F91FF90EF90DF90CF90BF9010
:10958000AF909F908F907F906F905F904F903F90A3
:109590002F9008950C9469AB0C9469ABCF93DF9333
:1095A00065E177E085E89CE00E947EA3E091600A97
:1095B000F091610A4481558160E070E08185928577
:1095C0000E9442B3C091600AD091610A209771F065
:1095D00089859A850E9469AB8E819F8197FD03C022
:1095E00060E00E944162CE010E9469AB1092490A7C
:1095F0001092480A81E090E0DF91CF910895CF93D7
:10960000DF93EC0165E277E085E89CE00E947EA3B1
:1096100060E08C810E94126260E08D810E94126283
:1096200040E050E0BA018A819B810E94635510920C
:10963000470A1092460A81E090E0DF91CF910895A9
:109640006F927F928F929F92AF92BF92CF92DF9252
:10965000EF92FF920F93CF93DF93EC016B014A01DE
:1096600059018A819B810E9472473C011C141D0490
:1096700034F4E114F10419F4EE24E394F12C60E0E5
:1096800070E18A819B810E94831B81E0E816F104CE
:1096900009F440C0E2E0EE16F10451F0E114F104E7
:1096A00009F0C5C066E271E185E89CE00E94199B63
:1096B000A114B10409F4C5C0892809F4C2C0F50198
:1096C00080809180092C000CAA08BB08B501A40178
:1096D0008A819B810E94CD1A8A819B81EF28A9F4FF
:1096E0001614170434F489288A288B2859F462E068
:1096F00007C0672839F489288A288B2819F061E087
:109700000E94D21B60E07BE071C060E07AE00E94C2
:10971000AF428AC06C2D8A819B810E94D21BF1E0EE
:10972000CF16D10431F082E0C816D10409F45AC032
:109730007EC0AA80BB80C5010E94051B6B017C0115
:10974000611571058105910561F06931710581052A
:1097500091053CF4002329F088E2C82ED12CE12C9D
:10976000F12CB701A601C5010E94CD1AC114D10484
:10977000E104F104D9F0002331F060E073E08A8164
:109780009B810E94AF426BE171E185E89CE00E9401
:10979000199B2AE030E0B701A60185E89CE00E9411
:1097A000F79B85E89CE00E94469C24C02AE030E0BC
:1097B00040E050E0BA0185E89CE00E94F79B6DEF25
:1097C00070E185E89CE00E94199B44E650E060E06F
:1097D00070E08A819B810E94CD1A002359F060E0DD
:1097E00073E004C0002331F060E071E08A819B8166
:1097F0000E94AF428A819B810E944955672B682B4A
:10980000692B91F00E9412994F8158856A01550F7A
:10981000EE08FF08AB01BC014C0D5D1D6E1D7F1DE8
:109820008A819B810E94635581E090E00CC061EFCA
:1098300070E185E89CE00E94199B85E89CE00E940D
:10984000469C80E090E0DF91CF910F91FF90EF90E8
:10985000DF90CF90BF90AF909F908F907F906F9050
:1098600008954F925F926F927F928F929F92AF92E4
:10987000BF92CF92DF92EF92FF920F931F93CF93FD
:10988000DF93EC010A811B8160E070E1C8010E9456
:10989000BB1B892B09F48FC160E070E2C8010E94F4
:1098A000BB1B892B79F480912702882309F483C19B
:1098B00060E070E2C8010E94831B80912702815002
:1098C000809327020A811B81C8010E9449556B01C0
:1098D0007C01C8010E94FD1B823049F018F48130E0
:1098E00049F00DC0853019F0863021F008C000E045
:1098F00010E007C0C8010E94051B8B0102C00FEFDA
:109900001FEF8E819AEC980F903158F549845A8454
:10991000612C712C8B849C84A12CB12C0E944663F9
:10992000092E000CAA0BBB0B9C01AD0128193909AB
:109930004A095B09A4E6B0E00E94A2B5A301920126
:10994000281939094A095B090E9483B5590137FD75
:1099500027C1253631050CF425C184E6A82EB12C8B
:1099600021C1C114D104E104F104D1F0AA24AA94C4
:10997000BA2C0E941299C616D706E806F90658F4C2
:1099800063EE70E185E89CE00E94199B85E89CE00D
:109990000E94469CDEC08FEFA816B80609F008C1E9
:1099A000025311090E3F8FEF18070CF05DC060E005
:1099B0008D810E9412628A819B810E944955672B8A
:1099C000682B692B91F40E9412994F8158856A0186
:1099D000550FEE08FF08AB01BC014C0D5D1D6E1D5F
:1099E0007F1D8A819B810E946355FC808EEF8F0DC5
:1099F0008C3020F084ED8F0D833038F4AA27BB27FC
:109A0000A01BB10B2FEF30E05DC08D819EEF980F52
:109A100061E09C3020F08C52833008F096C08F2D8E
:109A20000E94126222273327201B310BA1E0BFEFD7
:109A30000E94E7B52AE030E040E050E00E9483B5A4
:109A4000DA01C90181509F4FAF4FBF4FBC018F3F1B
:109A5000910509F02CF497FF05C060E070E002C0AA
:109A60006FEF70E08D816EC0033011050CF471C092
:109A700060E08C810E9412628A819B810E9449551C
:109A8000672B682B692B91F40E9412994F8158859E
:109A90006A01550FEE08FF08AB01BC014C0D5D1DBE
:109AA0006E1D7F1D8A819B810E946355FD808EEF14
:109AB0008F0D8C3020F084ED8F0D8330C8F42FEFA4
:109AC00030E0D8010E94EFB52AE030E040E050E0FD
:109AD0000E9483B5B9012F3F310509F02CF437FFFF
:109AE00005C060E070E002C06FEF70E08F2D2AC00B
:109AF0008C819EEF980F61E09C3018F08C5283307F
:109B000020F58F2D0E9412629801A1E0BFEF0E9404
:109B1000E7B52AE030E040E050E00E9483B5DA018A
:109B2000C90181509F4FAF4FBF4FBC018F3F91057F
:109B300009F02CF497FF05C060E070E002C06FEF01
:109B400070E08C810E947D6236C08F2D0E9412626F
:109B500032C063E377E085E89CE00E947EA360E08A
:109B60008C810E94126260E08D810E94126240E04E
:109B700050E0BA018A819B810E94635560E070E1E8
:109B80008A819B810E94491B60E070E28A819B81EF
:109B90000E94491B809127028F5F809327020BC090
:109BA000A12CB12CC114D104E104F10409F0E1CEDF
:109BB0000A191B09F7CE80E090E0DF91CF911F9149
:109BC0000F91FF90EF90DF90CF90BF90AF909F905C
:109BD0008F907F906F905F904F9008950F931F9399
:109BE000CF93DF93EC010A811B8160E070E0C80134
:109BF0000E941F1B18160CF083E08E8361E070E05A
:109C0000C8010E941F1B1816190614F08BE290E081
:109C10009D838C8362E070E0C8010E941F1B1816B0
:109C2000190614F088E590E098878F83DF91CF9133
:109C30001F910F91089508950F931F93CF93DF9372
:109C4000EC010A811B8160E070E0C8010E941F1BCB
:109C50009FEF980F953408F080E28C8361E070E00C
:109C6000C8010E941F1B9FEF980F953408F081E2F6
:109C70008D8362E070E0C8010E941F1B863410F4DF
:109C80008E8301C01E8263E070E0C8010E941F1B2A
:109C90009C01215031092115344018F49A87898795
:109CA00002C01A86198664E070E0C8010E941F1B7A
:109CB000813024E0920710F080E094E09C878B874D
:109CC00065E070E0C8010E941F1B1816190614F009
:109CD00080E197E298878F83DF91CF911F910F9159
:109CE0000895CF93DF93EC010E941C4E6AE377E066
:109CF00085E89CE00E947EA361E08C810E94416225
:109D000061E08D810E94416260E08C810E9412625C
:109D100060E08D810E94126260E08E810E9441624B
:109D200040E050E0BA018A819B810E94635560E067
:109D300070E18A819B810E94491B60E070E28A8108
:109D40009B810E94491B81E090E09093470A809399
:109D5000460A82E08093270281E090E0DF91CF9174
:109D6000089508950F931F93CF93DF938C010E9462
:109D7000EE4D65E477E085E89CE00E947EA380914B
:109D8000600A9091610A892B09F586E190E00E94B2
:109D9000D1AAEC01F801278130854681042E000C00
:109DA000550B648175810E940994D093610AC09318
:109DB000600A8E819F8197FD07C061E00E94416229
:109DC00060E08E810E94126281E0898381E090E0F0
:109DD0009093490A8093480ADF91CF911F910F9188
:109DE0000895EF92FF920F931F93CF93DF93EC01AF
:109DF0008A819B810E9469A5082F10E0C801880F05
:109E0000991F9C01235B3C4F79010430110574F4C8
:109E1000F701819191917F010E94E0A3BC018A81A9
:109E20009B810E94C3A30F5F1F4FEFCFEA80FB808F
:109E300060E0C7010E948AA2FC0111851A8761E0D7
:109E4000C7010E948AA29D838C8362E0C7010E94A1
:109E50008AA29F838E8364E0C7010E948AA29987A9
:109E600088871B3091F01C3001F11A3079F584E0BD
:109E700090E00E94D1AAFC01D383C28329EF32E093
:109E8000318320839C878B8721C089E090E00E94EA
:109E9000D1AA8C01FC01D383C28389EB92E0918328
:109EA0008083C8010E94EE4D0FC08DE090E00E94BB
:109EB000D1AA8C01FC01D383C28389ED92E0918306
:109EC0008083C8010E941C4E1C870B87DF91CF91B5
:109ED0001F910F91FF90EF9008958F929F92AF92F4
:109EE000BF92CF92DF92EF92FF920F931F93CF9387
:109EF000DF93CDB7DEB767970FB6F894DEBF0FBE1E
:109F0000CDBF8C017B0181EB92E0F80191838083CE
:109F10004801FDE08F0E911C9F8A8E8AF8011486FD
:109F200013861586108E178A672B09F448C0A090F7
:109F30004E0AB0904F0AA114B10409F440C06FE278
:109F400070E0C7010E9400BA6C01892B81F1D70132
:109F5000FE01319680E090E0BF012D91222341F077
:109F60002F3231F08431910519F021930196F5CF0C
:109F7000FB01E80FF91F1082C5010E944BA2F801F6
:109F800093838283B6016F5F7F4F4AE050E0C40144
:109F90000E9439BACE0146960E947018F801908F3F
:109FA000878B8E899F89892B69F415860BC0B70131
:109FB000C5010E944BA2F8019383828303C0F8017C
:109FC00013821282C8010E94C01A882319F0C801A6
:109FD0000E94F14E67960FB6F894DEBF0FBECDBF5C
:109FE000DF91CF911F910F91FF90EF90DF90CF9075
:109FF000BF90AF909F908F90089521EB32E0DC01ED
:10A0000011963C932E931B968D919C911C970097D3
:10A0100039F0DC01ED91FC910280F381E02D19947F
:10A0200008953F924F925F926F927F928F929F928C
:10A03000AF92BF92CF92DF92EF92FF920F931F9356
:10A04000CF93DF93CDB7DEB7C054D1090FB6F894E4
:10A05000DEBF0FBECDBF6115710509F41DC1342EE1
:10A060008B012C01FB018085853019F08630D9F0F9
:10A0700013C180914D0A8F5F80934D0AFB010681C9
:10A0800017810115110549F0432DB801C2010E9445
:10A090001150F80102811381F4CF80914D0A815053
:10A0A00080934D0AF9C065ED74E0C8010E944BA28F
:10A0B0007C0162E577E0C8010E944BA25C0167E584
:10A0C00077E0C8010E944BA24C016CE577E0C80123
:10A0D0000E944BA23C0161E677E0C8010E944BA2BE
:10A0E0006C016AED74E0C8010E944BA28C018114DE
:10A0F000910461F0332051F0F4018085843031F413
:10A10000A184B284C114D10491F415C0A114B10486
:10A1100039F0F5018085843019F4A184B28402C03D
:10A12000A12CB12CC114D10431F0332021F0F6015F
:10A130008085843039F06114710439F0F301808531
:10A14000843019F4C184D28402C0C12CD12CF20114
:10A15000938068E971E185E89CE00E94199B4AE0E0
:10A1600050E0692D85E89CE00E94AE9B64E971E1B6
:10A1700085E89CE00E94199B85E89CE00E94469C33
:10A18000E114F104F1F0F7016185728585E89CE046
:10A190000E944A9C6FE871E185E89CE00E94199B4F
:10A1A000B50185E89CE00E944A9C85E89CE00E94FD
:10A1B000469C0115110549F4A114B10409F04EC0E3
:10A1C00069C00115110509F465C0F8016185728542
:10A1D00085E89CE00E944A9C6AE871E185E89CE081
:10A1E0000E94199BB60185E89CE00E944A9C85E884
:10A1F0009CE00E94469CC114D10459F1F80180856D
:10A20000843039F56185728540E450E0CE010196D5
:10A210000E9439BA0E94D4918823D9F080914C0AC7
:10A22000811117C06FE270E0CE0101960E9400BA62
:10A23000892B51F4F8012185328543E050E060E438
:10A24000CE0101960E945E69B601CE0101960E9480
:10A250003AA2E114F10409F0AFCF1CC0F7018085E8
:10A260008430C1F461857285CE0101960E946D4FE4
:10A27000CE0101960E94C01A882341F020E030E010
:10A2800041E0B501CE0101960E94A618CE010196CB
:10A290000E94FD4F81E001C080E0C05CDF4F0FB63F
:10A2A000F894DEBF0FBECDBFDF91CF911F910F910C
:10A2B000FF90EF90DF90CF90BF90AF909F908F90E6
:10A2C0007F906F905F904F903F9008958F929F92F4
:10A2D000AF92BF92CF92DF92EF92FF920F931F93B4
:10A2E000CF93DF93CDB7DEB7DA950FB6F894DEBF24
:10A2F0000FBECDBFC82E8091F70D8983CA8221E0A1
:10A30000C216A0F074E07C1518F487E1C8120EC0E4
:10A310008091F80D9091F90D9B838C838091FA0DBB
:10A320009091FB0D9D838E8386E001C082E08E01BB
:10A330000F5F1F4F90E19C1528F0AFE0CA1630F474
:10A340009BEF01C09AEE9C0D923078F420917C0E28
:10A3500090917D0EF801E80FF11D908391E0980F28
:10A36000F801E90FF11D8E5F2083BFE0CB1641F1AC
:10A37000BC1558F0E5E0CE16A1F0F6E0CF12B6C05D
:10A380002091800E9091810E10C026E1C21609F432
:10A390008EC077E1C71609F459C090E1C912A6C072
:10A3A00055C020917E0E90917F0EF801E80FF11DAF
:10A3B000908391E0980FF801E90FF11D8E5F95C031
:10A3C00020917E0E30917F0EF801E80FF11D308351
:10A3D00042E0480F91E0980FF801E90FF11D20834A
:10A3E000B90167707727A3E036952795AA95E1F71D
:10A3F000672B19F091E0920F01C0922FB3E0B80FD4
:10A40000F801E40FF11D90838C5F60E070E0A0E044
:10A410004FEF480F9A1303C08B2F890F67C050E08E
:10A420009B0135952795400F511F220F331FF901CE
:10A43000E058F14FA0FD02C0208101C02181FA0146
:10A440002083AF5F6F5F7F4F8F5FE2CF20917E0EE3
:10A4500030917F0EF801E80FF11D308391E0980FE5
:10A46000F801E90FF11D208392E0980FF801E90F40
:10A47000F11D8D5F922F990F908390E03327E92F84
:10A48000F0E0E217F30794F5EE0FFF1FE058F14FED
:10A4900050814181F801E80FF11D408341E0480FF0
:10A4A000F801E40FF11D8E5F50839F5FE8CF90911C
:10A4B000800E2091810EF801E80FF11D208321E02C
:10A4C000280FF801E20FF11D90832091820E9091E8
:10A4D000830E32E0380FF801E30FF11D908393E013
:10A4E000980FF801E90FF11D8C5F20837801F801C6
:10A4F0002FEF3FEFD02E9E2F901B9817A0F4919135
:10A50000292748E050E0B9017695679520FF06C0FD
:10A510009B0191E0292790EA392701C09B01415016
:10A52000510989F7E8CFF801E80FF11D2083B2E067
:10A53000BB2EB80E8F5FF801E80FF11D3083F801D4
:10A54000EB0DF11D10828091F50D9091F60DDC015F
:10A55000ED91FC910284F385E02D1995019699F710
:10A56000E0910B0FF0910C0F309709F01995809145
:10A57000F50D9091F60D2E2D2D192B1558F4F70190
:10A5800061917F01DC01ED91FC910190F081E02D62
:10A590001995EDCFDC01ED91FC910680F781E02D5E
:10A5A0001995E0910D0FF0910E0F309709F0199564
:10A5B0000E9412994B015C01A8E0EA2EF12CD12CEB
:10A5C0008091F50D9091F60DDC01ED91FC910084E8
:10A5D000F185E02D1995892BC1F08091F50D9091B1
:10A5E000F60DDC01ED91FC910284F385E02D1995C7
:10A5F0009091F70D891711F0FF2099F1F801EF0DF7
:10A60000F11D8083EA94F39407C0E091090FF09163
:10A610000A0F309709F01995B5E0FB1222C0EA81C4
:10A620008E2F8F7790E08C159D0509F0A2C0E7FF73
:10A6300004C08B81882381F181C08E2F90E0FC01C2
:10A640003197E731F10568F48827EE5FFE4F8F4FB1
:10A650000C94D8B5F3E0EF2E04C0EB8002C0E5E027
:10A66000EE2E0E941299DC01CB0188199909AA09E2
:10A67000BB09813D9740A105B10538F480E0EE208B
:10A6800031F0882309F49CCF59C082EEF8CF8111B4
:10A6900055C0F4E0FF15C0F58FEF9FEF60E0EF2DA0
:10A6A000F0E09F0122503109462F50E0D8014217B7
:10A6B0005307BCF4A40FB51F4C91842748E050E029
:10A6C000DC01B695A79580FF06C0CD0171E0872714
:10A6D00070EA972701C0CD014150510989F76F5F9A
:10A6E000E3CFA20FB31F2C9130E0AC0155274217E6
:10A6F000530709F040C0892F9927EC0FFD1F2081D7
:10A7000030E082179307B9F58A818530B0F5833040
:10A71000B0F5813090F05B81652F70E0759567959D
:10A720002091080F40E0842F90E0861797070CF4E3
:10A7300052C02093080F50FD6CC080E01092020FB1
:10A740001092040F1092030F1092070FD3950FB6BB
:10A75000F894DEBF0FBECDBFDF91CF911F910F9157
:10A76000FF90EF90DF90CF90BF90AF909F908F9031
:10A77000089581EEE3CF83EEE1CF8731F1F66B816F
:10A7800070E0759567952091080F40E0842F90E068
:10A79000861797071CF02093080FCFCF4034C0F4E2
:10A7A0009C012E5F3F4F220F331F880F991FFC0122
:10A7B000EB50F24FDE01A20FB31F8C9190E0982F67
:10A7C0008827D801A20FB31F2C91822B90878783F3
:10A7D000242F4F5FDBCF4034C8F4880F991FFC0152
:10A7E000EB50F24FA5E0B0E0AC0FBD1FA80FB91FB2
:10A7F0002C9130E0322F2227A4E0B0E0AC0FBD1F37
:10A80000A80FB91F8C91282B30872783242F4F5FE7
:10A810008ACF403468F4880F991FFC01EB50F24F47
:10A82000DE01A80FB91F14968C9190E09087878362
:10A8300081E0840F8093080F80CFCF92DF92EF9258
:10A84000FF92CF93DF93EC016A017B01E889F989DC
:10A8500082E080834115514E61057105B1F060E0E1
:10A8600079E08DE390E0A70196010E9461B5DA01DD
:10A87000C9010197A109B109B695A7959795879543
:10A880009C01211580E13807A8F0E889F989108238
:10A8900060E874E88EE190E0A70196010E9461B53E
:10A8A000DA01C9010197A109B109B695A795979554
:10A8B00087959C01EC85FD853083EE85FF8520839F
:10A8C000188EEC89FD8986E08083EA89FB89808186
:10A8D00080618083EA89FB89808188608083EA893E
:10A8E000FB89808180688083EA89FB8980818F7DF4
:10A8F0008083DF91CF91FF90EF90DF90CF9008950C
:10A900004F925F926F927F928F929F92AF92BF927F
:10A91000EF92FF920F931F934B015C0129013A01C3
:10A920006E0D7F1D801F911F2FEF3FEF40E050E025
:10A930000E9461B5641575058605970570F4481485
:10A9400059046A047B0410F421E013C021E0861648
:10A950009706A806B90668F00BC086169706A806E3
:10A96000B90630F421E0481459046A047B0408F065
:10A9700020E0822F1F910F91FF90EF90BF90AF903A
:10A980009F908F907F906F905F904F9008950F935E
:10A990001F93CF93DF93082FEB01142F60913E0D8F
:10A9A00080913C0D90913D0D0E94706880913C0D0E
:10A9B00090913D0DDC01ED91FC910190F081E02D35
:10A9C000602F199580913C0D90913D0D0E94696812
:10A9D00081111EC0412F60913E0D80913C0D9091E0
:10A9E0003D0D0E949768CE01810F911D8C018091D1
:10A9F0003C0D90913D0DDC01ED91FC910084F185C1
:10AA0000E02D1995892B39F0C017D10739F403C00F
:10AA100082E090E010C080E090E00DC080913C0D9D
:10AA200090913D0DDC01ED91FC910284F385E02DC8
:10AA300019958993DCCFDF91CF911F910F910895E4
:10AA40000F931F93CF93DF93FC0183859485009729
:10AA5000C9F08B01EF01DC01ED91FC910484F585D7
:10AA6000E02D1995892B71F08B859C85DC01ED918A
:10AA7000FC910480F581E02DB801DF91CF911F9109
:10AA80000F91199484E690E0DF91CF911F910F917F
:10AA90000895FC0180859185009789F0FC0120854F
:10AAA000223041F0253059F460E00E948AA20097DC
:10AAB00031F0FC016185728583859485089560E09D
:10AAC00070E0CB010895CF92DF92EF92FF920F9347
:10AAD0001F93CF93DF93EC016A017B0188859985F1
:10AAE000892BE1F48A819B810E9469A5082F10E0DF
:10AAF0000530110564F480E090E00E94E0A3BC0101
:10AB00008A819B810E94C3A30F5F1F4FF1CF64E036
:10AB10008A819B810E948AA299878887E885F98526
:10AB200080858230F1F4C186D286E386F4866EE7B2
:10AB300071E185E89CE00E94199B2AE030E0B701B2
:10AB4000A60185E89CE00E94F79B85E89CE0DF91E8
:10AB5000CF911F910F91FF90EF90DF90CF900C94C9
:10AB6000469CDF91CF911F910F91FF90EF90DF9066
:10AB7000CF900895CF93DF93EC0181EB92E099831E
:10AB800088837B836A831C861B86CE010E94C01A41
:10AB9000882329F0CE01DF91CF910C94F14EDF9103
:10ABA000CF910895AF92BF92CF92DF92EF92FF9232
:10ABB0000F931F93CF93DF938C01EB0162E070E062
:10ABC0000E941F1B7C0197FF03C080E090E076C0CD
:10ABD00063E070E0C8010E941F1BAC011816190643
:10ABE00014F04FE350E081E0E816F10421F4CD2F9A
:10ABF000DD0FDD0B04C082E0E816F1040CF4DD2764
:10AC000024E630E0DE010E94EFB59A01550F440BB7
:10AC1000550B0E9483B569017A015901C8010E9450
:10AC2000FD1BC82FD0E0C8010E94051B0D2C000C95
:10AC3000EE08FF086C157D058E059F0549F4AB28CD
:10AC4000E9F1C230D10561F0C530D105B9F508C0D0
:10AC5000AB28E1F0C630D10539F0C130D10521F083
:10AC600061E0C8010E94D21BB701A601C8010E9481
:10AC7000CD1AC230D10511F0259729F460E071E0BA
:10AC8000C8010E94AF4260E072E00BC0C530D10540
:10AC9000A9F0229799F062E0C8010E94D21B60E0FF
:10ACA00071E0C801DF91CF911F910F91FF90EF905C
:10ACB000DF90CF90BF90AF900C94AF42DF91CF91D7
:10ACC0001F910F91FF90EF90DF90CF90BF90AF90CA
:10ACD0000895CF93DF93EC0160E073E00E94BB1B0B
:10ACE000009791F020914A0A30914B0A24303105A7
:10ACF00059F4BC01CE010E94AF4260E073E0CE0186
:10AD0000DF91CF910C94491BDF91CF9108958F92E1
:10AD10009F92AF92BF92EF92FF920F931F93CF93A8
:10AD2000DF938C017B0149015A010E9413A0EC01C1
:10AD3000892BF9F083E0888789869A86AB86BC8662
:10AD400088819981009711F00E9469ABC7010E9428
:10AD5000A0B999838883BE01C801DF91CF911F916B
:10AD60000F91FF90EF90BF90AF909F908F900C94B9
:10AD7000C3A3DF91CF911F910F91FF90EF90BF90F0
:10AD8000AF909F908F9008950F931F93CF93DF9371
:10AD9000EC012097F9F00A811B81888587FD06C0A8
:10ADA0008E819F81009711F00E94C456888584305F
:10ADB00031F489859A85009711F00E9469AB8881EA
:10ADC0009981009711F00E9469ABCE010E9469AB96
:10ADD000E801DFCFDF91CF911F910F9108952F925E
:10ADE0003F924F925F926F927F928F929F92AF921B
:10ADF000BF92CF92DF92EF92FF920F931F93CF9368
:10AE0000DF93CDB7DEB728970FB6F894DEBF0FBE3D
:10AE1000CDBF8C016B010E94D597019609F4D3C276
:10AE2000D801ED91FC910284F385E02DC8011995BC
:10AE30007C018F3FBFEF9B0709F4C5C2D801ED919C
:10AE4000FC910684F785E02D682FC8011995B2E2C0
:10AE5000EB16F10429F4B601C8010E945B9FB5C24C
:10AE6000EDE2EE16F10429F0C701C0970A9708F049
:10AE700044C1D801ED91FC910284F385E02DC80115
:10AE800019957C018F3FBFEF9B0709F49CC28D97FA
:10AE900089F4D801ED91FC910284F385E02DC8017D
:10AEA00019957C01019609F48EC2EFEFFFEFF88748
:10AEB000EF8304C021E030E038872F83C701C097BB
:10AEC000A12CB12C0A97C8F49AE0992E9A9CC00143
:10AED0009B9C900D1124B701605371095B01A80E72
:10AEE000B91ED801ED91FC910284F385E02DC801D3
:10AEF00019957C01C0970A9748F3BEE2EB16F1045E
:10AF0000D1F0C7018F7D85349105A9F0EF81F885D7
:10AF1000AE9EC001AF9E900DBE9E900D1124092ED5
:10AF2000000CAA0BBB0BF60181879287A387B4871D
:10AF300082E08087D8C0B501BB0C880B990B0E94BA
:10AF40001EB42B013C01FEE2EF16F104A1F5D8017D
:10AF5000ED91FC910284F385E02DC80119957C01E7
:10AF6000212C312C20E030E040E251E4C301B20159
:10AF70000E947DB44B015C01B70160537109072E3B
:10AF8000000C880B990B0E941EB4A50194010E942D
:10AF90000BB62B013C01B1E02B1A3108D801ED9121
:10AFA000FC910284F385E02DC80119957C01C097BE
:10AFB0000A97C0F202C0212C312CC7018F7D853445
:10AFC000910509F042C0D801ED91FC910284F3850E
:10AFD000E02DC80119957C018B32910559F4D801F7
:10AFE000ED91FC910284F385E02DC80119957C0157
:10AFF000B1E00CC08D9761F4D801ED91FC91028411
:10B00000F385E02DC80119957C01BFEFBE8302C016
:10B01000E1E0EE83A12CB12C8AE0982EC701C09705
:10B020008A309105B0F49A9C90019B9C300D1124BC
:10B030005C01A20EB31ED801ED91FC910284F38550
:10B04000E02DC80119957C01E9CFB1E0BE83A12CA8
:10B05000B12CEF81F885BF01FF0F880B990B0E947F
:10B060001EB4A30192010E947DB42B013C01B501E5
:10B07000BB0C880B990B0E941EB44B015C01FE8136
:10B080006F2FFF0F770B880B990B0E941EB49B014B
:10B09000AC01C501B4010E947DB44B015C01B1015A
:10B0A000330C880B990B0E941EB49B01AC01C501A7
:10B0B000B4010E940BB69B01AC0160E070E080E23D
:10B0C00091E40E9424B79B01AC01C301B2010E942C
:10B0D0007DB4D60119966D937D938D939C931C97A7
:10B0E00083E018968C93D801ED91FC910684F78546
:10B0F000E02D6E2DC801199522C0BBE5EB16F104B9
:10B1000009F060C0D801ED91FC910284F385E02D37
:10B11000C80119958B35910509F055C185E0F601F7
:10B120008087C8010E94D597D801ED91FC910284D7
:10B13000F385E02DC80119958D35910519F480E04E
:10B1400090E043C1D801ED91FC910684F785E02D94
:10B15000682FC8011995BB24BA940E9413A07C01E2
:10B16000009709F430C1BB2021F0F6019783868354
:10B1700008C0D40113969C938E931297FC0195827C
:10B180008482C8010E94D597B701C8010E94EF567A
:10B19000892B09F018C1C8010E94D597D801ED91FB
:10B1A000FC910284F385E02DC8011995B12C47016B
:10B1B0008C32910591F221E030E08D35910509F056
:10B1C00089C086C0BBE7EB16F10409F088C0D8013E
:10B1D000ED91FC910284F385E02DC80119958B3720
:10B1E000910509F0F0C086E0F6018087C8010E9451
:10B1F000D597D801ED91FC910284F385E02DC8012B
:10B2000019958D37910509F49ACFD801ED91FC91EC
:10B210000684F785E02D682FC801199599249A9422
:10B220000E9413A07C01009709F4CDC0992021F061
:10B23000F6019783868308C0D50113969C938E935D
:10B240001297FC01B582A482C8010E94D597B7016C
:10B25000C8010E945B9F019609F4B5C0C8010E9415
:10B26000D597D70119968D919C911A9711969C9319
:10B270008E931A961C921E921997D801ED91FC910B
:10B280000284F385E02DC8011995CA9709F09BC087
:10B29000C8010E94D597B701C8010E94EF560196D8
:10B2A00009F491C0C8010E94D597D801ED91FC9195
:10B2B0000284F385E02DC8011995912C57018C3239
:10B2C000910509F4ADCF21E030E08D37910511F4FF
:10B2D00020E030E088279927821B930B76C0BEE6DA
:10B2E000EB16F10411F519821A821B821C82D80117
:10B2F000ED91FC910484F585E02D44E050E0BE0121
:10B300006F5F7F4FC8011995049709F05CC044E056
:10B3100050E066E677E0CE0101960E942BBA0097D6
:10B3200009F051C0F601108650C0F6E6EF16F104A0
:10B3300021F59E012F5F3F4F790185E0D9011D92D4
:10B340008A95E9F7D801ED91FC910484F585E02D0B
:10B3500045E050E0B901C80119950597A1F545E010
:10B3600050E06BE677E0C7010E942BBA009759F5D1
:10B3700021E0F6012087118628C0F4E7EF16F104DA
:10B3800011F519821A821B821C82D801ED91FC9161
:10B390000484F585E02D44E050E0BE016F5F7F4FEF
:10B3A000C8011995049779F444E050E061E777E02B
:10B3B000CE0101960E942BBA009729F421E0F601F4
:10B3C0002087218702C08FEF9FEF28960FB6F89451
:10B3D000DEBF0FBECDBFDF91CF911F910F91FF90C8
:10B3E000EF90DF90CF90BF90AF909F908F907F9025
:10B3F0006F905F904F903F902F900895CF92DF9283
:10B40000EF92FF92CF93DF93EC010E9412996B01B0
:10B410007C018091580D9091590DDC01ED91FC91CA
:10B420000084F185E02D1995892B79F40E941299F9
:10B43000DC01CB018C199D09AE09BF0988399A43FB
:10B44000A105B10530F380E00DC08091580D9091B9
:10B45000590DDC01ED91FC910284F385E02D1995E5
:10B46000888381E0DF91CF91FF90EF90DF90CF90C4
:10B470000895DF92EF92FF920F931F93CF93DF9384
:10B48000CDB7DEB729970FB6F894DEBF0FBECDBF9C
:10B490008C017B01AE014F5F5F4F0E94B979D82EBE
:10B4A000882309F459C0F7018081803109F454C020
:10B4B0008FE78D83F801858196810E942A79B701F3
:10B4C000F801858196810E94E07840E06EE4F80101
:10B4D000858196810E94BE7840E06B81F80185816C
:10B4E00096810E94BE7840E06C81F801858196814A
:10B4F0000E94BE78F7018081803139F040E06D8193
:10B50000F801858196810E94BE78F8018581968137
:10B510000E942A79B701F801858196810E94E0781E
:10B52000F801408168E4858196810E94BE7864E1DB
:10B5300070E080E090E00E946563F80180818823DC
:10B5400031F06AE070E080E090E00E946563F8010D
:10B55000858196810E942A798D2D29960FB6F894BF
:10B56000DEBF0FBECDBFDF91CF911F910F91FF9036
:10B57000EF90DF900895EF92FF920F931F93CF9378
:10B58000DF93EC018C01085F1F4F7E01699170E031
:10B5900084E0759567958A95E1F740E150E085E88C
:10B5A0009CE00E943F9CF70160816F7070E040E179
:10B5B00050E085E89CE00E943F9CC017D10729F726
:10B5C000DF91CF911F910F91FF90EF9008950F930E
:10B5D0001F93CF93DF93009791F08C010E9413A0EB
:10B5E000EC01892B61F0C8010E94D597BE01C8010A
:10B5F0000E94EF56019631F4CE010E94C45680E0BD
:10B6000090E001C0CE01DF91CF911F910F9108957D
:10B61000CF93C82F462F61E070E00E94977C61E0D5
:10B6200070E08C2F0E946D7D8111F9CFCF9108952C
:10B6300020E5FC01208311820895FC01848584307B
:10B6400011F00C94FD7E80E008952F923F924F926E
:10B650005F926F927F928F929F92AF92BF92CF92A2
:10B66000DF92EF92FF920F931F93CF93DF9300D05F
:10B6700000D0CDB7DEB71C018AE59DE00E94FE59DF
:10B6800081113BC036C07801CE0101960E94FE595F
:10B69000882379F187010F5F1F4FE981D601ED9370
:10B6A0006D01AE2FAF77B0E0A50194010E94A2B565
:10B6B000460E571E681E791E47E0880C991CAA1C6E
:10B6C000BB1C4A95D1F7E7FF2BC005301105D9F611
:10B6D0008FEF9FEF9093F40D8093F30D8091580DB1
:10B6E0009091590DDC01ED91FC910488F589E02DD4
:10B6F000199560E070E0CB01B0C0F0915A0DFA836B
:10B7000019828BE5C82E8DE0D82EEE24E394F12C1F
:10B71000412C512C3201812C912C54018394B4CFB3
:10B72000BA81B07FBA838FEF800FF1018083B0338D
:10B7300021F5C801865A924F0E94FE598823C9F20A
:10B74000C701845A924F0E94FE59882391F20E5FDE
:10B750001F4FD101EC91F0E0EC5AF24FC780D12C91
:10B76000DC2CCC248085C80ED11C80915A0D81FF21
:10B7700008C0B2E0CB0ED11C04C080E0C12CD12C9B
:10B7800001C082E090E0A0E0B0E04801A12CB12C23
:10B790009C01AD01281939094A095B092B833C83B7
:10B7A0004D835E83E12CF12C8B819C81AD81BE8128
:10B7B000880D991DAA1DBB1D84159505A605B70505
:10B7C000D8F5CE0101960E94FE59882309F491CF45
:10B7D0008091F10D9091F20D0097F1F03A813033A4
:10B7E000D9F4D1012C914EEF5FEF6FEF7FEF421B49
:10B7F000510961097109480D591D6A1D7B1DC41647
:10B80000D506E606F70640F4DC01ED91FC910190C7
:10B81000F081E02D698119950038110538F4F8019F
:10B82000EC5AF24F898186830F5F1F4FBFEF8B1A4F
:10B830009B0AAB0ABB0AB8CF8091F10D9091F20D33
:10B84000892B41F4E1E88E169104A104B10410F0B3
:10B8500000E010E0B80180E090E026960FB6F89482
:10B86000DEBF0FBECDBFDF91CF911F910F91FF9033
:10B87000EF90DF90CF90BF90AF909F908F907F9090
:10B880006F905F904F903F902F9008952F923F922E
:10B890004F925F926F927F928F929F92AF92BF92E0
:10B8A000CF92DF92EF92FF920F931F93CF93DF938C
:10B8B00000D0CDB7DEB70E94D491382E882309F48A
:10B8C00028C10E9412994B015C018091E00D90917A
:10B8D000E10DA091E20DB091E30DA5019401281BAB
:10B8E000390B4A0B5B0BDA01C90189399A43A1056F
:10B8F000B105A8F48091DC0D9091DD0DA091DE0DD5
:10B90000B091DF0DA5019401281B390B4A0B5B0B8D
:10B91000DA01C90189399A43A105B105C8F120911D
:10B92000E40D8091580D9091590D222371F02CEF68
:10B930003FEF3093F40D2093F30DDC01ED91FC917A
:10B940000488F589E02D1995E3C020EC20935A0D69
:10B9500010925B0DDC01ED91FC910280F381E02DF2
:10B9600042E050E06AE57DE019958092DC0D90920E
:10B97000DD0DA092DE0DB092DF0D8092E00D909271
:10B98000E10DA092E20DB092E30D81E08093E40D11
:10B990008091580D9091590DDC01ED91FC9100843E
:10B9A000F185E02D1995892B09F4B3C0CE010196DC
:10B9B0000E94255B2B013C01672B09F4A5C08092F6
:10B9C000E00D9092E10DA092E20DB092E30D809116
:10B9D0005A0D807F803309F07BC08091E50D9091F6
:10B9E000E60D892B09F495C0E980F12CF701EC5A9A
:10B9F000F24F078110E0102F00278085080F111DDE
:10BA00009701245A324F6901B701635A724FA80156
:10BA1000C9010E94D0B9B8016E0D7F1DDB01AC5A7F
:10BA2000B24F18961C92189780915A0D8670282E46
:10BA3000E091E50DF091E60D32E083133CC01996DC
:10BA40008C91199790E0982F88271A962C91AC0129
:10BA5000420F511D5B834A834BEF5FEF4E195F0925
:10BA6000401B510B440D551D615A724FC60119956B
:10BA700080E480935A0D20925B0D5B8150935C0DA6
:10BA80008A8180935D0D8091580D9091590DDC0154
:10BA9000ED91FC910280F381E02D44E050E06AE5F5
:10BAA0007DE019958092DC0D9092DD0DA092DE0D67
:10BAB000B092DF0D2EC04DEF5FEF4E195F09401BB6
:10BAC000510B440D551D635A724FC601199521C083
:10BAD000803CA9F480ED80935A0D10925B0D80910B
:10BAE000580D9091590DDC01ED91FC910280F3818C
:10BAF000E02D42E050E06AE57DE019950AC0803D06
:10BB000041F41092E40D05C00E94D491811101C04E
:10BB1000312C832D0F900F900F90DF91CF911F91BB
:10BB20000F91FF90EF90DF90CF90BF90AF909F90DC
:10BB30008F907F906F905F904F903F902F900895DF
:10BB4000AF92BF92CF92DF92EF92FF921F93CF936B
:10BB5000DF9300D000D0CDB7DEB76C017C0110E0E0
:10BB60008AE0A82EB12C1330A9F0F701828190E071
:10BB7000A0E0B0E089839A83AB83BC83BE82AD82B0
:10BB8000BE016F5F7F4F85E89CE00E940A1C6FE951
:10BB900071E114C0F601858190E0A0E0B0E08983F6
:10BBA0009A83AB83BC83BE82AD82BE016F5F7F4F41
:10BBB00085E89CE00E940A1C6CE971E10E94199BD7
:10BBC0001F5FFFEFEF1AFF0A143069F626960FB6D3
:10BBD000F894DEBF0FBECDBFDF91CF911F91FF90D4
:10BBE000EF90DF90CF90BF90AF9008950F931F9389
:10BBF000CF93DF931F921F92CDB7DEB78C018CE8F5
:10BC000094E0F8019183808312821382148215825A
:10BC1000CE0101960E94185B89819A810E94037669
:10BC2000B8016E5F7F4F44E050E08FE090E00E94EB
:10BC300003A10E940276C8010F900F90DF91CF916F
:10BC40001F910F910895CF93DF93C4E5DDE080EE5F
:10BC50008E831F828C819D81DC01ED91FC9102809D
:10BC6000F381E02D42E050E06AE57DE019958FEF29
:10BC70009FEF9093F40D8093F30D8C819D81DC01F7
:10BC8000ED91FC910680F781E02D19958C819D81C5
:10BC9000DC01ED91FC910488F589E02D19950E9455
:10BCA00012996093DC0D7093DD0D8093DE0D9093FF
:10BCB000DF0D6093E00D7093E10D8093E20D9093A2
:10BCC000E30DDF91CF910895AF92BF92CF92DF92B3
:10BCD000EF92FF920F931F93CF93DF931F921F92C8
:10BCE000CDB7DEB77A836983BA01A901E981FA8108
:10BCF000F770082F10E0000F111F085A154FD801D8
:10BD00008D919C918E0F9F1F9F01240F351F213015
:10BD10003840A0F07A015B0160E078E06B01CE1A58
:10BD2000DF0AA601B5010E9403A1A7014C195D0914
:10BD3000B5016C0D7D1DF801808191810F900F90F0
:10BD4000DF91CF911F910F91FF90EF90DF90CF90F7
:10BD5000BF90AF900C9403A12F923F924F925F92AD
:10BD60006F927F928F929F92AF92BF92CF92DF920B
:10BD7000EF92FF920F931F93CF93DF93CDB7DEB770
:10BD80006D970FB6F894DEBF0FBECDBF5C017B8709
:10BD90006A875F8B4E8BD22EF32E1D8B0C8BED8E14
:10BDA000C88EC11066C0DB011196CC901197EC9043
:10BDB00012960C91129713961C911F772E2D30E03E
:10BDC000AFEFB0E00E94B5B524E6422E512C612CB5
:10BDD000712CA30192010E9483B5922E2C2D30E08C
:10BDE000AFEFB0E00E94B5B5A30192010E9483B508
:10BDF000822E9801AFEFBFEF0E94B5B52DE631E07E
:10BE000040E050E00E9483B5DA01C901492D682D58
:10BE10000E94FA92698F7A8F8B8F9C8F6AE072E111
:10BE200085E89CE00E94199B4AE050E0B80185E853
:10BE30009CE00E94A89B68E072E185E89CE00E947B
:10BE4000199B4AE050E06C2D85E89CE00E94AE9B77
:10BE500066E072E185E89CE00E94199B4AE050E0B0
:10BE60006E2D85E89CE00E94AE9B85E89CE00E94D8
:10BE7000469CF501848195810C891D890817190755
:10BE80002CF08C01015011091D8B0C8B6D2C7F2C1B
:10BE900077FE02C0612C712C8301000F111F000F6F
:10BEA000111F1B8B0A8BC301880F991F8C01060D74
:10BEB000171D198B088B0C891D89061517050CF4A5
:10BEC0006AC18090600A9090610A2E893F89213072
:10BED000310541F02230310509F02FC120E030E07A
:10BEE000A90147C1D40112968D919C9113976816B0
:10BEF000790608F01DC11E968C911E971B961C9109
:10BF00001B9719962D903C901A971896CC901897DD
:10BF1000A82EB12C811368C008891989020D131D40
:10BF20001C968C91CC2009F444C0D12CE12CF12C2E
:10BF3000F801E80FF11D608170E0762F6627072E6B
:10BF4000000C880B990BA70196010E9461B5222471
:10BF5000322E432E542EF801EA0DFB1D608170E055
:10BF6000762F6627072E000C880B990BA7019601E8
:10BF70000E9461B5D90199278827282A392A4A2A97
:10BF80005B2AF4018585F801E80FF11D608170E0FE
:10BF9000762F6627072E000C880B990BA7019601B8
:10BFA0000E9461B5D201C101822B932BA42BB52B2A
:10BFB000BBC0F801E80FF11D8081F801EA0DFB1DFF
:10BFC0002081422F50E060E070E0BA0155274427FD
:10BFD000582BD4011D968C91F801E80FF11D80813A
:10BFE0008A019B01082B9EC02A893B89220E331EA1
:10BFF000CC2009F475C0D12CE12CF12CF101EA0D13
:10C00000FB1D608170E0762F6627072E000C880BE1
:10C01000990BA70196010E9461B5B22FAA27992713
:10C0200088278C879D87AE87BF87F101E10FF11DBF
:10C03000608170E0762F6627072E000C880B990B25
:10C04000A70196010E9461B5D901992788270C851F
:10C050001D852E853F85082B192B2A2B3B2B0C8702
:10C060001D872E873F87D4011D968C91F101E80F23
:10C07000F11D608170E0762F6627072E000C880B7B
:10C08000990BA70196010E9461B58C859D85AE85AF
:10C09000BF85822B932BA42BB52B8C879D87AE87D6
:10C0A000BF87D4011C968C91F101E80FF11D6081CE
:10C0B00070E0762F6627072E000C880B990BA701DE
:10C0C00096010E9461B5B42FA32F922F88270C856B
:10C0D0001D852E853F85802B912BA22BB32B24C051
:10C0E000F101EA0DFB1D8081F101E10FF11D2081BD
:10C0F000422F50E060E070E0BA0155274427782BCA
:10C10000D4011D968C911D97F101E80FF11D8081DE
:10C11000482B1C968C91F101E80FF11D80818A015A
:10C120009B01182BD901C801892B8A2B8B2B29F550
:10C130002FEF3FEF4FEF50E01CC0188D1123A9F0F7
:10C14000AA85BB858C9111962C911197422F50E0B6
:10C1500060E070E0762F652F542F4427682B1296ED
:10C160008C919A01AB01282B04C0298D3A8D4B8DFF
:10C170005C8DB301C4010E949493BFEF6B1A7B0ADC
:10C180000A891B890C5F1F4F1B8B0A8B0889198931
:10C190000D5F1F4F8ECE1D8D112309F4B9C0009184
:10C1A000600A1091610AD80119968D919C911A9795
:10C1B000892B09F4A3C00E94ED98F801C784D088A8
:10C1C000E188F288DC01CB018C199D09AE09BF0919
:10C1D0008C329140A105B10570F3F894D801149602
:10C1E0008D919C9115979A8389831996ED91FC9175
:10C1F0001A977F01BFEFEB1AFB0A80818987F8014C
:10C2000090810388F489E02DD80155968C9199236B
:10C2100009F430C09081982B98879081809589236C
:10C220008F838F818C8388E08B8358856F814985CC
:10C230003B812C8189819A81D701508347FD252F2D
:10C240003A952083262F39F0441F00C000006083F8
:10C25000000000C0F2CF38E04D91608300000197EC
:10C2600061F7D8015496FC93EE93539749873B832B
:10C270002C833AC09081982B988790818095892350
:10C280008F838F818E8388E08D8358856F81498568
:10C290003D812E8189819A81D701508347FD252FC9
:10C2A00000C000C0208300C000C000C000C000C0AB
:10C2B00060830000262F3A9541F0441F000000C023
:10C2C00000C000C000C000C0E8CF38E04D9100C001
:10C2D000608300C0019709F7D8015496FC93EE9350
:10C2E000539749873D832E839A83898378940E944C
:10C2F000ED98F8016787708B818B928B61E072E11A
:10C3000085E89CE00E94199B85E89CE00E94469C81
:10C3100081E090E06D960FB6F894DEBF0FBECDBF02
:10C32000DF91CF911F910F91FF90EF90DF90CF9011
:10C33000BF90AF909F908F907F906F905F904F9045
:10C340003F902F900895FC01A089B1898C91A68916
:10C35000B78982FD0FC09C91818D8F5F8F73228D75
:10C36000821749F0218DDF01A20FB11D5D969C93CC
:10C37000818F08958C91089590E0FC013197E2310E
:10C38000F10508F04EC08827E75EFE4F8F4F0C94F2
:10C39000D8B5809180008F7703C0809180008F7D19
:10C3A00080938000089580918000877FF9CF84B5C5
:10C3B0008F7702C084B58F7D84BD08958091B000D1
:10C3C0008F7703C08091B0008F7D8093B000089577
:10C3D000809190008F7707C0809190008F7D03C07F
:10C3E00080919000877F8093900008958091A000B5
:10C3F0008F7707C08091A0008F7D03C08091A0003F
:10C40000877F8093A0000895809120018F7707C0D7
:10C41000809120018F7D03C080912001877F8093D0
:10C42000200108951F93CF93DF93282F30E0F90167
:10C43000E554FE4E8491F901E957FD4ED491F9017E
:10C44000E353FD4EC491CC23C1F0162F81110E94FD
:10C45000BC61EC2FF0E0EE0FFF1FEF55FE4EA591F3
:10C46000B4919FB7F894111104C08C91D095D82342
:10C4700002C0EC91DE2BDC939FBFDF91CF911F9127
:10C480000895CF93DF9390E0FC01E957FD4E24918E
:10C49000FC01E353FD4E8491882361F190E0880F05
:10C4A000991FFC01E359FD4EC591D491FC01EF5554
:10C4B000FE4EA591B491611109C09FB7F89488818F
:10C4C000209582238883EC912E230BC0623061F487
:10C4D0009FB7F8948881322F309583238883EC911D
:10C4E0002E2B2C939FBF06C08FB7F894E8812E2B7C
:10C4F00028838FBFDF91CF9108951F93CF93DF9350
:10C50000182FEB0161E00E944162209711F460E076
:10C5100004C0CF3FD10539F461E0812FDF91CF9185
:10C520001F910C941262E12FF0E0E554FE4EE4916D
:10C530008E2F90E0FC013197E231F10508F09DC0AB
:10C540008827E55DFE4F8F4F0C94D8B584B5806881
:10C5500084BDC7BD97C084B5806284BDC8BD92C08C
:10C5600080918000806880938000D0938900C09380
:10C57000880088C080918000806280938000D09382
:10C580008B00C0938A007EC0809180008860809379
:10C590008000D0938D00C0938C0074C08091B00057
:10C5A00080688093B000C093B3006CC08091B000ED
:10C5B00080628093B000C093B40064C0809190000A
:10C5C000806880939000D0939900C09398005AC0DF
:10C5D00080919000806280939000D0939B00C093E4
:10C5E0009A0050C080919000886080939000D09312
:10C5F0009D00C0939C0046C08091A00080688093FD
:10C60000A0008091A0008F7B8093A000D093A90010
:10C61000C093A80037C08091A00080628093A000E2
:10C62000D093AB00C093AA002DC08091A000886079
:10C630008093A000D093AD00C093AC0023C0809144
:10C640002001806880932001D0932901C0932801A4
:10C6500019C080912001806280932001D0932B012A
:10C66000C0932A010FC0809120018860809320012F
:10C67000D0932D01C0932C0105C0C038D1050CF01A
:10C680004BCF45CFDF91CF911F910895863308F0AE
:10C69000865390917B00282F2870977F922B909340
:10C6A0007B008770806480937C0080917A00806436
:10C6B00080937A0080917A0086FDFCCF809178008B
:10C6C0002091790090E0922B08958F929F92AF92E3
:10C6D000BF92CF92DF92EF92FF926B017C010E949A
:10C6E000ED984B015C01C114D104E104F104F1F0B7
:10C6F0000E94ED98DC01CB0188199909AA09BB09B0
:10C70000883E9340A105B10570F321E0C21AD1081B
:10C71000E108F10888EE880E83E0981EA11CB11C88
:10C72000C114D104E104F10419F7DDCFFF90EF90BB
:10C73000DF90CF90BF90AF909F908F9008954F92D1
:10C740005F926F927F928F929F92AF92BF92CF92A1
:10C75000DF92EF92FF920F931F93CF93DF93CDB7AA
:10C76000DEB763970FB6F894DEBF0FBECDBF7C0176
:10C770005B013A01FB0120E080E090E06AE031914A
:10C78000332309F140ED430F4A3080F4689FA00144
:10C79000699F500D1124CA01C097830F911D37FD69
:10C7A0009A958F3F910559F350F313C03E3289F4A7
:10C7B000233079F0D301A20FB11D12968C932F5F15
:10C7C00080E090E0DCCF233021F4F301858381E029
:10C7D00021C0F70142815381648175818091240DCC
:10C7E0009091250DA091260DB091270D481759075E
:10C7F0006A077B0709F499C10E9412998701085FB3
:10C800001F4F6F7077277C5FC8010E941C7F8130AB
:10C8100019F080E090E0FCC18CE894E09A83898371
:10C82000F70182819381A481B5818B839C83AD8341
:10C83000BE8345E350E0BE016F5F7F4FC8010E9499
:10C840001C80892B19F4C12CD12C6AC10E94129929
:10C85000F701778366837627672776277A8369834C
:10C8600042E050E0BE016F5F7F4FC8010E94717BC4
:10C8700081E090E09E878D8742E050E0BE01635FDB
:10C880007F4FC8010E94717B80E091E09E878D8779
:10C8900042E050E0BE01635F7F4FC8010E94717BA0
:10C8A0001E861D8642E050E0BE01635F7F4FC801D7
:10C8B0000E94717B42E050E0BE01635F7F4FC80180
:10C8C0000E94717B42E050E0BE01635F7F4FC80170
:10C8D0000E94717B4501F5018081882301F164018B
:10C8E0005601F60181912F01882321F08E3211F03B
:10C8F0006201F6CFC818D9081C141D0474F4CF8641
:10C9000041E050E0BE01615F7F4FC8010E94717B32
:10C91000A601B401C8010E94717B4201DCCF1F86D1
:10C9200041E050E0BE01615F7F4FC8010E94717B12
:10C93000C12CDD24D394DE86CD8642E050E0BE01DA
:10C94000635F7F4FC8010E94717BDE86CD8642E027
:10C9500050E0BE01635F7F4FC8010E94717BC80138
:10C960000E94497F892B09F46ECFE3E0AE2EB12CF3
:10C97000230122E0420E511C0E9412993B014C01FE
:10C98000C8010E94A37E18161906B4F00E941299DD
:10C99000DC01CB0186199709A809B909813A9F40A2
:10C9A000A105B105E0F40E948B8261E070E080E0B7
:10C9B00090E00E946563E4CFF70142815381648176
:10C9C0007581808D918DA28DB38D481759076A07A7
:10C9D0007B0749F4848D958DC59729F409C0CC2433
:10C9E000CA94DC2C92C05EEFC52EDD24DA948DC093
:10C9F000F70181A192A10C970CF49FC04CE050E08C
:10CA0000BE016F5F7F4FC8010E945B7E8B819C815E
:10CA10009827892798279A8B898B29813A813227F1
:10CA200023273227F701468157812417350709F05C
:10CA30007FC097FF7DC08F709270892B09F0E3C093
:10CA40006F8078847624672476246114710409F455
:10CA5000D5C0C12CD12C8D819E81982789279827FC
:10CA6000C816D90608F46EC0812C912C41E050E024
:10CA7000BE016D5E7F4FC8010E945B7E8B89982F3F
:10CA8000907C09F091C0811185C042E050E0BE0168
:10CA9000615F7F4FC8010E945B7E42E050E0BE01B3
:10CAA000635F7F4FC8010E945B7EC8010E947A7E4F
:10CAB000C8010E947A7EC8010E947A7EC8010E9445
:10CAC0007A7E42E050E0BE016F5E7F4FC8010E9457
:10CAD0005B7E8F8598898115914009F06DC0CD846A
:10CAE000DE84DC24CD24DC2481E0C816D10409F0E6
:10CAF00063C089899A898115944009F07AC044E01D
:10CB000050E0B201C8010E945B7E0E948B8281E0EE
:10CB1000A81AB10829F0FFEFCF16DF0609F42CCFD1
:10CB2000C8010E94107DC60173C08EEF9FEF70C0D8
:10CB30004CEFC42EDD24DA94E8CF9DEFC92EDD241E
:10CB4000DA94E3CF41E050E0BE01635F7F4FC8015C
:10CB50000E945B7E8D85882351F08D859FEF980F15
:10CB60009D87882321F0C8010E947A7EF6CF8D85AB
:10CB70008111E8CFC8010E947A7EC8010E947A7EA6
:10CB8000C8010E947A7EC8010E947A7EFFEFCF1A08
:10CB9000DF0A61CF8B899FEF980F9B8B882341F031
:10CBA000C8010E947A7EF6CFC8010E947A7E1B8A55
:10CBB0008B8981115BCF69CFC12CD12C89899A894E
:10CBC000982789279827C816D90638F4C8010E94E3
:10CBD0007A7EFFEFCF1ADF0AF1CF2FEF821A920A87
:10CBE0006814790409F042CF26EFC22EDD24DA94CE
:10CBF0008CCF77EFC72EDD24DA9487CF3AEFC32EA0
:10CC0000DD24DA9482CF8BEFC82EDD24DA947DCF39
:10CC100063960FB6F894DEBF0FBECDBFDF91CF9104
:10CC20001F910F91FF90EF90DF90CF90BF90AF904A
:10CC30009F908F907F906F905F904F90089585EDBB
:10CC40008093BC008091BC0084FDFCCF1092251124
:10CC500008954091D80A262F30E0240F311D21324B
:10CC60003105DCF4209125112430C9F4FC0180E069
:10CC700090E0861758F43091D80A2191DC01A8542D
:10CC8000B54FA30FB11D2C930196F3CF8091D80A15
:10CC9000680F6093D80A80E0089581E0089582E0EB
:10CCA000089508950895E091291180912811E817B9
:10CCB00030F4F0E0E856F54F808190E008958FEF72
:10CCC0009FEF08959091291180912811981750F4A1
:10CCD000E92FF0E0E856F54F208130E09F5F909318
:10CCE000291102C02FEF3FEFC9010895809128114B
:10CCF00090E020912911821B91090895CF92DF9233
:10CD0000EF92FF920F931F93CF93DF937C01CB01A0
:10CD10008A012091970A222389F0EB016B01C40E4E
:10CD2000D51ECC15DD0569F06991D701ED91FC9117
:10CD30000190F081E02DC7011995F3CF642F0E9477
:10CD40002966C801DF91CF911F910F91FF90EF905D
:10CD5000DF90CF900895CF93DF931F92CDB7DEB7CA
:10CD600069832091970A2223D1F020912611203245
:10CD700040F021E030E0FC013383228380E090E04A
:10CD800015C080912711E82FF0E0E958F54F9981FF
:10CD900090838F5F809327118093261105C061E0F7
:10CDA000CE0101960E94296681E090E00F90DF910C
:10CDB000CF9108950C9469AB1F920F920FB60F920A
:10CDC00011240BB60F922F933F934F935F936F9362
:10CDD0007F938F939F93AF93BF93EF93FF93809134
:10CDE000B900887F803609F49CC068F5883209F460
:10CDF0005BC090F4803109F454C038F4882309F4FE
:10CE0000F6C0883009F44DC0F6C0883109F44CC032
:10CE1000803209F45DC0EFC0803409F468C048F482
:10CE2000803309F455C0883309F0E5C08093FB0ACC
:10CE3000D8C0803509F44FC0883509F45DC0883406
:10CE400009F0D9C0D6C0883909F4C7C0A8F488371A
:10CE500009F467C038F4883609F463C0803709F4F0
:10CE600060C0C9C0883809F4B8C0803909F45FC00F
:10CE7000803809F0C0C05BC0803B09F486C038F43C
:10CE8000803A09F466C0883A09F47FC0B4C0803C97
:10CE900009F4A7C0883C09F4A4C0883B09F48AC0FF
:10CEA000AAC080911E0B10C090911D0B80911C0B8D
:10CEB000981770F5E0911D0B81E08E0F80931D0B8C
:10CEC000F0E0E450F54F80818093BB0085EC86C094
:10CED0008093FB0A8EC0E0911D0B81E08E0F809342
:10CEE0001D0B8091BB00F0E0E450F54F80839091E2
:10CEF0001D0B80911C0B6EC0E0911D0B81E08E0F0D
:10CF000080931D0B8091BB00F0E0E450F54F8083CF
:10CF10008091241181116DC081E08093231184EAF6
:10CF200061C083E0809325111092FA0ACFCF8091DF
:10CF3000FA0A803208F051C0E091FA0A81E08E0FBF
:10CF40008093FA0A8091BB00F0E0E652F54F8083AF
:10CF5000BDCF85EC8093BC00109225118091FA0A18
:10CF6000803230F4E091FA0AF0E0E652F54F108298
:10CF70006091FA0A70E0E0911F11F09120118AEDA2
:10CF80009AE019951092FA0A36C084E08093251130
:10CF90001092D90A1092D80AE0912111F091221131
:10CFA00019958091D80A811105C081E08093D80A33
:10CFB0001092B80AE091D90A81E08E0F8093D90AC5
:10CFC000F0E0E854F54F80818093BB009091D90A3E
:10CFD0008091D80A981708F479CF85E88093BC002F
:10CFE0000AC085EC8093BC001092251104C01092F9
:10CFF000FB0A0E941F66FF91EF91BF91AF919F9135
:10D000008F917F916F915F914F913F912F910F90F1
:10D010000BBE0F900FBE0F901F90189530912611E8
:10D02000313208F04AC0809125118111FCCF9091D6
:10D03000760A22E020932511609324112FEF20938C
:10D04000FB0A10921D0B30931C0BE7E7FAE0ACEFE4
:10D05000BAE020E0321721F041914D932F5FFACFD3
:10D0600010921E0B20911E0B990F922B90931E0B6A
:10D0700090912311913061F41092231190911E0B25
:10D080009093BB009091BC0093FDF8CF95EC01C04C
:10D0900095EE9093BC00909125119230E1F3909120
:10D0A000FB0A9F3F79F08091FB0A803241F080912A
:10D0B000FB0A803331F084E005C081E003C082E0E8
:10D0C00001C083E010922711109226111092970A46
:10D0D000089561E00C940E6880E39DE00C9469680B
:10D0E00081E08093970A6093760A1092271110923C
:10D0F00026110895FC01618180E39DE00C94706825
:10D100001F93CF93DF93EC01162F0E947A6861EE94
:10D1100080E39DE00E94AB66612F80E39DE00E946A
:10D12000AB66CE01DF91CF911F910C946C6880911A
:10D1300025118111FCCF413208F040E281E080935B
:10D140002511809324119FEF9093FB0A10921D0BE1
:10D15000940F90931C0B80931E0B80911E0B660FF7
:10D16000682B60931E0B80912311813061F4109223
:10D17000231180911E0B8093BB008091BC0083FD26
:10D18000F8CF85EC01C085EE8093BC00809125111D
:10D190008130E1F380911D0B841710F440911D0B39
:10D1A000ECEFFAE0A8E9BAE080E0841721F0919171
:10D1B0009D938F5FFACF10922911809328110895C3
:10D1C00041E0FC01618180E39DE00E94976880E37B
:10D1D0009DE00E9462660895CF93DF93EC0163ECBB
:10D1E0000E948068CE01DF91CF910C94E068CF93CC
:10D1F000DF93EC010E94EC68682F6460CE01DF9140
:10D20000CF910C94FF788F929F92AF92BF92CF9262
:10D21000DF92EF92FF920F931F93CF93DF93CDB7DF
:10D22000DEB72B970FB6F894DEBF0FBECDBF8C01D3
:10D23000CE0101967C016C018AE0882E912CA12CF4
:10D24000B12CC6018E199F09411551056105710563
:10D2500081F0CB01BA01A50194010E9461B5942F20
:10D26000852F605DF60161936F01A901692F782F09
:10D27000E8CFFC013197EE0DFF1DD8019E01215032
:10D28000310940814D933197E217F307D1F7F80147
:10D29000E80FF91F10822B960FB6F894DEBF0FBE71
:10D2A000CDBFDF91CF911F910F91FF90EF90DF9055
:10D2B000CF90BF90AF909F908F9008958F929F9244
:10D2C000AF92BF92CF92DF92EF92FF920F931F9394
:10D2D000CF93DF938C014A015901E0906E0AF090E0
:10D2E0006F0AC62F660FDD0BE114F10461F1F7013F
:10D2F0008085863041F566E777E0C7010E944BA242
:10D300006C01F2E08F16910439F083E088169104E5
:10D3100051F46EE877E002C06BE777E0C7010E9446
:10D320004BA27C0102C0E12CF12CC114D10469F0A4
:10D33000F6018085843049F461857285AE01C801AB
:10D340000E9439BA08C0E12CF12CAE0166E672E108
:10D35000C8010E94E9ACAE016BE775E0C8010E940C
:10D360001BBAE114F10439F0F7018085843019F417
:10D37000618572850FC0F2E08F169104A1F083E001
:10D380008816910461F08A94892899F460916C0A56
:10D3900070916D0AAE01C8010E941BBA0AC0AE01AD
:10D3A00060E672E103C0AE016DE572E1C8010E9462
:10D3B000CBACAE016BE775E0C8010E941BBAA114AB
:10D3C000B10429F0AE01B501C8010E941BBAC80121
:10D3D000DF91CF911F910F91FF90EF90DF90CF9051
:10D3E000BF90AF909F908F900895CF92DF92EF9271
:10D3F000FF920F931F93CF93DF936B017C01EA01A0
:10D400000E94E9B68B011F936F938CE097E09F9386
:10D410008F93DF93CF930E9490BA0F900F900F904D
:10D420000F900F900F9020E030E0A901C701B601E6
:10D430000E941FB7181624F0F7FAF094F7F8F0944A
:10D4400009900020E9F721978EE28883B80117FF41
:10D4500003C0719561957109072E000C880B990B1B
:10D460000E941EB49B01AC01C701B6010E940AB61E
:10D4700020E030E040E251E40E947DB40E94E9B631
:10D48000605D69831A82DF91CF911F910F91FF90A8
:10D49000EF90DF90CF900895CF93DF931F921F926C
:10D4A000CDB7DEB780912D1190912E11009711F418
:10D4B00087E391E1BE016F5F7F4F681B790B072EF9
:10D4C000000C880B990B0F900F90DF91CF9108956E
:10D4D0009FE9980F963010F4875508959FEB980FA9
:10D4E000963010F48753089580538A3008F080E016
:10D4F0000895CF93DF93DA01382FEC018C2F831B33
:10D500008617C8F4CE01E991F0E024E0F595E7959F
:10D510002A95E1F7E55AFC4F20812C93FC0180818C
:10D52000E82FEF70F0E0E55AFC4F808111968C9364
:10D5300011971296E3CFFA01E60FF11DE60FF11DE8
:10D540001082DF91CF9108952F923F924F925F9278
:10D550006F927F928F929F92AF92BF92CF92DF9203
:10D56000EF92FF920F931F93CF93DF93CDB7DEB768
:10D570002D970FB6F894DEBF0FBECDBF0E94129953
:10D580000091720A1091730A2091740A3091750A01
:10D59000601771078207930708F490C20E941299DE
:10D5A0004B015C0180916A0A90916B0A009709F423
:10D5B000E7C1E091F30FF091F40F2281223059F48A
:10D5C00063E472E185E89CE00E94199B85E89CE099
:10D5D0000E94469CD5C12091700A3091710A6091D9
:10D5E000680A7091690A261737070CF4B3C00E94C5
:10D5F00012992B013C0128E8420E23E1521E611CC6
:10D60000711C69E372E185E89CE00E9478A2E091D8
:10D61000F30FF091F40F309751F08FEF838714865A
:10D62000DF0113963B961D92AE17BF07E1F7E0911D
:10D63000620AF091630A80E090E02091680A3091DC
:10D64000690A821793070CF07DC0208131812E7FFB
:10D65000219331930196F1CF6091680A7091690A24
:10D6600033E0660F771F3A95E1F72091660A309113
:10D67000670A620F731F0E94FA7918160CF002C233
:10D68000E090680AF090690A34E1E316F1040CF0C6
:10D69000F9C10E941299641575058605970508F071
:10D6A000F1C1C090660AD090670A170183E0220C8E
:10D6B000331C8A95E1F72C0C3D1C67E0C1010E94E8
:10D6C0006D78D10117969C9189133CC000E010E061
:10D6D0000E151F050CF06AC148E050E0B101C6010B
:10D6E0000E94BAB948E0C40ED11C892B09F05BC175
:10D6F000000F111FE091620AF091630AE00FF11F21
:10D700008081918181609183808362E372E185E809
:10D710009CE00E94199B8091680A9091690A23E01D
:10D72000880F991F2A95E1F72091660A3091670AC0
:10D73000820F931F0E94BB5A6BE272E185E89CE066
:10D740000E9478A28091F30F9091F40F009709F056
:10D7500083CF98C10091660A1091670AA901E3E09E
:10D76000440F551FEA95E1F7040F151FF80140819A
:10D77000483209F0FAC0AE014F5F5F4FB8010E9416
:10D78000B979882369F12A8130E0C901982F882767
:10D79000990F990F990F6981F8E06F9FB0011124DB
:10D7A0009C01262B372BD8018C918031E1F46885C0
:10D7B00070E08F81FB01E81BF109CF019695982F4E
:10D7C0008827979587950E94C4B560517109207F7D
:10D7D00013E0220F331F1A95E1F7620F731F04C085
:10D7E00060E874EE01C0B9016138F4EE7F077CF0A7
:10D7F000072E000C880B990B0E941EB420E030E02D
:10D8000040E05CE30E947DB49B01AC0104C020E0D9
:10D8100030E04EEF52ECE091640AF091650A3097E7
:10D8200089F08091700A9091710ABC01A3E0660FA3
:10D83000771FAA95E1F7A091660AB091670A6A0F6F
:10D840007B1F19950091700A1091710A43E0000F37
:10D85000111F4A95E1F78091660A9091670A080FB7
:10D86000191FE0906A0AF0906B0AD8018C91803100
:10D8700049F0B801C7010E94CC79D82E882309F459
:10D8800068C002C03CE0D32EF701858196810E94DA
:10D890002A79882309F45DC0B801D70115968D91C6
:10D8A0009C9116970E94E078F701408164E485819D
:10D8B00096810E94BE78D70112968C91882309F434
:10D8C00048C0E7EFED0DE33040F4F0E0EE0FFF1F4E
:10D8D000EB5AFC4FC080D18004C09EEEC92E92E06E
:10D8E000D92E0115110579F1F7018381882359F1AA
:10D8F0008081811128C00E9412992B013C01960160
:10D90000DD0C440B550B2A873B874C875D87AE01A6
:10D910004F5F5F4FB801C7010E9463798981811110
:10D9200018C00E941299DC01CB012A853B854C85E9
:10D930005D85821B930BA40BB50B84159505A6057D
:10D94000B70528F306C0B601DD0C880B990B0E94C1
:10D9500065638091700A9091710A01969093710AA3
:10D960008093700A64EC79E00DC02F5F3F4F3093D5
:10D97000710A2093700A80ED97E00E94C4B502C03E
:10D9800060EA76E8CB01770FAA0BBB0B880E991ED5
:10D99000AA1EBB1E8092720A9092730AA092740A09
:10D9A000B092750A8BC00F5F1F4F92CE80916A0AAA
:10D9B00090916B0A892B09F4C5CEE091680AF09129
:10D9C000690AEE0FFF1F8091620A9091630AE80FC7
:10D9D000F91F81E090E0918380830091680A1091A3
:10D9E000690A66E272E185E89CE00E94199B4AE0C0
:10D9F00050E0B80185E89CE00E943F9C6FE172E135
:10DA000085E89CE00E94199B8091680A9091690AC0
:10DA1000B3E0880F991FBA95E1F72091660A30911B
:10DA2000670A820F931F0E94BB5A85E89CE00E9400
:10DA3000469C6091680A7091690A13E0660F771F2F
:10DA40001A95E1F78091660A9091670A680F791F2D
:10DA5000DB018C91883261F480916A0A90916B0AA3
:10DA60000E94395A8091F30F9091F40F0E94F76849
:10DA70008091680A9091690A01969093690A80934F
:10DA8000680A60CE0091680A1091690A60E172E14B
:10DA900085E89CE00E94199B4AE050E0B80185E8C7
:10DAA0009CE00E943F9C85E89CE00E94469C10926E
:10DAB000710A1092700A60E47FE164CF2D960FB670
:10DAC000F894DEBF0FBECDBFDF91CF911F910F91B4
:10DAD000FF90EF90DF90CF90BF90AF909F908F908E
:10DAE0007F906F905F904F903F902F900895089592
:10DAF00020E3FC0120833296862F82958F7090E17F
:10DB0000899F601911246A3014F4605D01C0695C5A
:10DB10006293682F8111F0CF08957F928F929F9228
:10DB2000AF92BF92CF92DF92EF92FF920F931F932B
:10DB3000CF93DF93CDB7DEB7A6970FB6F894DEBFCD
:10DB40000FBECDBF8C01762E942E852E20E2B22EF4
:10DB5000CE0101967C01FC012B2D11922A95E9F74B
:10DB60008CE894E09AA389A38FEF8BA38CA38DA359
:10DB70008EA3680183E4C80ED11C43E450E0BE01CB
:10DB80006F5D7F4FC6010E941C80019609F4B9C0E9
:10DB900081E089838A8386E0A82EAB821C82F8010B
:10DBA00064817581868197810E94E0B56D837E8353
:10DBB0008F83988789869A8680E890E09C878B87F8
:10DBC0004CE150E0B701C6010E94717BF7012B2D9B
:10DBD00011922A95E9F7480188E0880E911CF4011A
:10DBE000D70101900D92AA94E1F740E150E0B7010E
:10DBF000C6010E94717BF7011192BA94E9F796E091
:10DC0000A92EB12C40E250E0B701C6010E94717B01
:10DC1000F1E0AF1AB108B1F783E6898392E89A83FD
:10DC200093E59B838C8385E38D8381E08E837F8264
:10DC30009DE3988797E099878A8786E0F401DE0163
:10DC40001B9601900D928A95E1F78CE0898B8A8B67
:10DC500060E877E0CE0143960E9414BAF80163852C
:10DC6000CE0149960E94786DF8016485CE014B96ED
:10DC70000E94786DF8016585CE014D960E94786D01
:10DC80004EE150E0B701C6010E94717BF3E07F12C4
:10DC90001EC082E3898384E08A83F80196859B8392
:10DCA00097859C8390899D8391899E8396E39F832A
:10DCB0008887828D8987838D8A87848D8B87858DE0
:10DCC0008C874CE050E0B701C6010E94717B87E36E
:10DCD000898386E08A8391E09B8393E09C838D8394
:10DCE0008FE08E838AE38F838BE388878FEF89872A
:10DCF00049E050E0B701C6010E94717BC6010E9455
:10DD0000497FA6960FB6F894DEBF0FBECDBFDF9158
:10DD1000CF911F910F91FF90EF90DF90CF90BF9028
:10DD2000AF909F908F907F9008959F92AF92BF92F7
:10DD3000CF92DF92EF92FF920F931F93CF93DF93D7
:10DD4000982E8B015A01690164E270E00E946D7D9A
:10DD5000E82EF12C65E270E0892D0E946D7DFE2C8D
:10DD6000EE24E82AE801CE0DDF1D9E013770E92C74
:10DD7000F12CC701880F991FAC01405B554F7A0108
:10DD8000FA0180819181820F931FA9014C0D5D1DC5
:10DD90004130584090F000E018E0021B130BA8013E
:10DDA000B5010E9433A1A601401B510BB501600FC4
:10DDB000711FF7018081918102C0A601B5010E9407
:10DDC00033A1CC0DDD1D4D2F64E270E0892D0E9442
:10DDD000977C4C2F65E270E0892DDF91CF911F91E8
:10DDE0000F91FF90EF90DF90CF90BF90AF909F90FA
:10DDF0000C94977CFF920F931F93CF93DF93F82E91
:10DE000000E010E08F2D0E9495A1EC01892B21F0FC
:10DE10008F2D0E9495A18C01C017D10799F7CE01D3
:10DE2000DF91CF911F910F91FF900895CF93DF93D2
:10DE3000FC0101900020E9F79F01281B390B285FA6
:10DE40003F4F2138310570F5EC010E94D4918823B1
:10DE500049F18091DA0D9091DB0D019611F481E08A
:10DE600090E09093DB0D8093DA0D8091DA0D909124
:10DE7000DB0D90935F0D8093600D47E050E06AE505
:10DE80007DE0CE010E944B91FC01EC5AF24F1682CC
:10DE9000AC01445051096AE57DE082E8DF91CF9101
:10DEA0000C946B9180E0DF91CF9108951F93CF93F5
:10DEB000DF931F921F92CDB7DEB76CE271E080E076
:10DEC00090E00E9465631FB7F8948091250B811143
:10DED00027C0E2E0F3E18491ECEBF2E19491E82FCA
:10DEE000F0E0EE0FFF1FE359FD4EA591B491EC91C8
:10DEF000E92321F461E085E30E94126261E085E399
:10DF00000E9441628CB580618CBD8CB580648CBDF3
:10DF100061E084E30E94416261E083E30E94416228
:10DF20008091250B8F5F8093250B1FBF249ACE0114
:10DF300001960E94185B89819A810E94037667E0AE
:10DF400080E090E00E9462A165E58BE190E00E9494
:10DF500062A165E58AE190E00E9462A10E940276DA
:10DF600080E090E49093510A8093500A80E090E61C
:10DF70009093590A8093580A80E098E49093530A4A
:10DF80008093520A80E098E690935B0A80935A0A45
:10DF900080E090E59093550A8093540A80E090E7E2
:10DFA00090935D0A80935C0A80E098E59093570A0D
:10DFB0008093560A80E098E790935F0A80935E0A08
:10DFC0000F900F90DF91CF911F910895AF92BF9264
:10DFD000CF92DF92EF92FF920F931F93CF93DF9335
:10DFE0001F921F92CDB7DEB75C018B016A017901E8
:10DFF0000E94566FCE0101960E94185B89819A811A
:10E000000E94037646E050E06FE17BE089E090E01B
:10E010000E9433A1C50102960E94ED75C6010296C9
:10E020000E94FB75C70102960E94F4750E94027659
:10E03000F80182819381A481B58180932A0D909308
:10E040002B0DA0932C0DB0932D0D0F900F90DF9101
:10E05000CF911F910F91FF90EF90DF90CF90BF90E5
:10E06000AF900895CF92DF92EF92FF92CF93DF931C
:10E07000CDB7DEB768970FB6F894DEBF0FBECDBF41
:10E08000FA012CE834E03A8329835FEF5B835C83F9
:10E090005D831E8238872F83C280D380E480F58021
:10E0A000C986DA86EB86FC863E872D87FB01428196
:10E0B0005381648175814F87588B698B7A8B3C8B38
:10E0C0002B8BFC0182819381A481B5818D8B9E8BEA
:10E0D000AF8BB88F9E012F5F3F4FAE01495F5F4FFF
:10E0E000BE01635F7F4FCE0143960E94E66F689644
:10E0F0000FB6F894DEBF0FBECDBFDF91CF91FF907A
:10E10000EF90DF90CF9008950F931F93CF93DF93FD
:10E11000CDB7DEB768970FB6F894DEBF0FBECDBFA0
:10E12000FB01DC0112964D915D916D917C911597EB
:10E130004D8B5E8B6F8B788F8CE894E09A8389830C
:10E1400021E0288F0D891E892F89388D0B831C8330
:10E150002D833E8398878F830281138124813581AB
:10E1600009871A872B873C879E878D874F87588B17
:10E17000698B7A8BAE014F5F5F4FBE01695F7F4F46
:10E18000CE010D960E94327068960FB6F894DEBFED
:10E190000FBECDBFDF91CF911F910F910895CF9307
:10E1A000DF93CDB7DEB762970FB6F894DEBF0FBE30
:10E1B000CDBFFC0182819381A481B5818F87988B2B
:10E1C000A98BBA8B2CE834E03A83298341E04A8B4F
:10E1D0004F85588969897A894B835C836D837E83F7
:10E1E00038872F8389879A87AB87BC87BE016F5F8B
:10E1F0007F4FCE0107960E94847062960FB6F89406
:10E20000DEBF0FBECDBFDF91CF910895CF92DF92D9
:10E21000EF92FF920F931F93CF93DF936C01EB016B
:10E220007B0182E0E80EF11C00E010E0C601800FE7
:10E23000911F0E943BB5F70181937F010F5F1F4F34
:10E240000430110599F78A81882361F08F3F61F4CA
:10E250008B818F3F49F48C818F3F31F481E09D8128
:10E260009F3F19F480E001C081E090E0DF91CF9101
:10E270001F910F91FF90EF90DF90CF900895EF9254
:10E28000FF920F931F93CF93DF937C018B010E5F5F
:10E290001F4FC0E0D0E0F80161918F01C7018C0FE2
:10E2A0009D1F0E9443B52196C430D105A1F7DF918F
:10E2B000CF911F910F91FF90EF900895FC01DC0129
:10E2C0008D918111FDCF40E050E020E030E08AE008
:10E2D0009191992301F1243031055CF59E3271F45E
:10E2E0004F3F510509F02CF5DB01A20FB31F129629
:10E2F0004C932F5F3F4F40E050E0EACF849FD00126
:10E30000859FB00D1124492F990F550B405351098A
:10E310004A0F5B1FDDCF4F3F510509F054F4243005
:10E3200031053CF4FB01E20FF31F428381E090E0F2
:10E33000089580E090E00895EF92FF920F931F936D
:10E34000CF93DF936115710511F480E01CC0411576
:10E350005105C1F07B01EC018C819D818A01080F80
:10E36000191FB801CE010E946899882371F3288192
:10E3700039818C819D81B701820F931F0E9414BA4D
:10E380001D830C8381E0DF91CF911F910F91FF904E
:10E39000EF900895EF92FF920F931F93CF93DF9327
:10E3A000CDB7DEB729970FB6F894DEBF0FBECDBF4D
:10E3B0008C01862FF801118210821382128215823D
:10E3C000148240E19E012F5F3F4F7901B90190E037
:10E3D0000E942BADF70101900020E9F73197AF01C2
:10E3E0004E195F09B701C8010E948F9929960FB68F
:10E3F000F894DEBF0FBECDBFDF91CF911F910F917B
:10E40000FF90EF9008952F923F924F925F926F92FC
:10E410007F928F929F92AF92BF92CF92DF92EF92B4
:10E42000FF920F931F93CF93DF93CDB7DEB7E297A1
:10E430000FB6F894DEBF0FBECDBF7C012A013B01B1
:10E4400069010E9412994B015C0187010D5B1F4F0E
:10E45000C8010E94A37E18161906A4F00E94129902
:10E46000DC01CB0188199909AA09BB09481659068C
:10E470006A067B06D8F062E370E080E090E00E94DC
:10E480006563E6CF42E250E0BE016F5F7F4FC80197
:10E490000E945B7E8981823011F080E060C1F801CA
:10E4A0008489958983349105C1F702C08FEF57C1E4
:10E4B0006D817E818F8198850E94E0B54B015C0162
:10E4C000F601608371838283938346E050E0B70155
:10E4D000685F7F4FCE014D960E94BAB9892BE9F64D
:10E4E000F70180819181A281B38188169906AA06DD
:10E4F000BB0698F284819581A681B781881599051C
:10E50000AA05BB0550F289899A89AB89BC8986879F
:10E510009787A08BB18B8EECC82ED12CC8010E949E
:10E520007A7EF1E0CF1AD108C9F7712CC701829623
:10E530009AA789A7F701B696FCA7EBA708969EA70E
:10E540008DA73C974F01899698AB8FA73897FAAB68
:10E55000E9AB1701F6E12F0E311C27018EE1480EC1
:10E56000511CF801818D928D181619060CF0F6C019
:10E57000C8010E947A7E8333910509F4C9C0F4F47E
:10E5800081309105B9F11CF4892B59F3DBC083303C
:10E590009105C1F1069709F0D5C0C8010E947A7EA5
:10E5A0006C0144E050E0B201C8010E945B7EA12CE6
:10E5B000B12CDD2494E0C91AD1083FC08A339105FB
:10E5C00009F47AC03CF48533910561F0C69709F4EB
:10E5D0003FC0B8C08B33910509F484C08F3F9105CB
:10E5E00001F2B0C0C8010E947A7EC8010E947A7E02
:10E5F000782EB7CFC8010E947A7E44E050E069A926
:10E600007AA93AC0C8010E947A7E6C0144E050E0C9
:10E61000B101C8010E945B7EA12CB12CDD24F4E085
:10E62000CF1AD108AC14BD040CF09BCFC8010E94D6
:10E630007A7E8FEFA81AB80AF5CFAC14BD040CF09F
:10E6400090CFC8010E947A7EEFEFAE1ABE0AF5CFD6
:10E65000C8010E947A7E682EF701828D811110C058
:10E66000838D81110DC0848D81110AC0858D81112A
:10E6700007C044E050E0B401C8010E945B7E71CF46
:10E68000EFA5F8A9A080B180C280D380B401CE01EB
:10E6900083960E944C9C8DA19EA1AFA1B8A5A816FF
:10E6A000B906CA06DB0629F3662009F45ACFC80169
:10E6B0000E947A7E6A94F8CFC8010E947A7E44E074
:10E6C00050E06BA57CA5C8010E945B7EF70166A1A6
:10E6D00077A180A591A50E94E0B566A377A380A746
:10E6E00091A73FCFC8010E947A7E44E050E06DA51B
:10E6F0007EA5C8010E945B7EF70162A573A584A573
:10E7000095A50E94E0B562A773A784A795A729CF16
:10E71000C8010E947A7E44E050E069A57AA5C8014C
:10E720000E945B7EF70162A173A184A195A10E9462
:10E73000E0B562A373A384A395A366A777A780AB74
:10E7400091AB0FCFC8010E947A7ED82EDD2009F44C
:10E7500008CFC8010E947A7EDA94F8CF872DE2961E
:10E760000FB6F894DEBF0FBECDBFDF91CF911F91E2
:10E770000F91FF90EF90DF90CF90BF90AF909F9060
:10E780008F907F906F905F904F903F902F90089563
:10E790002F923F924F925F926F927F928F929F92B1
:10E7A000AF92BF92CF92DF92EF92FF920F931F939F
:10E7B000CF93DF9300D000D0CDB7DEB78C010E949D
:10E7C0003DAC2FEC37E040E050E00E9483B5DC0127
:10E7D000CB010196A11DB11DF80184839583A68309
:10E7E000B78380839183A283B3835801F3E4AF0E90
:10E7F000B11CC5010E94107D64E470E0C5010E9457
:10E800001C7F882309F436C10E9412992B013C0118
:10E81000812C912CC8018E5B9F4F9E838D8348EE87
:10E82000C42E43E0D42EE12CF12C52E0252EAD81F4
:10E83000BE818C91833009F404C1811120C0F8019C
:10E8400084819581A681B7810196A11DB11D848324
:10E850009583A683B7830E94129964197509860966
:10E860009709A70196010E9461B5A90161E0C8015D
:10E870000E948D6D81E0AD81BE818C93CAC08430D1
:10E88000F9F4F80184819581A681B7810196A11DD3
:10E89000B11D84839583A683B7830E94129964195E
:10E8A000750986099709A70196010E9461B5A9011A
:10E8B00063E0C8010E948D6DAD81BE812C92A9C01C
:10E8C000813059F5F80142AD53AD64AD75AD9E018F
:10E8D0002F5F3F4FC8010E940372382EF2E08F1362
:10E8E00092C089819A81AB81BC81F8018483958330
:10E8F000A683B7830E94129964197509860997093E
:10E90000A70196010E9461B5A90163E0C8010E94B8
:10E910008D6DAD81BE813C927CC0823009F079C0A2
:10E92000F80142AD53AD64AD75AD9E012F5F3F4F11
:10E93000C8010E940372382EF5E08F135DC0E3E03A
:10E94000AD81BE81EC93F80182A193A1A4A1B5A1F0
:10E95000892B8A2B8B2B41F484E893E0A0E0B0E074
:10E9600082A393A3A4A3B5A3F80186A197A1A0A510
:10E97000B1A5892B8A2B8B2B61F482A193A1A4A131
:10E98000B5A1B695A7959795879586A397A3A0A7B8
:10E99000B1A7F80182A593A5A4A5B5A5892B8A2BBB
:10E9A0008B2BA9F482A193A1A4A1B5A1AC01BD01B7
:10E9B00023E076956795579547952A95D1F7841B5F
:10E9C000950BA60BB70B82A793A7A4A7B5A7F80131
:10E9D00086A197A1A0A5B1A586A797A7A0ABB1AB2B
:10E9E00082A593A5A4A5B5A582AB93ABA4ABB5AB0B
:10E9F00088248394912C0DC0F6E08F1304C0AD8160
:10EA0000BE811C9206C0BFEF3B1203C0ED81FE81A8
:10EA10001082F1E08F16910409F409CF0E94129937
:10EA2000DC01CB0184199509A609B709F80126A9CB
:10EA300037A940AD51AD281739074A075B0708F0E1
:10EA4000F6CEC5010E94107DF80184819581A681D2
:10EA5000B7810196A11DB11D84839583A683B783D9
:10EA60000E941299F801FE966083718382839383DA
:10EA7000C40102C080E090E026960FB6F894DEBF95
:10EA80000FBECDBFDF91CF911F910F91FF90EF90FF
:10EA9000DF90CF90BF90AF909F908F907F906F90BE
:10EAA0005F904F903F902F900895CF93DF931F92E8
:10EAB000CDB7DEB76983DC01ED91FC910280F38173
:10EAC000E02D41E050E0BE016F5F7F4F19950F9040
:10EAD000DF91CF910895DC01ED91FC91068CF78DCB
:10EAE000E02D199591E089270895862F089581E0FA
:10EAF00086270895CF93DF931F92CDB7DEB7898322
:10EB00002091270B3981E091280BF091290B822F5E
:10EB100090E080959095F8940080082200824BE068
:10EB200000C05DE000005A95E9F7008008220894D3
:10EB3000379508F4022A00824A9599F778940F9045
:10EB4000DF91CF9108950F931F93CF93DF931F927F
:10EB5000CDB7DEB78C01DC01ED91FC910084F1852D
:10EB6000E02D1995892B51F0BE016F5F7F4FF801A1
:10EB700084850E948B7D898190E002C08FEF9FEF9A
:10EB80000F90DF91CF911F910F910895FC01848523
:10EB90000C94DC7DCF93DF931F92CDB7DEB741E0BD
:10EBA00050E0BE016F5F7F4FFC0184850E94DC7DD9
:10EBB000181619061CF4898190E002C08FEF9FEFB0
:10EBC0000F90DF91CF910895FC018485843011F07E
:10EBD0000C94E27B80E090E0089544E050E0BC01BA
:10EBE0008FE090E00C9433A144E050E0BC0185E05C
:10EBF00090E00C9433A144E050E0BC0181E090E04F
:10EC00000C9433A108958CBD9DBD08956F927F92A1
:10EC10008F929F92AF92BF92CF92DF92EF92FF922C
:10EC20001F93CF93DF931F921F92CDB7DEB75C0186
:10EC30003B016A01FC011485143041F481E090E04D
:10EC4000F5019383828380E090E05BC07A014130DC
:10EC5000584018F0E12C88E0F82ECE0101960E9471
:10EC6000185B89819A810E940376812F0E94FA6E37
:10EC70004C0163E070E0812F0E946D7D873111F0BF
:10EC80008C3121F48E149F0440F302C0E12CF12C4E
:10EC9000CE0101960E94185B89819A810E940376B9
:10ECA0009701A30160E070E0812F0E94956E60E201
:10ECB00070E0812F0E94085B62E070E0812F0E946B
:10ECC0006D7D84FD14C063E070E0812F0E946D7D36
:10ECD000811104C0812F0E94A17CB0CFCE0101968A
:10ECE0000E94185B89819A810E940376E5CF40E1FA
:10ECF00062E070E0812F0E94977CEF2809F49ECF9C
:10ED0000C6010F900F90DF91CF911F91FF90EF9070
:10ED1000DF90CF90BF90AF909F908F907F906F903B
:10ED200008958F929F92AF92BF92DF92EF92FF92DF
:10ED30000F931F93CF93DF931F921F92CDB7DEB730
:10ED4000FC012485243009F082C05A018B017C012A
:10ED5000D12C8D2D0E94FD7E811103C0F701D48638
:10ED600007C08B7F8831D1F3D394F4E0DF12F1CF69
:10ED7000F7018485843009F46AC020912B02309118
:10ED80002C022F5F3F4F11F420E030EC30932C0227
:10ED900020932B0240912B0250912C0220E061E045
:10EDA0000E94C47CF80182818F3F51F483818F3FA0
:10EDB00099F484818F3F81F485818F3F69F444C049
:10EDC00081110AC0F8018381811106C084818111FB
:10EDD00003C085818823C1F1A114B104A9F1F70111
:10EDE000D484CE0101960E94185B89819A810E9489
:10EDF0000376B8016E5F7F4F8D2D0E94A47FB50111
:10EE00008D2D0E94937F64E070E08D2D0E94085B41
:10EE10000E9412994B015C01F4E98F0EF1E19F1EF3
:10EE2000A11CB11CC7010E941D5B873141F161E04B
:10EE300070E080E090E00E9465630E948B82C701D1
:10EE40000E941D5B811106C084E0F701848780E089
:10EE500090E01DC00E94129986169706A806B90672
:10EE600008F7F70184850E94A17C84E0F70184877C
:10EE70006EE174E185E89CE00E9478A2E8CF63E14E
:10EE800074E185E89CE00E9478A281E090E00F9018
:10EE90000F90DF91CF911F910F91FF90EF90DF9036
:10EEA000BF90AF909F908F90089578941F920F928B
:10EEB0000FB60F9211240BB60F92CF92DF92EF9202
:10EEC000FF920F931F932F933F934F935F936F93F3
:10EED0007F938F939F93AF93BF93CF93DF93EF93E2
:10EEE000FF93809170008E7F809370000FE310E09D
:10EEF0008BE1E82EF12C9BE2C92ED12CC0912A0B7C
:10EF0000D0912B0B2097F9F40332110508F43BC084
:10EF100003521109E091280BF091290B9081209167
:10EF2000270B822F8095982390839BE0D701119720
:10EF3000F1F79150D9F78081822B8083C601019728
:10EF4000F1F780E00DC00B301105E8F00B5011090E
:10EF5000E0912C0BF0912D0BEC0FFD1F3197808170
:10EF60000E947A752196D0932B0BC0932A0B809127
:10EF7000290290912A028C179D0708F0BFCF1092AA
:10EF80002B0B10922A0B809170008160809370008F
:10EF9000FF91EF91DF91CF91BF91AF919F918F91B1
:10EFA0007F916F915F914F913F912F911F910F91A1
:10EFB000FF90EF90DF90CF900F900BBE0F900FBEA1
:10EFC0000F901F90189581E08093260B8091280266
:10EFD000282F30E0F901E353FD4EE491F0E0EE0F0D
:10EFE000FF1FEF55FE4E459154915093290B4093CE
:10EFF000280BF901E957FD4EE491E093270B61E0FE
:10F000000E94416283E08093B100E0E7F0E08081FC
:10F01000816080830895CF93DF931816190644F01A
:10F02000809170008E7F809370001092260B19C023
:10F03000EC0180912C0B90912D0B0E9469ABCE01BD
:10F04000C130D24014F080E092E090932A02809385
:10F0500029020E94D1AA90932D0B80932C0B892B0F
:10F0600029F410922A021092290208C08091260BDE
:10F07000811104C0DF91CF910C94E377DF91CF91A0
:10F080000895FF920F931F93CF93DF938C01F62E79
:10F090008091260B811102C00E94E377E80121973D
:10F0A000C11582E0D80798F48091290290912A0234
:10F0B0008017910718F4C8010E940B7880912C0BDF
:10F0C00090912D0B009719F0C80FD91FF882DF918E
:10F0D000CF911F910F91FF900895DC0180E0615066
:10F0E00040F09D91E82FE927F0E0ED5EFC4E849121
:10F0F000F6CF0895AF92BF92CF92DF92EF92FF9238
:10F100001F93CF93DF93EC010E9412996B017C0156
:10F1100028EEC20E23E0D21EE11CF11C8BE4A82EC7
:10F12000B12C0E9412996C157D058E059F0598F4EF
:10F1300060EFCE010E948068CE010E94E068182F27
:10F1400080FF11C0EF85F889309709F01995C50146
:10F150000197F1F7E6CF81E08A8367E877E085E8F9
:10F160009CE00E947EA3812FDF91CF911F91FF90A1
:10F17000EF90DF90CF90BF90AF9008950F931F93C3
:10F18000CF93DF93EC01162F042F0E947A7800238F
:10F1900019F0CE010E94F768CE010E947A6865EAF4
:10F1A00080E39DE00E94AB66612F80E39DE00E94BA
:10F1B000AB66CE01DF91CF911F910F910C946C68DB
:10F1C000EF92FF920F931F93CF93DF938C017B01FC
:10F1D00040E065E50E94BE78E70188E0E80EF11C9A
:10F1E000699140E0C8010E94BE78CE15DF05C1F7E5
:10F1F000DF91CF911F910F91FF90EF9008951F9392
:10F20000CF93DF93EC01162F0E947A78CE010E94F3
:10F210007A6862ED80E39DE00E94AB66612F70E04A
:10F220006095709584E0660F771F8A95E1F7612BF2
:10F2300080E39DE00E94AB66CE010E946C68CE0127
:10F240000E94E068181711F084E08A83DF91CF9163
:10F250001F9108951F93CF93DF93EC010E947A785A
:10F2600080FD2CC0CE010E94EC6860E0CE010E94BF
:10F27000FF78CE010E947A78CE010E947A6864EB12
:10F2800080E39DE00E94AB66CE010E946C68CE01D7
:10F290000E947A78182F82FF02C082E08A838881D8
:10F2A000882341F0CE010E94EC68682F6160CE0196
:10F2B0000E94FF7811FB882780F901C080E0DF9170
:10F2C000CF911F910895CF92DF92EF92FF920F930B
:10F2D0001F93CF93DF937C01EB018A01FC018581B1
:10F2E00096810E942A798823C9F1BE01F7018581A0
:10F2F00096810E94E07840E06EEBF701858196816F
:10F300000E94BE78E8016801F9E0CF0ED11CF70138
:10F3100005811681C8010E947A78C8010E947A6826
:10F3200066E980E39DE00E94AB66C8010E946C68BC
:10F33000C8010E947A7861EEC8010E948068C80105
:10F340000E94E0688993CC16DD0609F7F7018581F4
:10F3500096810E942A7991E0813009F090E0892F0E
:10F36000DF91CF911F910F91FF90EF90DF90CF90A1
:10F370000895CF93DF93EA010E946379882339F0DF
:10F3800068E0CE010E946D7891E02885281390E016
:10F39000892FDF91CF910895CF93DF93CDB7DEB75B
:10F3A00029970FB6F894DEBF0FBECDBFAE014F5FF9
:10F3B0005F4F0E94B979882389F08D818F3361F086
:10F3C00020F48F3159F489E00CC08F3519F08F3754
:10F3D00039F004C08BE005C08AE003C080E001C0C2
:10F3E0008CE029960FB6F894DEBF0FBECDBFDF913B
:10F3F000CF9108956F927F928F929F92AF92BF921A
:10F40000CF92DF92EF92FF920F931F93CF93DF93F0
:10F41000FC01248521119EC0872E762EEC010E94CE
:10F420002A79811108C062E977E085E89CE00E94B2
:10F430007EA38FEF90C0CE010E947A7840E060EF0B
:10F44000CE010E94BE78C12CD12C66246A94EE2491
:10F45000E394F12C0C2D06950695069510E08C2D65
:10F460008770570101C0AA0C8A95EAF78B85082E90
:10F47000000C990BC816D90634F4FE01E00FF11FF9
:10F4800093809A2006C099249394C816D90609F04F
:10F49000912CCE010E947A78CE010E947A6868E7AA
:10F4A00080E39DE00E94AB66911002C060E001C065
:10F4B00060E880E39DE00E94AB66CE010E946C682C
:10F4C000CE010E947A78282F2074982F907885FF9B
:10F4D00011C02223A9F042E050E0682F85E89CE0AB
:10F4E0000E94AE9B6EE977E085E89CE00E947EA3D7
:10F4F0008EEF31C0211104C0911104C06C2C08C0E2
:10F50000992331F0FE01E00FF11F83818A2907C0A2
:10F51000FE01E00FF11F8A2D80959381892383835B
:10F52000FFEFCF1ADF0A80E4C816D10409F092CFAA
:10F530006B86EFEF6E1202C081E08C87DE011396BE
:10F54000E72DF82D2B968D918193CA17DB07D9F7FC
:10F5500081E001C080E0DF91CF911F910F91FF907A
:10F56000EF90DF90CF90BF90AF909F908F907F9063
:10F570006F900895AF92BF92CF92DF92EF92FF9279
:10F580000F931F93CF93DF93CDB7DEB7AF970FB62F
:10F59000F894DEBF0FBECDBF7C015B016A010CE8B1
:10F5A00014E01A8309831B821C821D821E82CE01F5
:10F5B00009960E94127C1BA70AA71CA61DA61EA6C0
:10F5C0001FA680912A0D90912B0DA0912C0DB0912A
:10F5D0002D0D8EA39FA3A8A7B9A78B839C83AD8372
:10F5E000BE8318861F82AE01465D5F4FB501CE0116
:10F5F00001960E949F6381309105B1F4D701ED918E
:10F60000FC910684F785E02D1DA30CA38CA59DA578
:10F61000AEA5BFA58EA39FA3A8A7B9A7A601BE01AB
:10F620006C5D7F4FC7011995AF960FB6F894DEBF9A
:10F630000FBECDBFDF91CF911F910F91FF90EF9043
:10F64000DF90CF90BF90AF9008950895CF93DF9350
:10F650001F92CDB7DEB76983DC01ED91FC9102808A
:10F66000F381E02D41E050E0BE016F5F7F4F1995BF
:10F670000F90DF91CF910895FC01818D928D0895B7
:10F68000FC018489958908952CE834E0FC013183DC
:10F690002083FB014089518962897389FC0142837F
:10F6A0005383648375830895DC01ED91FC91048C90
:10F6B000F58DE02D199480E00895FC019485FB01FF
:10F6C0008485981303C081E0943009F480E00895A4
:10F6D00021E0FC018485843009F420E0822F089524
:10F6E00008958F929F92AF92BF92DF92EF92FF9216
:10F6F0000F931F93CF93DF931F921F92CDB7DEB767
:10F700007C014B018A01FC01A688B788D08CCE0110
:10F7100001960E94185B89819A810E9403768D2D43
:10F720000E94FA6E8017910720F48D2D0E94FA6EC8
:10F730008C019801A401B5018D2D0E94956E0E9447
:10F740000276F70186899789800F911F978B868BA8
:10F75000C8010F900F90DF91CF911F910F91FF90F3
:10F76000EF90DF90BF90AF909F908F900895CF93D0
:10F77000DF93FC0124852430D1F0EC010E941D5B55
:10F78000843181F0882371F0883161F08C3161F42B
:10F79000E881F9810084F185E02DCE01199521E001
:10F7A000892B19F420E001C021E0822F01C080E004
:10F7B000DF91CF9108958EBD00000DB407FEFDCFFF
:10F7C0008EB50895DF92EF92FF920F931F93CF9320
:10F7D000DF931F921F92CDB7DEB7D82ECE010196D0
:10F7E0000E94185B89819A810E940376E12CF12C9A
:10F7F0008D2D0E947DA18C01892B21F08D2D0E94E1
:10F800007DA17C010E151F0599F70E940276C801A3
:10F810000F900F90DF91CF911F910F91FF90EF907C
:10F82000DF900895FC011382128288EE93E0A0E03D
:10F83000B0E084839583A683B78386E793E09183C2
:10F8400080838CE894E097878687108A118A128AD1
:10F85000138A84E0808F0895AF92BF92CF92DF9297
:10F86000EF92FF920F931F93CF93DF93CDB7DEB745
:10F87000AF970FB6F894DEBF0FBECDBF7C015B0122
:10F880006A010CE814E01A8309831B821C821D8222
:10F890001E82CE0109960E94127C1BA70AA71CA6F5
:10F8A0001DA61EA61FA680912A0D90912B0DA0913A
:10F8B0002C0DB0912D0D8EA39FA3A8A7B9A78B8364
:10F8C0009C83AD83BE8318861F82AE01465D5F4F69
:10F8D000B501CE0101960E949F6381309105B1F47C
:10F8E000D701ED91FC910488F589E02D1DA30CA3AF
:10F8F0008CA59DA5AEA5BFA58EA39FA3A8A7B9A7BC
:10F90000A601BE016C5D7F4FC7011995AF960FB67A
:10F91000F894DEBF0FBECDBFDF91CF911F910F9145
:10F92000FF90EF90DF90CF90BF90AF9008959B0134
:10F9300090E00496982F8827642F820F931F0C94D1
:10F9400062A11F93CF93DF931F921F92CDB7DEB7B3
:10F95000182FCE0101960E94185B89819A810E941E
:10F96000037660E170E0812F0E94085B4FEF62E058
:10F9700070E0812F0E94977C0E9402760F900F907A
:10F98000DF91CF911F910895DF92EF92FF920F9335
:10F990001F93CF93DF931F921F92CDB7DEB7182F1F
:10F9A000D62E7A01022F0E94A17CCE0101960E94E0
:10F9B000185B89819A810E9403764D2D402B60E06F
:10F9C00070E0812F0E94977CE114F10459F4E090DB
:10F9D000360BF090370B8FEFE81AF80AF092370BDE
:10F9E000E092360B4F2D64E070E0812F0E94977CEF
:10F9F0004E2D65E070E0812F0E94977C61E070E001
:10FA0000812F0E94085B0E94027681E00F900F9088
:10FA1000DF91CF911F910F91FF90EF90DF900895AC
:10FA2000CF93DF93FC01808D843029F0EF010E9499
:10FA3000A17C84E0888FDF91CF910895CF92DF92EF
:10FA4000EF92FF920F931F93CF93DF931F921F921A
:10FA5000CDB7DEB7FC01F484F4E0FF1699F18C0118
:10FA6000CE0101960E94185B89819A810E940376DB
:10FA700068E070E08F2D0E94085B0E9402760E9471
:10FA800012996B017C01C8010E941D5B8823B9F0AB
:10FA900062E370E080E090E00E9465630E9412994A
:10FAA000DC01CB018C199D09AE09BF09883E93404A
:10FAB000A105B10540F3F80184850E94A17C84E092
:10FAC000F80184870F900F90DF91CF911F910F91D4
:10FAD000FF90EF90DF90CF900895CF93DF9390E069
:10FAE0000496982F8827EC01C60FD71F0E9401A10A
:10FAF0008FE00E94DB7B8D2F0E94DB7B8C2F0E948E
:10FB0000DB7B80E00E94DB7BC82F0E94FFA08C2F54
:10FB1000DF91CF910895CF92DF92FF920F931F93C1
:10FB2000CF93DF931F921F92CDB7DEB7F82E6B01F4
:10FB3000CE0101960E94185B89819A810E9403760A
:10FB400068E270E08F2D0E946D7D082F10E069E261
:10FB500070E08F2D0E946D7D702F6627682B21E04D
:10FB600030E0A6018F2D0E94645E0E94027681E043
:10FB700090E00F900F90DF91CF911F910F91FF9028
:10FB8000DF90CF900895CF93DF931F92CDB7DEB76C
:10FB9000FC01218D328D232B49F0BE016F5F7F4F19
:10FBA000808D0E948B7D898190E002C08FEF9FEF56
:10FBB0000F90DF91CF9108958F929F92BF92CF9235
:10FBC000DF92EF92FF920F931F93CF93DF931F92D9
:10FBD0001F92CDB7DEB7B82E6B017A01CE01019628
:10FBE0000E94185B89819A810E940376812C912C56
:10FBF0008B2D0E947DA18C01892B21F08B2D0E94E1
:10FC00007DA14C010815190599F70115110599F405
:10FC100063E070E08B2D0E946D7D8431D9F18823E3
:10FC2000C9F101E010E08C3111F400E010E0119511
:10FC3000019511092FC0E016F1060CF4870110168A
:10FC4000110644F568E270E08B2D0E946D7DE82E70
:10FC5000F12C69E270E08B2D0E946D7DFE2CEE246C
:10FC6000E82A9801A601B7018B2D0E94645EE00E80
:10FC7000F11E4F2D68E270E08B2D0E94977C4E2D77
:10FC800069E270E08B2D0E94977C60E470E08B2D20
:10FC90000E94085B0E940276C8010F900F90DF91CE
:10FCA000CF911F910F91FF90EF90DF90CF90BF9079
:10FCB0009F908F900895CF93DF93FC01218D328D1B
:10FCC0002115310519F48FEF9FEF11C0EC01421798
:10FCD000530708F0A901888D0E94DC7D18161906CB
:10FCE00094F7298D3A8D281B390B3A8F298FDF9194
:10FCF000CF9108950F931F93CF93DF931F92CDB7AA
:10FD0000DEB7FC01218D328D232B61F08C0141E0A7
:10FD100050E0BE016F5F7F4F808D0E94DC7D181622
:10FD200019061CF08FEF9FEF08C0F801818D928DAE
:10FD30000197928F818F898190E00F90DF91CF9111
:10FD40001F910F9108950F931F93CF93DF93CDB71A
:10FD5000DEB728970FB6F894DEBF0FBECDBF8C017B
:10FD6000D80159968D919C915A97892B41F0ED912C
:10FD7000FC910284F385E02DC8011995F1CFF801BB
:10FD8000808D0E94E27B1816190654F548E050E079
:10FD9000BE016F5F7F4FD80158968C910E94DC7D29
:10FDA00018161906FCF4D801509684E0FE0131962D
:10FDB00001900D928A95E1F78D8190E0982F882728
:10FDC0002E81820F911DF801958B848B8F8190E09D
:10FDD000982F88272885820F911D928F818F02C0CE
:10FDE00080E090E028960FB6F894DEBF0FBECDBF3E
:10FDF000DF91CF911F910F9108951F93CF93DF93C0
:10FE00001F921F92CDB7DEB7182FCE0101960E9428
:10FE1000185B89819A810E94037663E070E0812FEC
:10FE20000E946D7D182F0E940276812F0F900F90F7
:10FE3000DF91CF911F910895EF92FF921F93CF937F
:10FE4000DF93FC01208D243011F080E01CC07B0189
:10FE5000EC0110E0812F0E94FD7E811102C0188FFD
:10FE600005C08831E1F31F5F1430A1F7888D84301D
:10FE700061F3FD86EC861A8E198E20E0A70162E000
:10FE80000E94C47C81E0DF91CF911F91FF90EF90A1
:10FE900008951F93CF93DF931F921F92CDB7DEB7C4
:10FEA000FC01108DCE0101960E94185B89819A8118
:10FEB0000E94037660E270E0812F0E94085B62E09E
:10FEC00070E0812F0E946D7D84FD1DC062E070E0B6
:10FED000812F0E946D7D83FF0BC048E162E070E0DE
:10FEE000812F0E94977C0E94027680E090E015C0EE
:10FEF0000E940276CE0101960E94185B89819A8148
:10FF00000E940376DCCF40E162E070E0812F0E9426
:10FF1000977C0E94027681E090E00F900F90DF9135
:10FF2000CF911F910895CF93DF93C82FD62F472FDE
:10FF300060E170E00E94977C4D2F61E170E08C2FB2
:10FF4000DF91CF910C94977C90E0982F882744E024
:10FF500050E0845F9B4F0C9433A1BF92CF92DF920D
:10FF6000EF92FF920F931F93CF93DF9300D000D0B7
:10FF7000CDB7DEB7FC01208D243009F04CC06A01FA
:10FF80007B018C01B12C63E070E08B2D0E946D7DB4
:10FF9000811103C0F801B08E06C08831D9F3B39443
:10FFA000F4E0BF12F0CFF801808D8430A1F196E02B
:10FFB000ECE6F3E0DE01119601900D929A95E1F7DF
:10FFC000F70193819F779C8394819D8395819E8384
:10FFD000B7016E5F7F4F0E94A47FB601F801808D4C
:10FFE0000E94937FF801808D90E0982F882746E04B
:10FFF00050E0BE016F5F7F4F8A5F9B4F0E9433A12D
:020000021000EC
:10000000F801128E118E20E8A60162E0808D0E9418
:10001000C47C81E001C080E026960FB6F894DEBF74
:100020000FBECDBFDF91CF911F910F91FF90EF9049
:10003000DF90CF90BF900895DF92EF92FF920F93E1
:100040001F93CF93DF931F921F92CDB7DEB7FB01B3
:10005000DC0157961C921E9256972281211109C0ED
:100060002381211106C02481211103C0258122236F
:10007000F1F041155105D9F07A018F01FC01D08CC6
:10008000CE0101960E94185B89819A810E940376B5
:10009000B8016E5F7F4F8D2D0E94A47FB7018D2D1B
:1000A0000E94937F0E94027681E090E002C080E08F
:1000B00090E00F900F90DF91CF911F910F91FF90E3
:1000C000EF90DF900895A8950895A8950E94E01FED
:1000D000029724F00E94465C0E94C9290C94EF1EEE
:1000E00060E08DE00C94126261E08DE00C9412628D
:1000F000CF92DF92EF92FF920F931F93CF93DF93F4
:100100006C01EB0109900020E9F72197C61BD70B82
:10011000C032D10514F0CFE1D0E08B01E12CF12CFD
:10012000EC16FD0664F4F80161918F01C7018C0D96
:100130009D1D0E9443B5FFEFEF1AFF0AF1CF60E06B
:10014000C6018C0F9D1FDF91CF911F910F91FF90E2
:10015000EF90DF90CF900C9443B5CF93DF931F9235
:10016000CDB7DEB71982892B21F0FB016281738143
:1001700003C0BE016F5F7F4F86E390E00E947880EE
:1001800061ED74E185E89CE00E94199B0F90DF917E
:10019000CF910895CF93DF93C0E0D0E060E0CE012F
:1001A0000E9443B52196C11582E0D807B9F761ECEA
:1001B00074E185E89CE0DF91CF910C94199BEF925C
:1001C000FF920F931F93CF93DF931F92CDB7DEB7AC
:1001D0008B01CE0101969F938F9384E29BE09F93C6
:1001E0008F9383E29BE09F938F9382E29BE09F93A8
:1001F0008F9381E29BE09F938F9380E29BE09F939C
:100200008F938FE19BE09F938F9388EA97E09F9372
:100210008F93FB0183818F9382818F930E94BFBA5A
:100220000FB6F894DEBF0FBECDBF06977CF4F80181
:100230000281138163EE74E185E89CE00E94199BC2
:10024000B80185E89CE00E944A9C19C00E94CF41F9
:100250008FE1E82E8BE0F82E00E010E0F7016191CD
:100260007F01C8010E9443B50F5F1F4F0630110583
:10027000A9F765EF74E185E89CE00E94199B0F9057
:10028000DF91CF911F910F91FF90EF900895EF9222
:10029000FF920F931F93CF93DF93CDB7DEB72C97C9
:1002A0000FB6F894DEBF0FBECDBF8C017B018CE88A
:1002B00094E09A8389831B821C821D821E82988708
:1002C0008F8319861A861B861C86053011055CF003
:1002D000BE01695F7F4FF701808591850E945E7145
:1002E000892B09F052C0BE016F5F7F4F82E190E021
:1002F0000E943F71043011050CF44FC0BE01695FCC
:100300007F4FF701868197810E945E71892B09F4E6
:1003100044C0BE01695F7F4F8EE090E00E943F7154
:10032000BE01695F7F4FF701848195810E945E71F4
:10033000892BF1F1BE01695F7F4F8AE090E00E9456
:100340003F71BE01695F7F4FF701828193810E94F7
:100350005E71892BC1F1BE01695F7F4F86E090E03D
:100360000E943F716AEA74E185E89CE00E94199B53
:100370002C960FB6F894DEBF0FBECDBFDF91CF91A4
:100380001F910F91FF90EF900895BE01695F7F4F1D
:1003900082E190E00E943F71B1CFBE016F5F7F4F5D
:1003A0008EE090E00E943F71033011050CF0B8CF51
:1003B000BE016F5F7F4F8AE090E00E943F71023084
:1003C00011050CF0BECFBE016F5F7F4F86E090E05D
:1003D0000E943F710130110529F6BE016F5F7F4F0A
:1003E00086E090E00E943F7161EB74E185E89CE05B
:1003F0000E94199BB7CFCF93DF93CDB7DEB72C9771
:100400000FB6F894DEBF0FBECDBF1C821B821E82CA
:100410001D828FEF9FEF98878F838EE993E09A83F9
:10042000898388E490E09A8789871C861B8660E927
:1004300074E185E89CE00E94199B60913C0B7091EF
:100440003D0BCE0101960E94B8966FEFCE0101964A
:100450000E943C9E60E874E185E89CE00E94199B44
:100460002C960FB6F894DEBF0FBECDBFDF91CF91B3
:100470000895CF93DF93CDB7DEB769970FB6F894A1
:10048000DEBF0FBECDBF8FE290E09A838983FE016D
:10049000339687E1DF011D928A95E9F76BE674E1F7
:1004A00085E89CE00E94199BAE014E5F5F4F66E0BD
:1004B0008FE19BE00E94796A1E866CEB77E0CE01AB
:1004C00001960E94F5B9BE016F5F7F4F85E89CE001
:1004D0000E944A9CCE0101960E94166F1E8664EC13
:1004E00077E0CE0101960E94F5B9BE016F5F7F4FA4
:1004F00085E89CE00E944A9C6EEC77E0CE01019674
:100500000E9454A469960FB6F894DEBF0FBECDBF0B
:10051000DF91CF91089580914C0A8F5F80934C0AB0
:10052000A8950E94C92980914C0A815080934C0A59
:10053000089568E477E185E89CE00E94199B65E3F3
:1005400077E185E89CE00E94199B67E277E185E806
:100550009CE00E94199B6FE177E185E89CE00E9496
:10056000199B85E89CE00E94469C62E177E185E862
:100570009CE00E94199B62E077E185E89CE00E9484
:10058000199B66EF76E185E89CE00E94199B6FED70
:1005900076E185E89CE00E94199B6BEC76E185E8AA
:1005A0009CE00E94199B66EB76E185E89CE00E9446
:1005B000199B67EA76E185E89CE00E94199B6FE948
:1005C00076E185E89CE00E94199B64E976E185E884
:1005D0009CE00E94199B6AE876E185E89CE00E9415
:1005E000199B62E876E185E89CE00E94199B66E72A
:1005F00076E185E89CE00E94199B6CE576E185E850
:100600009CE00E94199B6DE376E185E89CE00E94E6
:10061000199B68E276E185E89CE00E94199B6BE1FA
:1006200076E185E89CE00E94199B6DE076E185E823
:100630009CE00E94199B61E076E185E89CE00E94C5
:10064000199B65EF75E185E89CE00E94199B85E8A0
:100650009CE00C94469CAF92BF92CF92DF92EF92B7
:10066000FF920F931F93CF93DF936C017B018A015D
:100670000E943BB581508E3FA0F45701C0E0D0E00E
:1006800001501109C017D1077CF4C6018C0F9D1FC2
:100690000E943BB5F50181935F01882329F02196E3
:1006A000F1CF80E090E005C0CE0DDF1D188281E023
:1006B00090E0DF91CF911F910F91FF90EF90DF902D
:1006C000CF90BF90AF900895882319F06EEF74E13A
:1006D00002C060E075E185E89CE00C94199BCF9323
:1006E000DF93CDB7DEB72C970FB6F894DEBF0FBE01
:1006F000CDBF60E574E185E89CE00E94199B85E828
:100700009CE00E94469C88E490E00E943BB58B37B9
:10071000A1F51C821B821E821D828FEF9FEF98879E
:100720008F838EE993E09A83898388E490E09A87A7
:1007300089871C861B860E942242CE0101960E9458
:10074000E75A90933D0B80933C0B892B19F463E39C
:1007500074E115C06CE274E185E89CE00E94199B8D
:1007600085E89CE00E94469C0E9475338FE09FE0E4
:100770000E941E7D81E090E00CC06FE374E185E88B
:100780009CE00E94199B85E89CE00E94469C80E0CA
:1007900090E02C960FB6F894DEBF0FBECDBFDF9170
:1007A000CF910895AF92BF92CF92DF92EF92FF92D6
:1007B0000F931F93CF93DF93CDB7DEB7C058D10906
:1007C0000FB6F894DEBF0FBECDBF8E010F5B1F4F7B
:1007D000D8011D921C92FE01ED5BFF4F2EE1DF015F
:1007E0001D922A95E9F70297CCF0FB016281738193
:1007F0004FE150E0C8010E9439BAB80186E190E0AB
:100800000E947880B80185E89CE00E944A9C6EEEC8
:1008100075E185E89CE00E94199B1BC040E250E016
:10082000B80186E190E00E942B83892BB1F440E26D
:1008300050E062EE75E1C8010E94E9AC64EC75E13C
:1008400085E89CE00E94199BB80185E89CE00E9425
:100850004A9C85E89CE00E94469C8091240B1F9254
:100860008F938091230B1F928F938091220B1F9265
:100870008F938091210B1F928F938091200B1F9259
:100880008F9380911F0B1F928F9380ED97E09F9322
:100890008F931F9280E48F93CE0101966C019F93FA
:1008A0008F930E9453BA60EB75E185E89CE00E944B
:1008B000199BB80185E89CE00E944A9CB60185E836
:1008C0009CE00E944A9C85E89CE00E94469C0FB6F2
:1008D000F894A895809160008861809360001092E0
:1008E00060000FBE7E0191E6E90EF11CD701139660
:1008F0001C921E92129788EE93E0A0E0B0E0F70100
:1009000084839583A683B78384E0848786E694E016
:100910009183808316870587108A178680E590E08B
:10092000928B818B158A67EC7EE986E490EA0E94BF
:100930005CAD8C010FB6F894DEBF0FBECDBF892B26
:10094000E1F183E090E00E94D1AAD8011D969C932A
:100950008E931C97FC01F182E0821282C7010E94F3
:10096000B77B882319F0C7010E941E7DD7011F960F
:100970006D917C9150975196AD90BC9052976115B6
:10098000710569F0CE0189589F4F0E944C9CA501CA
:10099000BE0169587F4FC7010E94917607C0F701D9
:1009A00065857685A501C7010E94BA7A18161906D1
:1009B0000CF498C0C8010E941FA000E010E0F701ED
:1009C000E388F48899E288E10FB6F894A8958093BB
:1009D00060000FBE909360000115110509F469C015
:1009E000F8ECEF16F10409F056C064EA75E185E809
:1009F0009CE00E94199BEB961FAE1EAEEB97ED9606
:100A00001FAE1EAEED978FEF9FEFEF969FAF8EAFAD
:100A1000EF9784EB93E0E9969FAF8EAFE997C158CB
:100A2000DF4F19830883CF57D040F8940E942242A9
:100A3000CE0189589F4F0E94E75A90933D0B8093B7
:100A40003C0B7894C8010E941FA080913C0B9091B0
:100A50003D0B892B79F46DE875E185E89CE00E94F7
:100A6000199B0E941299DC01CB018856954CAF4F1F
:100A7000BF4F2DC062E875E185E89CE00E94199B9C
:100A80000E9475336BE775E185E89CE00E94199B35
:100A900082E090E0C7C063E675E185E89CE00E94D3
:100AA000199B4AE050E0B70185E89CE00E943F9C1A
:100AB00006C060E575E185E89CE00E94199B0E94F4
:100AC0001299DC01CB0188579C4EAF4FBF4F8093EA
:100AD000380B9093390BA0933A0BB0933B0B85EFF7
:100AE0009FEFA0C0D7011D96BC901D971E96AC909D
:100AF000DF92CF928CE495E19F938F931F930F9396
:100B00000E94E5ADDF92CF9287E495E19F938F93AA
:100B10001F930F930E94E5ADD8011C96ED91FC91B7
:100B20001D9781E08283DF92CF9284E495E19F93C9
:100B30008F931F930F930E94E5ADD8011C96ED9102
:100B4000FC911D971282AF92BF928EE095E19F9328
:100B50008F931F930F930E94E5AD89E495E19F93D6
:100B60008F931F930F930E94E5ADF701148A138AA8
:100B7000D8011C96ED91FC911D97A080B1800FB615
:100B8000F894DEBF0FBECDBF83E3C82ED12CD501B4
:100B9000ED91FC910084F185E02DC50119954197F7
:100BA0005CF4B1E0CB1AD10839F064E170E080E088
:100BB00090E00E946563EBCF6E01F7E7CF0ED11C8A
:100BC000DF92CF9282E095E19F938F931F930F93D3
:100BD0000E9402AE0F900F900F900F900F900F9009
:100BE000019709F0ECCEF60180819181D7015496EE
:100BF0009C938E935397D12C80E08A3039F4BAE0DD
:100C0000DB1609F4DCCE9AE0D92E03C08D3009F052
:100C1000D82EC8010E94A7AD8F3F79F7C8010E9466
:100C20001FA0CDCEC058DF4F0FB6F894DEBF0FBE69
:100C3000CDBFDF91CF911F910F91FF90EF90DF908B
:100C4000CF90BF90AF9008950E94D28390934B0AAB
:100C500080934A0A8FE09FE00C941E7D8F929F92B2
:100C6000AF92BF92CF92DF92EF92FF920F931F93BA
:100C7000CF93DF9300D01F92CDB7DEB761307105FF
:100C800009F0F4C08C018091420B81110BC061E02E
:100C900078E185E89CE00E94199B85E89CE00E9431
:100CA000469CE4C06FEF77E085E89CE00E944A9C98
:100CB00082E00E9490A3E92EF12C60E170E0C70170
:100CC0000E9466A28FEFE816F10409F4C3C06BE03E
:100CD00078E085E89CE00E944A9C80E00E9490A316
:100CE000BC0180E090E00E941CB420E030E040E8CD
:100CF00057E30E947DB420E030E045E253E40E94D7
:100D00007DB420E030E040E252E40E940AB66B017C
:100D10007C0122E0AB01BC0185E89CE00E9477A544
:100D20006FE078E085E89CE00E944A9C81E00E94A8
:100D300090A3BC0180E090E00E941CB420E030E071
:100D400040E857E30E947DB420E030E048EC52E4F4
:100D50000E947DB44B015C0122E0AB01BC0185E83F
:100D60009CE00E9477A566E178E085E89CE00E941F
:100D70007EA328E138E0B701A601C8010E94B51F93
:100D80002BE138E0B501A401C8010E94B51F809194
:100D9000070A882309F46DC020E030E048EC51ECEC
:100DA000C701B6010E9417B487FD63C020E030E0A0
:100DB00048E452E4C701B6010E941FB718160CF4AC
:100DC00058C020E030E0A901C501B4010E9417B469
:100DD00087FD4FC020E030E048EC52E4C501B4018B
:100DE0000E941FB718160CF444C020E030E04AE718
:100DF00054E4C501B4010E947DB40E94F0B666506F
:100E00007F4F8F4F9F4F24EF822E99249394A12CD4
:100E1000B12CA50194010E9461B529831A8220E0BA
:100E200030E04AE754E4C701B6010E947DB40E9455
:100E3000F0B66E557D498F4F9F4FA50194010E94DA
:100E400061B52B831C82BE016F5F7F4F85E00E94DE
:100E50000EA30FC06EE178E085E89CE00E947EA3BF
:100E600061E080E39DE00E940E6803C080E090E0B6
:100E700002C084E690E00F900F900F900F90DF91EA
:100E8000CF911F910F91FF90EF90DF90CF90BF9087
:100E9000AF909F908F900895EF92FF920F931F93C2
:100EA000CF93DF93CDB7DEB760970FB6F894DEBF70
:100EB0000FBECDBF8091420B882369F062EE77E1CF
:100EC00085E89CE00E94199B85E89CE00E94469C76
:100ED00080E090E089C068E278E085E89CE00E94CC
:100EE0007EA30E944CA380E48093530D0E944CA3E8
:100EF00010E01B7F6091530D80E39DE00E947068BD
:100F000062E080E39DE00E94AB66612F80E39DE09C
:100F10000E94AB6660E080E39DE00E94AB6680E3E8
:100F20009DE00E9469686AE070E080E090E00E94C5
:100F3000656366E378E085E89CE00E944A9C8EEF5A
:100F40000E9490A340E150E0BC0185E89CE00E9433
:100F5000A89B85E89CE00E94469C69E478E085E8CF
:100F60009CE00E944A9C8FEF0E9490A340E150E0D9
:100F7000BC0185E89CE00E94A89B85E89CE00E945B
:100F8000469C66E578E085E89CE00E944A9C8BEFF1
:100F90000E9490A3182F092F8CEF0E9490A3F82E87
:100FA000E92E8DEF0E9490A39F938F93EF92FF9273
:100FB0000F931F938CE698E09F938F938E010F5FA2
:100FC0001F4F1F930F930E9490BAB80185E89CE0D1
:100FD0000E947EA381E08093420B0FB6F894DEBF9F
:100FE0000FBECDBF81E090E060960FB6F894DEBFF3
:100FF0000FBECDBFDF91CF911F910F91FF90EF906A
:1010000008950F931F93CF93DF93CDB7DEB7279744
:101010000FB6F894DEBF0FBECDBF8091070A8823BC
:1010200059F064EC77E185E89CE00E94199B85E823
:101030009CE00E94469CC6C061E083E00E94416241
:1010400060E083E00E9412626BE778E085E89CE054
:101050000E947EA30E944CA38091C6039091C70377
:10106000A091C803B091C90389839A83AB83BC83E1
:1010700080E39DE090933D0D80933C0D1E8280E1C6
:1010800097E22E812F5F2E830197D9F71D82BE0133
:101090006B5F7F4F80E20E94B9A2009741F431E07C
:1010A00020E08D81813809F430E0832F922F009762
:1010B00009F078C0BE016F5F7F4F8FEF0E940EA3D3
:1010C0001F8280E89EE32F812F5F2F830197D9F73E
:1010D000BE016B5F7F4F80E00E94B9A28D8180FFCF
:1010E00003C003E010E062C0BE016B5F7F4F80E091
:1010F0000E94B9A2892BA9F78D8184FFF2CF60915C
:101100003E0D80913C0D90913D0D0E947068809144
:101110003C0D90913D0DDC01ED91FC910190F08131
:10112000E02D64EF199580913C0D90913D0D0E944A
:101130006968811139C0BE016B5F7F4F81E00E94F9
:10114000B9A2009779F51D811F7810611D83609108
:101150003E0D80913C0D90913D0D0E9470688091F4
:101160003C0D90913D0DDC01ED91FC910190F081E1
:10117000E02D61E0199580913C0D90913D0DDC01D1
:10118000ED91FC910190F081E02D612F19958091F6
:101190003C0D90913D0D0E946968811105C000E0F1
:1011A00010E004C08C0102C002E010E0011511053E
:1011B00061F067E878E085E89CE00E944A9CC801FD
:1011C0000E9497A280E090E005C081E08093070A2A
:1011D00081E090E027960FB6F894DEBF0FBECDBF3A
:1011E000DF91CF911F910F910895AF92BF92CF924F
:1011F000DF92EF92FF920F931F93CF93DF93209193
:101200004E0A30914F0A2115310509F469C06A016F
:101210007B01BC01C9010E944BA2EC01009709F4BB
:101220005FC064E070E00E94E38B882309F45BC038
:10123000CE010E9469A5843031F50E9413A08C0173
:10124000892B19F085E0F80180870E9413A05C01CA
:10125000892B39F083E0F5018087C186D286E38649
:10126000F48688EC90E00E94E0A37C01B501C801FF
:101270000E94C3A3B701C8010E94C3A3B801CE0155
:101280000E94C3A330C064E0CE010E948AA28C01F8
:10129000009749F161E00E948AA25C0160E0C80108
:1012A0000E948AA2FC01C186D286E386F486F501FB
:1012B00081859285A385B485892B8A2B8B2B31F46C
:1012C000688179818AE998E00E9454A488EC90E0D2
:1012D000A0E0B0E0F50181879287A387B48703C0BF
:1012E00080E090E002C081E090E0DF91CF911F911B
:1012F0000F91FF90EF90DF90CF90BF90AF90089547
:101300002F923F924F925F926F927F928F929F9215
:10131000AF92BF92CF92DF92FF920F931F93CF9322
:10132000DF93CDB7DEB7C855D1090FB6F894DEBF4D
:101330000FBECDBF0E94129900913E0B10913F0B42
:101340002091400B3091410B601771078207930782
:1013500008F420C2E0914E0AF0914F0A309709F448
:1013600019C280914D0A8F5F80934D0A06811781C3
:10137000F12C0115110509F4E7C065E070E0C80122
:101380000E94E38B882309F4DBC064E0C8010E945B
:101390008AA26C01009709F4D3C00E9469A582302B
:1013A00008F4CEC061E0C8010E948AA2FC01F18469
:1013B000328462E0C8010E948AA2FC014184528406
:1013C0006384748463E0C8010E948AA2FC012185C1
:1013D00032854385548567962CAF3DAF4EAF5FAFE6
:1013E000679760E0C6010E948AA2FC018184928412
:1013F000A384B48461E0C6010E948AA2FC014185F5
:10140000528563857485411551056105710509F0A3
:10141000F5C0F8016081718185E89CE00E944A9CDA
:101420006AEB77E185E89CE00E94199B20E030E0C0
:1014300048E152E4C501B4010E941FB718163CF4FC
:10144000F8016081718185EB98E00E9454A4629656
:10145000FFAE629763963FAE6397C301B2010E94ED
:101460001EB42B013C0165962EAC3FAC6597F8018C
:101470000190F081E02D6996FFAFEEAF699785E8A6
:101480009CE00E94469C69966EAD7FAD699785E8A9
:101490009CE00E944A9C64EB77E185E89CE00E9416
:1014A000199B22E0B301A20185E89CE00E9477A588
:1014B0006EEA77E185E89CE00E94199B22E0B50185
:1014C000A40185E89CE00E9477A568EA77E185E8B9
:1014D0009CE00E94199B4AE050E065966EAD7FAD9E
:1014E000659785E89CE00E943F9C63962EAD3FADDA
:1014F000639761E08F2D37FD81950E94416261E025
:10150000C6010E948AA2FC0181859285A385B485CB
:10151000892B8A2B8B2B09F087C063962EAD3FADAC
:10152000639737FFD1C060E08F2D81950E941262D2
:1015300063EA77E185E89CE00E94199BFF24F3941D
:10154000F8010281138115CF80914D0A815080935B
:101550004D0A0E941299DC01CB01805D9A48AF4F81
:10156000BF4F80933E0B90933F0BA093400BB093E3
:10157000410B0E944C6A2B013C010E9412994B01C5
:101580005C010E94D491882329F080914C0A882321
:1015900009F49DC0FF20C9F00E944C6A4B015C0118
:1015A00065E877E185E89CE00E94199B2AE030E03D
:1015B000B501A40185E89CE00E949B9B68E978E066
:1015C00085E89CE00E944A9CE5C00E944C6A4B0161
:1015D0005C0163E877E185E89CE00E94199B2AE0C2
:1015E00030E0B501A40185E89CE00E949B9B61E886
:1015F00077E185E89CE00E94199BCCC041505109DD
:1016000061097109FC014187528763877487452B03
:10161000462B472B09F00ACFF8016081718189EAD6
:1016200098E00E9454A402CFF6E02F16310479F01E
:101630002CF42A94232809F070CF09C04AE024161C
:10164000310429F05CE02516310409F066CF20E072
:1016500030E040E85FE3C301B2010E940AB69B019B
:10166000AC01C501B4010E9417B487FF11C0639695
:101670008EAD9FAD639797FF04C060E08F2D81957D
:1016800002C061E08F2D0E9412626FE977E152CFB4
:10169000A5019401C301B2010E9417B418168CF081
:1016A0006396EEADFFAD6397F7FF04C061E08F2D49
:1016B000819502C060E08F2D0E9412626AE977E195
:1016C00039CF6BE877E136CF60E08F2D2FCF20E068
:1016D00030E041E050E060E4CE0101960E945E6996
:1016E00040E450E06AE777E1CE0101960E94CBAC7E
:1016F0006BE775E0CE0101960E94F5B940E450E039
:1017000061E777E1CE0101960E94CBACB301A20163
:10171000CE018F5B9F4F0E940369BE016F5B7F4FBD
:10172000CE0101960E943AA220E030E041E050E074
:1017300060E4CE0101960E945E6940E450E06AE7F1
:1017400077E1CE0101960E94CBAC6BE775E0CE014C
:1017500001960E94F5B940E450E06AE677E1CE01D7
:1017600001960E94CBACC501B40128EE33E040E005
:1017700050E00E9461B5BA01A901CE018F5B9F4F75
:101780000E940369BE016F5B7F4FCE0101960E94EC
:101790003AA200CFC85ADF4F0FB6F894DEBF0FBE93
:1017A000CDBFDF91CF911F910F91FF90DF90CF9030
:1017B000BF90AF909F908F907F906F905F904F9071
:1017C0003F902F9008950F931F93CF93DF93FC01C9
:1017D00020852530B9F48B01EC0160E00E948AA2DB
:1017E000FC0181859285A385B4850597A105B10586
:1017F00049F4CE010E9469A5282F30E081E020172E
:1018000031070CF480E0DF91CF911F910F91089583
:101810002F923F924F925F926F927F928F929F9200
:10182000AF92BF92CF92DF92EF92FF920F931F93EE
:10183000CF93DF93CDB7DEB7C555D1090FB6F89476
:10184000DEBF0FBECDBF80914D0A8F5F80934D0AE2
:10185000E0914E0AF0914F0A3097B1F0E680F780A0
:10186000C0904E0AD0904F0AC114D10469F0E1141F
:10187000F10451F0F70180858530B1F7C7010E946E
:1018800069A5823088F3B7C180914D0A8150809359
:101890004D0A80914A0A90914B0A039709F4E1C4DA
:1018A0000E941299C090470BD090480BE090490BD2
:1018B000F0904A0BC616D706E806F90608F0D1C420
:1018C00066961FAE669766246394712C6091450BF3
:1018D0007091460B6115710509F4C3C46696FFAD9E
:1018E0006697F111BEC4FB018085853009F068C19F
:1018F000CE01CA960E94BA5525968FAD259788309D
:1019000009F409C1893009F4DAC0843009F02FC123
:101910008091430B9091440B892B09F0C9C060E082
:1019200074E0CE01CA960E94BB1B892BC1F0CE0188
:10193000CA960E94051B6B017C0164E878E185E88A
:101940009CE00E94199B60E074E0CE01CA960E9460
:10195000491BB601CE01CA960E94B246A9C0CEACC0
:10196000DFACF6018085853009F05EC1C6010E94BA
:1019700069A5882E912CF2E08F1691040CF454C1C5
:101980007092440B6092430B60E070E0CE01CA9607
:101990000E941F1B5C0161E070E0CE01CA960E94AC
:1019A0001F1B7C01F5E08F1691040CF4ABC164E0C1
:1019B000C6010E948AA2FC01C184D28440E855E29B
:1019C00060E070E088EE9BE00E941D54A092F70D4D
:1019D00088EE9BE09093F60D8093F50D1092020F28
:1019E0001092040F1092030FF1E0CF16D10409F406
:1019F0003CC10CF420C192E0C916D10409F027C102
:101A0000F092F90DE092F80D7092FB0D6092FA0DD4
:101A100083E00E946651182F111158C1C090FC0D2F
:101A2000D090FD0DC6010D2C000CAA0BBB0B8983B9
:101A30009A83AB83BC8380E190E09E838D83ECAD81
:101A4000FDAD8080918066EB78E185E89CE00E94A6
:101A5000199BB40185E89CE00E944A9C6FEA78E1FA
:101A600085E89CE00E94199BBE016F5F7F4F85E86F
:101A70009CE00E940A1C0E94469CB601CE01CA96B8
:101A80000E94D2558090450B9090460BF4016281E4
:101A90007381CE0101960E94BA55892809F0F6C0DB
:101AA000CE0101960E94FD4F1092440B1092430B01
:101AB000CE01CA960E94695680ED97E062C080917F
:101AC000430B9091440B892B99F7CE01CA960E9443
:101AD000FD1BE82E60E074E0CE01CA960E94BB1B9D
:101AE000892B09F430C1CE01CA960E94051BF62E3F
:101AF00063E778E185E89CE00E94199B60E074E070
:101B0000CE01CA960E94491B4E2D6F2DCE01CA965A
:101B10000E940046CDCF8091430B9091440B892BBE
:101B200039F6CE01CA960E94FD1BE82E60E074E0F3
:101B3000CE01CA960E94BB1B892B09F4B9CFCE01F6
:101B4000CA960E94051BF62E69E178E185E89CE0C3
:101B50000E94199B60E074E0CE01CA960E94491B66
:101B60004E2D6F2DCE01CA960E94EF44A1CFCE011B
:101B7000CA960E94695661E070E0CE01CA960E9442
:101B800020556C01990FEE08FF08C114D104E1043F
:101B9000F10491F00E941299C60ED71EE81EF91E9C
:101BA000C092470BD092480BE092490BF0924A0B3F
:101BB000F1E06696FFAF6697CE01CA960E94FD4F90
:101BC000E091450BF091460B309709F44AC38281AE
:101BD00093819093460B8093450B892B09F076CE29
:101BE000E0914E0AF0914F0A868197819093460BBF
:101BF0008093450B36C3B701CE0101960E94BA55BA
:101C0000CE0101960E94C01A882331F062E070E094
